
output/main.elf:     file format elf32-littlearm


Disassembly of section .text:

08000000 <vector_table>:
 8000000:	00 30 00 20 65 16 00 08 61 16 00 08 5f 16 00 08     .0. e...a..._...
 8000010:	5f 16 00 08 5f 16 00 08 5f 16 00 08 00 00 00 00     _..._..._.......
	...
 800002c:	5d 02 00 08 61 16 00 08 00 00 00 00 61 02 00 08     ]...a.......a...
 800003c:	65 02 00 08 5f 16 00 08 5f 16 00 08 5f 16 00 08     e..._..._..._...
 800004c:	5f 16 00 08 5f 16 00 08 5f 16 00 08 5f 16 00 08     _..._..._..._...
 800005c:	5f 16 00 08 5f 16 00 08 5f 16 00 08 5f 16 00 08     _..._..._..._...
 800006c:	5f 16 00 08 5f 16 00 08 5f 16 00 08 5f 16 00 08     _..._..._..._...
 800007c:	5f 16 00 08 5f 16 00 08 5f 16 00 08 5f 16 00 08     _..._..._..._...
 800008c:	5f 16 00 08 5f 16 00 08 5f 16 00 08 5f 16 00 08     _..._..._..._...
 800009c:	5f 16 00 08 5f 16 00 08 5f 16 00 08 5f 16 00 08     _..._..._..._...
 80000ac:	5f 16 00 08 5f 16 00 08 5f 16 00 08 5f 16 00 08     _..._..._..._...
 80000bc:	5f 16 00 08 5f 16 00 08 5f 16 00 08 5f 16 00 08     _..._..._..._...
 80000cc:	5f 16 00 08 5f 16 00 08 5f 16 00 08 5f 16 00 08     _..._..._..._...
 80000dc:	5f 16 00 08 5f 16 00 08 5f 16 00 08 5f 16 00 08     _..._..._..._...
 80000ec:	5f 16 00 08 5f 16 00 08 5f 16 00 08 5f 16 00 08     _..._..._..._...
 80000fc:	5f 16 00 08 5f 16 00 08 5f 16 00 08 5f 16 00 08     _..._..._..._...
 800010c:	5f 16 00 08 5f 16 00 08 5f 16 00 08 5f 16 00 08     _..._..._..._...
 800011c:	5f 16 00 08 5f 16 00 08 5f 16 00 08 5f 16 00 08     _..._..._..._...
 800012c:	5f 16 00 08 5f 16 00 08 5f 16 00 08 5f 16 00 08     _..._..._..._...
 800013c:	5f 16 00 08 5f 16 00 08 5f 16 00 08 5f 16 00 08     _..._..._..._...
 800014c:	5f 16 00 08                                         _...

08000150 <vGetsTemp>:
  writeHEXc(val&0xff);
}

void vGetsTemp(void* dummy)
{
  volatile int i=0,k;
 8000150:	2300      	movs	r3, #0
{
 8000152:	b507      	push	{r0, r1, r2, lr}
  while(1){
    uart_puts("GetTemp\r\n");
 8000154:	4e12      	ldr	r6, [pc, #72]	; (80001a0 <vGetsTemp+0x50>)
#ifdef avec_mutex
    xSemaphoreTake(xMutex1, portMAX_DELAY);
 8000156:	4d13      	ldr	r5, [pc, #76]	; (80001a4 <vGetsTemp+0x54>)
    for (i=255;i>0;i--){
//      tempe[255-i]=readADC1(ADC_Channel_1);
        for (k=0x8fff;k>0;k--){}
    }
#ifdef avec_mutex
    xSemaphoreGive(xMutex2);
 8000158:	4c13      	ldr	r4, [pc, #76]	; (80001a8 <vGetsTemp+0x58>)
  volatile int i=0,k;
 800015a:	9300      	str	r3, [sp, #0]
    uart_puts("GetTemp\r\n");
 800015c:	4630      	mov	r0, r6
 800015e:	f000 f8d1 	bl	8000304 <uart_puts>
    xSemaphoreTake(xMutex1, portMAX_DELAY);
 8000162:	f04f 31ff 	mov.w	r1, #4294967295	; 0xffffffff
 8000166:	6828      	ldr	r0, [r5, #0]
 8000168:	f001 f83b 	bl	80011e2 <xQueueSemaphoreTake>
    for (i=255;i>0;i--){
 800016c:	23ff      	movs	r3, #255	; 0xff
        for (k=0x8fff;k>0;k--){}
 800016e:	f648 72ff 	movw	r2, #36863	; 0x8fff
    for (i=255;i>0;i--){
 8000172:	9300      	str	r3, [sp, #0]
 8000174:	9b00      	ldr	r3, [sp, #0]
 8000176:	2b00      	cmp	r3, #0
 8000178:	dc06      	bgt.n	8000188 <vGetsTemp+0x38>
    xSemaphoreGive(xMutex2);
 800017a:	2300      	movs	r3, #0
 800017c:	6820      	ldr	r0, [r4, #0]
 800017e:	461a      	mov	r2, r3
 8000180:	4619      	mov	r1, r3
 8000182:	f000 ff92 	bl	80010aa <xQueueGenericSend>
    uart_puts("GetTemp\r\n");
 8000186:	e7e9      	b.n	800015c <vGetsTemp+0xc>
        for (k=0x8fff;k>0;k--){}
 8000188:	9201      	str	r2, [sp, #4]
 800018a:	9b01      	ldr	r3, [sp, #4]
 800018c:	2b00      	cmp	r3, #0
 800018e:	dc03      	bgt.n	8000198 <vGetsTemp+0x48>
    for (i=255;i>0;i--){
 8000190:	9b00      	ldr	r3, [sp, #0]
 8000192:	3b01      	subs	r3, #1
 8000194:	9300      	str	r3, [sp, #0]
 8000196:	e7ed      	b.n	8000174 <vGetsTemp+0x24>
        for (k=0x8fff;k>0;k--){}
 8000198:	9b01      	ldr	r3, [sp, #4]
 800019a:	3b01      	subs	r3, #1
 800019c:	9301      	str	r3, [sp, #4]
 800019e:	e7f4      	b.n	800018a <vGetsTemp+0x3a>
 80001a0:	0800189c 	.word	0x0800189c
 80001a4:	2000001c 	.word	0x2000001c
 80001a8:	20000018 	.word	0x20000018

080001ac <vPrintUart>:
  }
}

/* Writes each 250 ms */
void vPrintUart(void* dummy)
{
 80001ac:	b5f7      	push	{r0, r1, r2, r4, r5, r6, r7, lr}
  int i=0;
  portTickType last_wakeup_time;
  last_wakeup_time = xTaskGetTickCount();
 80001ae:	f000 fb8b 	bl	80008c8 <xTaskGetTickCount>

  while(1){
    uart_puts("UART\r\n");
 80001b2:	4f0d      	ldr	r7, [pc, #52]	; (80001e8 <vPrintUart+0x3c>)
#ifdef avec_mutex
    xSemaphoreTake(xMutex2, portMAX_DELAY);
 80001b4:	4e0d      	ldr	r6, [pc, #52]	; (80001ec <vPrintUart+0x40>)
    for (i=255;i>0;i--){
   //   writeHEXi(tempe[255-i]);uart_putc(' ');
      vTaskDelayUntil(&last_wakeup_time, 1/portTICK_RATE_MS);
    }
#ifdef avec_mutex
    xSemaphoreGive(xMutex1);
 80001b6:	4d0e      	ldr	r5, [pc, #56]	; (80001f0 <vPrintUart+0x44>)
  last_wakeup_time = xTaskGetTickCount();
 80001b8:	9001      	str	r0, [sp, #4]
    uart_puts("UART\r\n");
 80001ba:	4638      	mov	r0, r7
 80001bc:	f000 f8a2 	bl	8000304 <uart_puts>
    xSemaphoreTake(xMutex2, portMAX_DELAY);
 80001c0:	f04f 31ff 	mov.w	r1, #4294967295	; 0xffffffff
 80001c4:	6830      	ldr	r0, [r6, #0]
 80001c6:	f001 f80c 	bl	80011e2 <xQueueSemaphoreTake>
 80001ca:	24ff      	movs	r4, #255	; 0xff
      vTaskDelayUntil(&last_wakeup_time, 1/portTICK_RATE_MS);
 80001cc:	2101      	movs	r1, #1
 80001ce:	a801      	add	r0, sp, #4
 80001d0:	f000 fcbc 	bl	8000b4c <xTaskDelayUntil>
    for (i=255;i>0;i--){
 80001d4:	3c01      	subs	r4, #1
 80001d6:	d1f9      	bne.n	80001cc <vPrintUart+0x20>
    xSemaphoreGive(xMutex1);
 80001d8:	4623      	mov	r3, r4
 80001da:	4622      	mov	r2, r4
 80001dc:	4621      	mov	r1, r4
 80001de:	6828      	ldr	r0, [r5, #0]
 80001e0:	f000 ff63 	bl	80010aa <xQueueGenericSend>
    uart_puts("UART\r\n");
 80001e4:	e7e9      	b.n	80001ba <vPrintUart+0xe>
 80001e6:	bf00      	nop
 80001e8:	080018a6 	.word	0x080018a6
 80001ec:	20000018 	.word	0x20000018
 80001f0:	2000001c 	.word	0x2000001c

080001f4 <main>:

  }
}


int main(void){
 80001f4:	b507      	push	{r0, r1, r2, lr}
//  Led_Init();
  Usart1_Init();
 80001f6:	f000 f851 	bl	800029c <Usart1_Init>

  GPIO_InitStructure . GPIO_Pin = GPIO_Pin_10 ;
  GPIO_InitStructure . GPIO_Mode = GPIO_Mode_IN_FLOATING ;
  GPIO_Init (GPIOA, &GPIO_InitStructure );
*/
  initADC1(); // Configure ADC1
 80001fa:	f000 f88c 	bl	8000316 <initADC1>

#ifdef avec_mutex
  xMutex1 = xSemaphoreCreateMutex();
 80001fe:	2001      	movs	r0, #1
 8000200:	f000 ffdd 	bl	80011be <xQueueCreateMutex>
 8000204:	4b0f      	ldr	r3, [pc, #60]	; (8000244 <main+0x50>)
  xMutex2 = xSemaphoreCreateMutex();
#endif

  if (!(pdPASS == xTaskCreate( vGetsTemp, (signed char*) "LedFloat",128,NULL,10,NULL ))) goto hell;
 8000206:	2400      	movs	r4, #0
  xMutex1 = xSemaphoreCreateMutex();
 8000208:	6018      	str	r0, [r3, #0]
  xMutex2 = xSemaphoreCreateMutex();
 800020a:	2001      	movs	r0, #1
 800020c:	f000 ffd7 	bl	80011be <xQueueCreateMutex>
  if (!(pdPASS == xTaskCreate( vGetsTemp, (signed char*) "LedFloat",128,NULL,10,NULL ))) goto hell;
 8000210:	250a      	movs	r5, #10
  xMutex2 = xSemaphoreCreateMutex();
 8000212:	4b0d      	ldr	r3, [pc, #52]	; (8000248 <main+0x54>)
  if (!(pdPASS == xTaskCreate( vGetsTemp, (signed char*) "LedFloat",128,NULL,10,NULL ))) goto hell;
 8000214:	2280      	movs	r2, #128	; 0x80
  xMutex2 = xSemaphoreCreateMutex();
 8000216:	6018      	str	r0, [r3, #0]
  if (!(pdPASS == xTaskCreate( vGetsTemp, (signed char*) "LedFloat",128,NULL,10,NULL ))) goto hell;
 8000218:	490c      	ldr	r1, [pc, #48]	; (800024c <main+0x58>)
 800021a:	4623      	mov	r3, r4
 800021c:	e9cd 5400 	strd	r5, r4, [sp]
 8000220:	480b      	ldr	r0, [pc, #44]	; (8000250 <main+0x5c>)
 8000222:	f000 fa43 	bl	80006ac <xTaskCreate>
 8000226:	2801      	cmp	r0, #1
 8000228:	d10b      	bne.n	8000242 <main+0x4e>
  if (!(pdPASS == xTaskCreate( vPrintUart, (signed char*) "Uart",   128,NULL,10,NULL ))) goto hell;
 800022a:	4623      	mov	r3, r4
 800022c:	2280      	movs	r2, #128	; 0x80
 800022e:	e9cd 5400 	strd	r5, r4, [sp]
 8000232:	4908      	ldr	r1, [pc, #32]	; (8000254 <main+0x60>)
 8000234:	4808      	ldr	r0, [pc, #32]	; (8000258 <main+0x64>)
 8000236:	f000 fa39 	bl	80006ac <xTaskCreate>
 800023a:	2801      	cmp	r0, #1
 800023c:	d101      	bne.n	8000242 <main+0x4e>

  vTaskStartScheduler();
 800023e:	f000 fb09 	bl	8000854 <vTaskStartScheduler>

 hell:              // should never be reached
  while(1);
 8000242:	e7fe      	b.n	8000242 <main+0x4e>
 8000244:	2000001c 	.word	0x2000001c
 8000248:	20000018 	.word	0x20000018
 800024c:	080018ad 	.word	0x080018ad
 8000250:	08000151 	.word	0x08000151
 8000254:	080018b6 	.word	0x080018b6
 8000258:	080001ad 	.word	0x080001ad

0800025c <sv_call_handler>:
//
//The only significant change to make is to redirect the sv, pendsv and systick libopencm3 interrupt handlers to those used by FreeRTOS:

void sv_call_handler(void)
{
      vPortSVCHandler();
 800025c:	f000 b920 	b.w	80004a0 <vPortSVCHandler>

08000260 <pend_sv_handler>:
}
 void pend_sv_handler(void)
{
      xPortPendSVHandler();
 8000260:	f000 b94e 	b.w	8000500 <xPortPendSVHandler>

08000264 <sys_tick_handler>:
}
void sys_tick_handler(void)
{
      xPortSysTickHandler();
 8000264:	f000 b96e 	b.w	8000544 <xPortSysTickHandler>

08000268 <clock_setup>:
int _write(int file, char *ptr, int len);
#endif


void clock_setup(void)
{
 8000268:	b508      	push	{r3, lr}
#ifdef STM32F1
#ifdef STM32F10X_LD_VL
 rcc_clock_setup_in_hse_8mhz_out_24mhz();  // STM32F100 discovery
 800026a:	f001 f961 	bl	8001530 <rcc_clock_setup_in_hse_8mhz_out_24mhz>
#endif
#else  // F4
 // rcc_clock_setup_hse_3v3(&rcc_hse_8mhz_3v3[RCC_CLOCK_3V3_168MHZ]); 
  core_clock_setup();
#endif
  rcc_periph_clock_enable(RCC_GPIOC); // Enable GPIOC clock
 800026e:	f44f 7041 	mov.w	r0, #772	; 0x304
 8000272:	f001 f999 	bl	80015a8 <rcc_periph_clock_enable>
  rcc_periph_clock_enable(RCC_GPIOD); // Enable GPIOD clock for F4 (LEDs)
 8000276:	f240 3005 	movw	r0, #773	; 0x305
 800027a:	f001 f995 	bl	80015a8 <rcc_periph_clock_enable>
  rcc_periph_clock_enable(RCC_GPIOA); // Enable GPIOA clock
 800027e:	f240 3002 	movw	r0, #770	; 0x302
 8000282:	f001 f991 	bl	80015a8 <rcc_periph_clock_enable>
#ifdef usart1
  rcc_periph_clock_enable(RCC_USART1);
 8000286:	f240 300e 	movw	r0, #782	; 0x30e
 800028a:	f001 f98d 	bl	80015a8 <rcc_periph_clock_enable>
#else
  rcc_periph_clock_enable(RCC_USART2);
#endif
  rcc_periph_clock_enable(RCC_ADC1);  // exemple ADC
}
 800028e:	e8bd 4008 	ldmia.w	sp!, {r3, lr}
  rcc_periph_clock_enable(RCC_ADC1);  // exemple ADC
 8000292:	f240 3009 	movw	r0, #777	; 0x309
 8000296:	f001 b987 	b.w	80015a8 <rcc_periph_clock_enable>
	...

0800029c <Usart1_Init>:


void Usart1_Init(void)
{ // Setup GPIO pin GPIO_USART1_TX/GPIO9 on GPIO port A for transmit. */
 800029c:	b510      	push	{r4, lr}
  gpio_set_af (GPIOA, GPIO_AF7, GPIO9);
  gpio_set_af (GPIOA, GPIO_AF7, GPIO10);
#endif

#ifdef usart1
  usart_set_baudrate(USART1, 115200);
 800029e:	4c14      	ldr	r4, [pc, #80]	; (80002f0 <Usart1_Init+0x54>)
  clock_setup();
 80002a0:	f7ff ffe2 	bl	8000268 <clock_setup>
  gpio_set_mode(GPIOA, GPIO_MODE_OUTPUT_50_MHZ,
 80002a4:	f44f 7300 	mov.w	r3, #512	; 0x200
 80002a8:	2202      	movs	r2, #2
 80002aa:	2103      	movs	r1, #3
 80002ac:	4811      	ldr	r0, [pc, #68]	; (80002f4 <Usart1_Init+0x58>)
 80002ae:	f001 f85b 	bl	8001368 <gpio_set_mode>
  usart_set_baudrate(USART1, 115200);
 80002b2:	4620      	mov	r0, r4
 80002b4:	f44f 31e1 	mov.w	r1, #115200	; 0x1c200
 80002b8:	f001 f984 	bl	80015c4 <usart_set_baudrate>
  usart_set_databits(USART1, 8);
 80002bc:	4620      	mov	r0, r4
 80002be:	2108      	movs	r1, #8
 80002c0:	f001 f994 	bl	80015ec <usart_set_databits>
  usart_set_stopbits(USART1, USART_STOPBITS_1);
 80002c4:	4620      	mov	r0, r4
 80002c6:	2100      	movs	r1, #0
 80002c8:	f001 f999 	bl	80015fe <usart_set_stopbits>
  usart_set_mode(USART1, USART_MODE_TX);
 80002cc:	4620      	mov	r0, r4
 80002ce:	2108      	movs	r1, #8
 80002d0:	f001 f9a1 	bl	8001616 <usart_set_mode>
  usart_set_parity(USART1, USART_PARITY_NONE);
 80002d4:	4620      	mov	r0, r4
 80002d6:	2100      	movs	r1, #0
 80002d8:	f001 f997 	bl	800160a <usart_set_parity>
  usart_set_flow_control(USART1, USART_FLOWCONTROL_NONE);
 80002dc:	4620      	mov	r0, r4
 80002de:	2100      	movs	r1, #0
 80002e0:	f001 f99f 	bl	8001622 <usart_set_flow_control>
  usart_enable(USART1);  // PA9 & PA10 for USART1
 80002e4:	4620      	mov	r0, r4
  usart_set_mode(USART2, USART_MODE_TX);
  usart_set_parity(USART2, USART_PARITY_NONE);
  usart_set_flow_control(USART2, USART_FLOWCONTROL_NONE);
  usart_enable(USART2);
#endif
}
 80002e6:	e8bd 4010 	ldmia.w	sp!, {r4, lr}
  usart_enable(USART1);  // PA9 & PA10 for USART1
 80002ea:	f001 b9a0 	b.w	800162e <usart_enable>
 80002ee:	bf00      	nop
 80002f0:	40013800 	.word	0x40013800
 80002f4:	40010800 	.word	0x40010800

080002f8 <uart_putc>:
  errno = EIO;
  return -1;
}
#endif

void uart_putc(char c) {
 80002f8:	4601      	mov	r1, r0
#ifdef usart1
usart_send_blocking(USART1, c); // USART1: send byte
 80002fa:	4801      	ldr	r0, [pc, #4]	; (8000300 <uart_putc+0x8>)
 80002fc:	f001 b99c 	b.w	8001638 <usart_send_blocking>
 8000300:	40013800 	.word	0x40013800

08000304 <uart_puts>:
usart_send_blocking(USART2, c); // USART2: send byte
#endif
}

/* Writes a zero teminated string over the serial line*/
void uart_puts(char *c) {while(*c!=0) uart_putc(*(c++));}
 8000304:	b510      	push	{r4, lr}
 8000306:	1e44      	subs	r4, r0, #1
 8000308:	f814 0f01 	ldrb.w	r0, [r4, #1]!
 800030c:	b900      	cbnz	r0, 8000310 <uart_puts+0xc>
 800030e:	bd10      	pop	{r4, pc}
 8000310:	f7ff fff2 	bl	80002f8 <uart_putc>
 8000314:	e7f8      	b.n	8000308 <uart_puts+0x4>

08000316 <initADC1>:
}

void initADC1(void)
{ 
 // TODO
}
 8000316:	4770      	bx	lr

08000318 <pvPortMalloc>:
        pxIterator->pxNextFreeBlock = pxBlockToInsert;                                                                              \
    }
/*-----------------------------------------------------------*/

void * pvPortMalloc( size_t xWantedSize )
{
 8000318:	b5f8      	push	{r3, r4, r5, r6, r7, lr}
 800031a:	4604      	mov	r4, r0
    BlockLink_t * pxNewBlockLink;
    PRIVILEGED_DATA static BaseType_t xHeapHasBeenInitialised = pdFALSE;
    void * pvReturn = NULL;
    size_t xAdditionalRequiredSize;

    vTaskSuspendAll();
 800031c:	f000 facc 	bl	80008b8 <vTaskSuspendAll>
    {
        /* If this is the first call to malloc then the heap will require
         * initialisation to setup the list of free blocks. */
        if( xHeapHasBeenInitialised == pdFALSE )
 8000320:	482b      	ldr	r0, [pc, #172]	; (80003d0 <pvPortMalloc+0xb8>)
 8000322:	6801      	ldr	r1, [r0, #0]
 8000324:	b971      	cbnz	r1, 8000344 <pvPortMalloc+0x2c>
     * blocks.  The void cast is used to prevent compiler warnings. */
    xStart.pxNextFreeBlock = ( void * ) pucAlignedHeap;
    xStart.xBlockSize = ( size_t ) 0;

    /* xEnd is used to mark the end of the list of free blocks. */
    xEnd.xBlockSize = configADJUSTED_HEAP_SIZE;
 8000326:	f241 35f8 	movw	r5, #5112	; 0x13f8
    pucAlignedHeap = ( uint8_t * ) ( ( ( portPOINTER_SIZE_TYPE ) & ucHeap[ portBYTE_ALIGNMENT - 1 ] ) & ( ~( ( portPOINTER_SIZE_TYPE ) portBYTE_ALIGNMENT_MASK ) ) );
 800032a:	4b2a      	ldr	r3, [pc, #168]	; (80003d4 <pvPortMalloc+0xbc>)
    xStart.pxNextFreeBlock = ( void * ) pucAlignedHeap;
 800032c:	4a2a      	ldr	r2, [pc, #168]	; (80003d8 <pvPortMalloc+0xc0>)
    pucAlignedHeap = ( uint8_t * ) ( ( ( portPOINTER_SIZE_TYPE ) & ucHeap[ portBYTE_ALIGNMENT - 1 ] ) & ( ~( ( portPOINTER_SIZE_TYPE ) portBYTE_ALIGNMENT_MASK ) ) );
 800032e:	f023 0307 	bic.w	r3, r3, #7
    xStart.xBlockSize = ( size_t ) 0;
 8000332:	e9c2 3100 	strd	r3, r1, [r2]
    xEnd.xBlockSize = configADJUSTED_HEAP_SIZE;
 8000336:	4a29      	ldr	r2, [pc, #164]	; (80003dc <pvPortMalloc+0xc4>)

    /* To start with there is a single free block that is sized to take up the
     * entire heap space. */
    pxFirstFreeBlock = ( BlockLink_t * ) pucAlignedHeap;
    pxFirstFreeBlock->xBlockSize = configADJUSTED_HEAP_SIZE;
    pxFirstFreeBlock->pxNextFreeBlock = &xEnd;
 8000338:	e9c3 2500 	strd	r2, r5, [r3]
            xHeapHasBeenInitialised = pdTRUE;
 800033c:	2301      	movs	r3, #1
    xEnd.pxNextFreeBlock = NULL;
 800033e:	e9c2 1500 	strd	r1, r5, [r2]
            xHeapHasBeenInitialised = pdTRUE;
 8000342:	6003      	str	r3, [r0, #0]
        if( xWantedSize > 0 )
 8000344:	2c00      	cmp	r4, #0
 8000346:	d040      	beq.n	80003ca <pvPortMalloc+0xb2>
            xAdditionalRequiredSize = heapSTRUCT_SIZE + portBYTE_ALIGNMENT - ( xWantedSize & portBYTE_ALIGNMENT_MASK );
 8000348:	f004 0207 	and.w	r2, r4, #7
            if( heapADD_WILL_OVERFLOW( xWantedSize, xAdditionalRequiredSize ) == 0 )
 800034c:	f1a2 0311 	sub.w	r3, r2, #17
 8000350:	42a3      	cmp	r3, r4
 8000352:	d33a      	bcc.n	80003ca <pvPortMalloc+0xb2>
 8000354:	3410      	adds	r4, #16
                xWantedSize += xAdditionalRequiredSize;
 8000356:	1aa0      	subs	r0, r4, r2
        if( heapBLOCK_SIZE_IS_VALID( xWantedSize ) != 0 )
 8000358:	2800      	cmp	r0, #0
 800035a:	dd36      	ble.n	80003ca <pvPortMalloc+0xb2>
            if( ( xWantedSize > 0 ) && ( xWantedSize <= xFreeBytesRemaining ) )
 800035c:	f8df c080 	ldr.w	ip, [pc, #128]	; 80003e0 <pvPortMalloc+0xc8>
 8000360:	f8dc 6000 	ldr.w	r6, [ip]
 8000364:	4286      	cmp	r6, r0
 8000366:	d330      	bcc.n	80003ca <pvPortMalloc+0xb2>
                pxBlock = xStart.pxNextFreeBlock;
 8000368:	491b      	ldr	r1, [pc, #108]	; (80003d8 <pvPortMalloc+0xc0>)
 800036a:	680b      	ldr	r3, [r1, #0]
                while( ( pxBlock->xBlockSize < xWantedSize ) && ( pxBlock->pxNextFreeBlock != NULL ) )
 800036c:	685f      	ldr	r7, [r3, #4]
 800036e:	4287      	cmp	r7, r0
 8000370:	d201      	bcs.n	8000376 <pvPortMalloc+0x5e>
 8000372:	681d      	ldr	r5, [r3, #0]
 8000374:	bb35      	cbnz	r5, 80003c4 <pvPortMalloc+0xac>
                if( pxBlock != &xEnd )
 8000376:	4d19      	ldr	r5, [pc, #100]	; (80003dc <pvPortMalloc+0xc4>)
 8000378:	42ab      	cmp	r3, r5
 800037a:	d026      	beq.n	80003ca <pvPortMalloc+0xb2>
                    if( ( pxBlock->xBlockSize - xWantedSize ) > heapMINIMUM_BLOCK_SIZE )
 800037c:	1b12      	subs	r2, r2, r4
                    pvReturn = ( void * ) ( ( ( uint8_t * ) pxPreviousBlock->pxNextFreeBlock ) + heapSTRUCT_SIZE );
 800037e:	680d      	ldr	r5, [r1, #0]
                    pxPreviousBlock->pxNextFreeBlock = pxBlock->pxNextFreeBlock;
 8000380:	f8d3 e000 	ldr.w	lr, [r3]
                    if( ( pxBlock->xBlockSize - xWantedSize ) > heapMINIMUM_BLOCK_SIZE )
 8000384:	443a      	add	r2, r7
 8000386:	2a10      	cmp	r2, #16
                    pvReturn = ( void * ) ( ( ( uint8_t * ) pxPreviousBlock->pxNextFreeBlock ) + heapSTRUCT_SIZE );
 8000388:	f105 0508 	add.w	r5, r5, #8
                    pxPreviousBlock->pxNextFreeBlock = pxBlock->pxNextFreeBlock;
 800038c:	f8c1 e000 	str.w	lr, [r1]
                    if( ( pxBlock->xBlockSize - xWantedSize ) > heapMINIMUM_BLOCK_SIZE )
 8000390:	d90b      	bls.n	80003aa <pvPortMalloc+0x92>
                        pxNewBlockLink = ( void * ) ( ( ( uint8_t * ) pxBlock ) + xWantedSize );
 8000392:	1819      	adds	r1, r3, r0
                        pxNewBlockLink->xBlockSize = pxBlock->xBlockSize - xWantedSize;
 8000394:	604a      	str	r2, [r1, #4]
                        pxBlock->xBlockSize = xWantedSize;
 8000396:	6058      	str	r0, [r3, #4]
                        prvInsertBlockIntoFreeList( ( pxNewBlockLink ) );
 8000398:	684f      	ldr	r7, [r1, #4]
 800039a:	4a0f      	ldr	r2, [pc, #60]	; (80003d8 <pvPortMalloc+0xc0>)
 800039c:	4610      	mov	r0, r2
 800039e:	6812      	ldr	r2, [r2, #0]
 80003a0:	6854      	ldr	r4, [r2, #4]
 80003a2:	42bc      	cmp	r4, r7
 80003a4:	d3fa      	bcc.n	800039c <pvPortMalloc+0x84>
 80003a6:	600a      	str	r2, [r1, #0]
 80003a8:	6001      	str	r1, [r0, #0]
                    xFreeBytesRemaining -= pxBlock->xBlockSize;
 80003aa:	685a      	ldr	r2, [r3, #4]
 80003ac:	1ab6      	subs	r6, r6, r2
                    heapALLOCATE_BLOCK( pxBlock );
 80003ae:	f042 4200 	orr.w	r2, r2, #2147483648	; 0x80000000
 80003b2:	605a      	str	r2, [r3, #4]
                    pxBlock->pxNextFreeBlock = NULL;
 80003b4:	2200      	movs	r2, #0
                    xFreeBytesRemaining -= pxBlock->xBlockSize;
 80003b6:	f8cc 6000 	str.w	r6, [ip]
                    pxBlock->pxNextFreeBlock = NULL;
 80003ba:	601a      	str	r2, [r3, #0]
    ( void ) xTaskResumeAll();
 80003bc:	f000 fb34 	bl	8000a28 <xTaskResumeAll>
}
 80003c0:	4628      	mov	r0, r5
 80003c2:	bdf8      	pop	{r3, r4, r5, r6, r7, pc}
 80003c4:	4619      	mov	r1, r3
 80003c6:	462b      	mov	r3, r5
 80003c8:	e7d0      	b.n	800036c <pvPortMalloc+0x54>
    void * pvReturn = NULL;
 80003ca:	2500      	movs	r5, #0
 80003cc:	e7f6      	b.n	80003bc <pvPortMalloc+0xa4>
 80003ce:	bf00      	nop
 80003d0:	20000020 	.word	0x20000020
 80003d4:	2000003b 	.word	0x2000003b
 80003d8:	2000002c 	.word	0x2000002c
 80003dc:	20000024 	.word	0x20000024
 80003e0:	20000000 	.word	0x20000000

080003e4 <vPortFree>:
{
 80003e4:	b510      	push	{r4, lr}
    if( pv != NULL )
 80003e6:	4604      	mov	r4, r0
 80003e8:	b1f8      	cbz	r0, 800042a <vPortFree+0x46>
        if( heapBLOCK_IS_ALLOCATED( pxLink ) != 0 )
 80003ea:	f850 3c04 	ldr.w	r3, [r0, #-4]
 80003ee:	2b00      	cmp	r3, #0
 80003f0:	da1b      	bge.n	800042a <vPortFree+0x46>
            if( pxLink->pxNextFreeBlock == NULL )
 80003f2:	f850 2c08 	ldr.w	r2, [r0, #-8]
 80003f6:	b9c2      	cbnz	r2, 800042a <vPortFree+0x46>
                heapFREE_BLOCK( pxLink );
 80003f8:	f023 4300 	bic.w	r3, r3, #2147483648	; 0x80000000
 80003fc:	f840 3c04 	str.w	r3, [r0, #-4]
                vTaskSuspendAll();
 8000400:	f000 fa5a 	bl	80008b8 <vTaskSuspendAll>
                    prvInsertBlockIntoFreeList( ( ( BlockLink_t * ) pxLink ) );
 8000404:	f854 1c04 	ldr.w	r1, [r4, #-4]
 8000408:	4b08      	ldr	r3, [pc, #32]	; (800042c <vPortFree+0x48>)
 800040a:	461a      	mov	r2, r3
 800040c:	681b      	ldr	r3, [r3, #0]
 800040e:	6858      	ldr	r0, [r3, #4]
 8000410:	4288      	cmp	r0, r1
 8000412:	d3fa      	bcc.n	800040a <vPortFree+0x26>
 8000414:	f844 3d08 	str.w	r3, [r4, #-8]!
 8000418:	6014      	str	r4, [r2, #0]
                    xFreeBytesRemaining += pxLink->xBlockSize;
 800041a:	4a05      	ldr	r2, [pc, #20]	; (8000430 <vPortFree+0x4c>)
}
 800041c:	e8bd 4010 	ldmia.w	sp!, {r4, lr}
                    xFreeBytesRemaining += pxLink->xBlockSize;
 8000420:	6813      	ldr	r3, [r2, #0]
 8000422:	440b      	add	r3, r1
 8000424:	6013      	str	r3, [r2, #0]
                ( void ) xTaskResumeAll();
 8000426:	f000 baff 	b.w	8000a28 <xTaskResumeAll>
}
 800042a:	bd10      	pop	{r4, pc}
 800042c:	2000002c 	.word	0x2000002c
 8000430:	20000000 	.word	0x20000000

08000434 <prvTaskExitError>:
}
/*-----------------------------------------------------------*/

static void prvTaskExitError( void )
{
    volatile uint32_t ulDummy = 0UL;
 8000434:	2300      	movs	r3, #0
{
 8000436:	b082      	sub	sp, #8
    volatile uint32_t ulDummy = 0UL;
 8000438:	9301      	str	r3, [sp, #4]

    portFORCE_INLINE static void vPortRaiseBASEPRI( void )
    {
        uint32_t ulNewBASEPRI;

        __asm volatile
 800043a:	f04f 03bf 	mov.w	r3, #191	; 0xbf
 800043e:	f383 8811 	msr	BASEPRI, r3
 8000442:	f3bf 8f6f 	isb	sy
 8000446:	f3bf 8f4f 	dsb	sy
     * Artificially force an assert() to be triggered if configASSERT() is
     * defined, then stop here so application writers can catch the error. */
    configASSERT( uxCriticalNesting == ~0UL );
    portDISABLE_INTERRUPTS();

    while( ulDummy == 0 )
 800044a:	9b01      	ldr	r3, [sp, #4]
 800044c:	2b00      	cmp	r3, #0
 800044e:	d0fc      	beq.n	800044a <prvTaskExitError+0x16>
         * about code appearing after this function is called - making ulDummy
         * volatile makes the compiler think the function could return and
         * therefore not output an 'unreachable code' warning for code that appears
         * after it. */
    }
}
 8000450:	b002      	add	sp, #8
 8000452:	4770      	bx	lr

08000454 <prvPortStartFirstTask>:
}
/*-----------------------------------------------------------*/

static void prvPortStartFirstTask( void )
{
    __asm volatile (
 8000454:	4806      	ldr	r0, [pc, #24]	; (8000470 <prvPortStartFirstTask+0x1c>)
 8000456:	6800      	ldr	r0, [r0, #0]
 8000458:	6800      	ldr	r0, [r0, #0]
 800045a:	f380 8808 	msr	MSP, r0
 800045e:	b662      	cpsie	i
 8000460:	b661      	cpsie	f
 8000462:	f3bf 8f4f 	dsb	sy
 8000466:	f3bf 8f6f 	isb	sy
 800046a:	df00      	svc	0
 800046c:	bf00      	nop
 800046e:	0000      	.short	0x0000
 8000470:	e000ed08 	.word	0xe000ed08

08000474 <pxPortInitialiseStack>:
    *pxTopOfStack = portINITIAL_XPSR;                                    /* xPSR */
 8000474:	f04f 7380 	mov.w	r3, #16777216	; 0x1000000
 8000478:	f840 3c04 	str.w	r3, [r0, #-4]
    *pxTopOfStack = ( StackType_t ) portTASK_RETURN_ADDRESS;             /* LR */
 800047c:	4b05      	ldr	r3, [pc, #20]	; (8000494 <pxPortInitialiseStack+0x20>)
    *pxTopOfStack = ( ( StackType_t ) pxCode ) & portSTART_ADDRESS_MASK; /* PC */
 800047e:	f021 0101 	bic.w	r1, r1, #1
 8000482:	f840 1c08 	str.w	r1, [r0, #-8]
    *pxTopOfStack = ( StackType_t ) portTASK_RETURN_ADDRESS;             /* LR */
 8000486:	f840 3c0c 	str.w	r3, [r0, #-12]
    *pxTopOfStack = ( StackType_t ) pvParameters;                        /* R0 */
 800048a:	f840 2c20 	str.w	r2, [r0, #-32]
}
 800048e:	3840      	subs	r0, #64	; 0x40
 8000490:	4770      	bx	lr
 8000492:	bf00      	nop
 8000494:	08000435 	.word	0x08000435
	...

080004a0 <vPortSVCHandler>:
    __asm volatile (
 80004a0:	4b07      	ldr	r3, [pc, #28]	; (80004c0 <pxCurrentTCBConst2>)
 80004a2:	6819      	ldr	r1, [r3, #0]
 80004a4:	6808      	ldr	r0, [r1, #0]
 80004a6:	e8b0 0ff0 	ldmia.w	r0!, {r4, r5, r6, r7, r8, r9, sl, fp}
 80004aa:	f380 8809 	msr	PSP, r0
 80004ae:	f3bf 8f6f 	isb	sy
 80004b2:	f04f 0000 	mov.w	r0, #0
 80004b6:	f380 8811 	msr	BASEPRI, r0
 80004ba:	f04e 0e0d 	orr.w	lr, lr, #13
 80004be:	4770      	bx	lr

080004c0 <pxCurrentTCBConst2>:
 80004c0:	2000151c 	.word	0x2000151c

080004c4 <vPortEnterCritical>:
 80004c4:	f04f 03bf 	mov.w	r3, #191	; 0xbf
 80004c8:	f383 8811 	msr	BASEPRI, r3
 80004cc:	f3bf 8f6f 	isb	sy
 80004d0:	f3bf 8f4f 	dsb	sy
/*-----------------------------------------------------------*/

void vPortEnterCritical( void )
{
    portDISABLE_INTERRUPTS();
    uxCriticalNesting++;
 80004d4:	4a02      	ldr	r2, [pc, #8]	; (80004e0 <vPortEnterCritical+0x1c>)
 80004d6:	6813      	ldr	r3, [r2, #0]
 80004d8:	3301      	adds	r3, #1
 80004da:	6013      	str	r3, [r2, #0]
     * assert function also uses a critical section. */
    if( uxCriticalNesting == 1 )
    {
        configASSERT( ( portNVIC_INT_CTRL_REG & portVECTACTIVE_MASK ) == 0 );
    }
}
 80004dc:	4770      	bx	lr
 80004de:	bf00      	nop
 80004e0:	20000004 	.word	0x20000004

080004e4 <vPortExitCritical>:
/*-----------------------------------------------------------*/

void vPortExitCritical( void )
{
    configASSERT( uxCriticalNesting );
    uxCriticalNesting--;
 80004e4:	4a03      	ldr	r2, [pc, #12]	; (80004f4 <vPortExitCritical+0x10>)
 80004e6:	6813      	ldr	r3, [r2, #0]
 80004e8:	3b01      	subs	r3, #1
 80004ea:	6013      	str	r3, [r2, #0]

    if( uxCriticalNesting == 0 )
 80004ec:	b90b      	cbnz	r3, 80004f2 <vPortExitCritical+0xe>
    }
/*-----------------------------------------------------------*/

    portFORCE_INLINE static void vPortSetBASEPRI( uint32_t ulNewMaskValue )
    {
        __asm volatile
 80004ee:	f383 8811 	msr	BASEPRI, r3
    {
        portENABLE_INTERRUPTS();
    }
}
 80004f2:	4770      	bx	lr
 80004f4:	20000004 	.word	0x20000004
	...

08000500 <xPortPendSVHandler>:

void xPortPendSVHandler( void )
{
    /* This is a naked function. */

    __asm volatile
 8000500:	f3ef 8009 	mrs	r0, PSP
 8000504:	f3bf 8f6f 	isb	sy
 8000508:	4b0d      	ldr	r3, [pc, #52]	; (8000540 <pxCurrentTCBConst>)
 800050a:	681a      	ldr	r2, [r3, #0]
 800050c:	e920 0ff0 	stmdb	r0!, {r4, r5, r6, r7, r8, r9, sl, fp}
 8000510:	6010      	str	r0, [r2, #0]
 8000512:	e92d 4008 	stmdb	sp!, {r3, lr}
 8000516:	f04f 00bf 	mov.w	r0, #191	; 0xbf
 800051a:	f380 8811 	msr	BASEPRI, r0
 800051e:	f000 fb41 	bl	8000ba4 <vTaskSwitchContext>
 8000522:	f04f 0000 	mov.w	r0, #0
 8000526:	f380 8811 	msr	BASEPRI, r0
 800052a:	e8bd 4008 	ldmia.w	sp!, {r3, lr}
 800052e:	6819      	ldr	r1, [r3, #0]
 8000530:	6808      	ldr	r0, [r1, #0]
 8000532:	e8b0 0ff0 	ldmia.w	r0!, {r4, r5, r6, r7, r8, r9, sl, fp}
 8000536:	f380 8809 	msr	PSP, r0
 800053a:	f3bf 8f6f 	isb	sy
 800053e:	4770      	bx	lr

08000540 <pxCurrentTCBConst>:
 8000540:	2000151c 	.word	0x2000151c

08000544 <xPortSysTickHandler>:
    );
}
/*-----------------------------------------------------------*/

void xPortSysTickHandler( void )
{
 8000544:	b508      	push	{r3, lr}
        __asm volatile
 8000546:	f04f 03bf 	mov.w	r3, #191	; 0xbf
 800054a:	f383 8811 	msr	BASEPRI, r3
 800054e:	f3bf 8f6f 	isb	sy
 8000552:	f3bf 8f4f 	dsb	sy
     * save and then restore the interrupt mask value as its value is already
     * known. */
    portDISABLE_INTERRUPTS();
    {
        /* Increment the RTOS tick. */
        if( xTaskIncrementTick() != pdFALSE )
 8000556:	f000 f9bd 	bl	80008d4 <xTaskIncrementTick>
 800055a:	b128      	cbz	r0, 8000568 <xPortSysTickHandler+0x24>
        {
            /* A context switch is required.  Context switching is performed in
             * the PendSV interrupt.  Pend the PendSV interrupt. */
            portNVIC_INT_CTRL_REG = portNVIC_PENDSVSET_BIT;
 800055c:	f04f 23e0 	mov.w	r3, #3758153728	; 0xe000e000
 8000560:	f04f 5280 	mov.w	r2, #268435456	; 0x10000000
 8000564:	f8c3 2d04 	str.w	r2, [r3, #3332]	; 0xd04
        __asm volatile
 8000568:	2300      	movs	r3, #0
 800056a:	f383 8811 	msr	BASEPRI, r3
        }
    }
    portENABLE_INTERRUPTS();
}
 800056e:	bd08      	pop	{r3, pc}

08000570 <vPortSetupTimerInterrupt>:
        ulStoppedTimerCompensation = portMISSED_COUNTS_FACTOR / ( configCPU_CLOCK_HZ / configSYSTICK_CLOCK_HZ );
    }
    #endif /* configUSE_TICKLESS_IDLE */

    /* Stop and clear the SysTick. */
    portNVIC_SYSTICK_CTRL_REG = 0UL;
 8000570:	f04f 23e0 	mov.w	r3, #3758153728	; 0xe000e000
 8000574:	2200      	movs	r2, #0
 8000576:	611a      	str	r2, [r3, #16]
    portNVIC_SYSTICK_CURRENT_VALUE_REG = 0UL;
 8000578:	619a      	str	r2, [r3, #24]

    /* Configure SysTick to interrupt at the requested rate. */
    portNVIC_SYSTICK_LOAD_REG = ( configSYSTICK_CLOCK_HZ / configTICK_RATE_HZ ) - 1UL;
 800057a:	4a02      	ldr	r2, [pc, #8]	; (8000584 <vPortSetupTimerInterrupt+0x14>)
 800057c:	615a      	str	r2, [r3, #20]
    portNVIC_SYSTICK_CTRL_REG = ( portNVIC_SYSTICK_CLK_BIT_CONFIG | portNVIC_SYSTICK_INT_BIT | portNVIC_SYSTICK_ENABLE_BIT );
 800057e:	2207      	movs	r2, #7
 8000580:	611a      	str	r2, [r3, #16]
}
 8000582:	4770      	bx	lr
 8000584:	0001193f 	.word	0x0001193f

08000588 <xPortStartScheduler>:
    portNVIC_SHPR3_REG |= portNVIC_PENDSV_PRI;
 8000588:	f04f 23e0 	mov.w	r3, #3758153728	; 0xe000e000
{
 800058c:	b510      	push	{r4, lr}
    uxCriticalNesting = 0;
 800058e:	2400      	movs	r4, #0
    portNVIC_SHPR3_REG |= portNVIC_PENDSV_PRI;
 8000590:	f8d3 2d20 	ldr.w	r2, [r3, #3360]	; 0xd20
 8000594:	f442 027f 	orr.w	r2, r2, #16711680	; 0xff0000
 8000598:	f8c3 2d20 	str.w	r2, [r3, #3360]	; 0xd20
    portNVIC_SHPR3_REG |= portNVIC_SYSTICK_PRI;
 800059c:	f8d3 2d20 	ldr.w	r2, [r3, #3360]	; 0xd20
 80005a0:	f042 427f 	orr.w	r2, r2, #4278190080	; 0xff000000
 80005a4:	f8c3 2d20 	str.w	r2, [r3, #3360]	; 0xd20
    vPortSetupTimerInterrupt();
 80005a8:	f7ff ffe2 	bl	8000570 <vPortSetupTimerInterrupt>
    uxCriticalNesting = 0;
 80005ac:	4b04      	ldr	r3, [pc, #16]	; (80005c0 <xPortStartScheduler+0x38>)
 80005ae:	601c      	str	r4, [r3, #0]
    prvPortStartFirstTask();
 80005b0:	f7ff ff50 	bl	8000454 <prvPortStartFirstTask>
    vTaskSwitchContext();
 80005b4:	f000 faf6 	bl	8000ba4 <vTaskSwitchContext>
    prvTaskExitError();
 80005b8:	f7ff ff3c 	bl	8000434 <prvTaskExitError>
}
 80005bc:	4620      	mov	r0, r4
 80005be:	bd10      	pop	{r4, pc}
 80005c0:	20000004 	.word	0x20000004

080005c4 <prvIdleTask>:
             * the list, and an occasional incorrect value will not matter.  If
             * the ready list at the idle priority contains more than one task
             * then a task other than the idle task is ready to execute. */
            if( listCURRENT_LIST_LENGTH( &( pxReadyTasksLists[ tskIDLE_PRIORITY ] ) ) > ( UBaseType_t ) 1 )
            {
                taskYIELD();
 80005c4:	f04f 23e0 	mov.w	r3, #3758153728	; 0xe000e000
 80005c8:	f04f 5280 	mov.w	r2, #268435456	; 0x10000000
            if( listCURRENT_LIST_LENGTH( &( pxReadyTasksLists[ tskIDLE_PRIORITY ] ) ) > ( UBaseType_t ) 1 )
 80005cc:	4905      	ldr	r1, [pc, #20]	; (80005e4 <prvIdleTask+0x20>)
 80005ce:	6808      	ldr	r0, [r1, #0]
 80005d0:	2801      	cmp	r0, #1
 80005d2:	d9fc      	bls.n	80005ce <prvIdleTask+0xa>
                taskYIELD();
 80005d4:	f8c3 2d04 	str.w	r2, [r3, #3332]	; 0xd04
 80005d8:	f3bf 8f4f 	dsb	sy
 80005dc:	f3bf 8f6f 	isb	sy
 80005e0:	e7f5      	b.n	80005ce <prvIdleTask+0xa>
 80005e2:	bf00      	nop
 80005e4:	200014b8 	.word	0x200014b8

080005e8 <prvAddCurrentTaskToDelayedList>:
#endif /* if ( ( configGENERATE_RUN_TIME_STATS == 1 ) && ( INCLUDE_xTaskGetIdleTaskHandle == 1 ) ) */
/*-----------------------------------------------------------*/

static void prvAddCurrentTaskToDelayedList( TickType_t xTicksToWait,
                                            const BaseType_t xCanBlockIndefinitely )
{
 80005e8:	b5f8      	push	{r3, r4, r5, r6, r7, lr}
    TickType_t xTimeToWake;
    const TickType_t xConstTickCount = xTickCount;
 80005ea:	4b20      	ldr	r3, [pc, #128]	; (800066c <prvAddCurrentTaskToDelayedList+0x84>)
    }
    #endif

    /* Remove the task from the ready list before adding it to the blocked list
     * as the same list item is used for both lists. */
    if( uxListRemove( &( pxCurrentTCB->xStateListItem ) ) == ( UBaseType_t ) 0 )
 80005ec:	4c20      	ldr	r4, [pc, #128]	; (8000670 <prvAddCurrentTaskToDelayedList+0x88>)
{
 80005ee:	4606      	mov	r6, r0
    const TickType_t xConstTickCount = xTickCount;
 80005f0:	681d      	ldr	r5, [r3, #0]
    if( uxListRemove( &( pxCurrentTCB->xStateListItem ) ) == ( UBaseType_t ) 0 )
 80005f2:	6820      	ldr	r0, [r4, #0]
{
 80005f4:	460f      	mov	r7, r1
    if( uxListRemove( &( pxCurrentTCB->xStateListItem ) ) == ( UBaseType_t ) 0 )
 80005f6:	3004      	adds	r0, #4
 80005f8:	f000 fea6 	bl	8001348 <uxListRemove>
 80005fc:	b940      	cbnz	r0, 8000610 <prvAddCurrentTaskToDelayedList+0x28>
    {
        /* The current task must be in a ready list, so there is no need to
         * check, and the port reset macro can be called directly. */
        portRESET_READY_PRIORITY( pxCurrentTCB->uxPriority, uxTopReadyPriority ); /*lint !e931 pxCurrentTCB cannot change as it is the calling task.  pxCurrentTCB->uxPriority and uxTopReadyPriority cannot change as called with scheduler suspended or in a critical section. */
 80005fe:	6822      	ldr	r2, [r4, #0]
 8000600:	491c      	ldr	r1, [pc, #112]	; (8000674 <prvAddCurrentTaskToDelayedList+0x8c>)
 8000602:	6ad0      	ldr	r0, [r2, #44]	; 0x2c
 8000604:	2201      	movs	r2, #1
 8000606:	680b      	ldr	r3, [r1, #0]
 8000608:	4082      	lsls	r2, r0
 800060a:	ea23 0302 	bic.w	r3, r3, r2
 800060e:	600b      	str	r3, [r1, #0]
        mtCOVERAGE_TEST_MARKER();
    }

    #if ( INCLUDE_vTaskSuspend == 1 )
    {
        if( ( xTicksToWait == portMAX_DELAY ) && ( xCanBlockIndefinitely != pdFALSE ) )
 8000610:	1c73      	adds	r3, r6, #1
 8000612:	d113      	bne.n	800063c <prvAddCurrentTaskToDelayedList+0x54>
 8000614:	b197      	cbz	r7, 800063c <prvAddCurrentTaskToDelayedList+0x54>
        {
            /* Add the task to the suspended task list instead of a delayed task
             * list to ensure it is not woken by a timing event.  It will block
             * indefinitely. */
            listINSERT_END( &xSuspendedTaskList, &( pxCurrentTCB->xStateListItem ) );
 8000616:	4b18      	ldr	r3, [pc, #96]	; (8000678 <prvAddCurrentTaskToDelayedList+0x90>)
 8000618:	6821      	ldr	r1, [r4, #0]
 800061a:	685a      	ldr	r2, [r3, #4]
 800061c:	608a      	str	r2, [r1, #8]
 800061e:	6890      	ldr	r0, [r2, #8]
 8000620:	6821      	ldr	r1, [r4, #0]
 8000622:	60c8      	str	r0, [r1, #12]
 8000624:	6821      	ldr	r1, [r4, #0]
 8000626:	3104      	adds	r1, #4
 8000628:	6041      	str	r1, [r0, #4]
 800062a:	6821      	ldr	r1, [r4, #0]
 800062c:	3104      	adds	r1, #4
 800062e:	6091      	str	r1, [r2, #8]
 8000630:	6822      	ldr	r2, [r4, #0]
 8000632:	6153      	str	r3, [r2, #20]
 8000634:	681a      	ldr	r2, [r3, #0]
 8000636:	3201      	adds	r2, #1
 8000638:	601a      	str	r2, [r3, #0]

        /* Avoid compiler warning when INCLUDE_vTaskSuspend is not 1. */
        ( void ) xCanBlockIndefinitely;
    }
    #endif /* INCLUDE_vTaskSuspend */
}
 800063a:	bdf8      	pop	{r3, r4, r5, r6, r7, pc}
            listSET_LIST_ITEM_VALUE( &( pxCurrentTCB->xStateListItem ), xTimeToWake );
 800063c:	6823      	ldr	r3, [r4, #0]
 800063e:	19ad      	adds	r5, r5, r6
 8000640:	605d      	str	r5, [r3, #4]
            if( xTimeToWake < xConstTickCount )
 8000642:	d307      	bcc.n	8000654 <prvAddCurrentTaskToDelayedList+0x6c>
                vListInsert( pxOverflowDelayedTaskList, &( pxCurrentTCB->xStateListItem ) );
 8000644:	4b0d      	ldr	r3, [pc, #52]	; (800067c <prvAddCurrentTaskToDelayedList+0x94>)
 8000646:	6818      	ldr	r0, [r3, #0]
 8000648:	6821      	ldr	r1, [r4, #0]
}
 800064a:	e8bd 40f8 	ldmia.w	sp!, {r3, r4, r5, r6, r7, lr}
                vListInsert( pxOverflowDelayedTaskList, &( pxCurrentTCB->xStateListItem ) );
 800064e:	3104      	adds	r1, #4
 8000650:	f000 be63 	b.w	800131a <vListInsert>
                vListInsert( pxDelayedTaskList, &( pxCurrentTCB->xStateListItem ) );
 8000654:	4b0a      	ldr	r3, [pc, #40]	; (8000680 <prvAddCurrentTaskToDelayedList+0x98>)
 8000656:	6818      	ldr	r0, [r3, #0]
 8000658:	6821      	ldr	r1, [r4, #0]
 800065a:	3104      	adds	r1, #4
 800065c:	f000 fe5d 	bl	800131a <vListInsert>
                if( xTimeToWake < xNextTaskUnblockTime )
 8000660:	4b08      	ldr	r3, [pc, #32]	; (8000684 <prvAddCurrentTaskToDelayedList+0x9c>)
 8000662:	681a      	ldr	r2, [r3, #0]
 8000664:	42aa      	cmp	r2, r5
                    xNextTaskUnblockTime = xTimeToWake;
 8000666:	bf88      	it	hi
 8000668:	601d      	strhi	r5, [r3, #0]
}
 800066a:	e7e6      	b.n	800063a <prvAddCurrentTaskToDelayedList+0x52>
 800066c:	20001458 	.word	0x20001458
 8000670:	2000151c 	.word	0x2000151c
 8000674:	20001454 	.word	0x20001454
 8000678:	20001460 	.word	0x20001460
 800067c:	20001488 	.word	0x20001488
 8000680:	2000148c 	.word	0x2000148c
 8000684:	2000143c 	.word	0x2000143c

08000688 <prvResetNextTaskUnblockTime>:
    if( listLIST_IS_EMPTY( pxDelayedTaskList ) != pdFALSE )
 8000688:	4a06      	ldr	r2, [pc, #24]	; (80006a4 <prvResetNextTaskUnblockTime+0x1c>)
 800068a:	6813      	ldr	r3, [r2, #0]
 800068c:	6819      	ldr	r1, [r3, #0]
 800068e:	4b06      	ldr	r3, [pc, #24]	; (80006a8 <prvResetNextTaskUnblockTime+0x20>)
 8000690:	b919      	cbnz	r1, 800069a <prvResetNextTaskUnblockTime+0x12>
        xNextTaskUnblockTime = portMAX_DELAY;
 8000692:	f04f 32ff 	mov.w	r2, #4294967295	; 0xffffffff
        xNextTaskUnblockTime = listGET_ITEM_VALUE_OF_HEAD_ENTRY( pxDelayedTaskList );
 8000696:	601a      	str	r2, [r3, #0]
}
 8000698:	4770      	bx	lr
        xNextTaskUnblockTime = listGET_ITEM_VALUE_OF_HEAD_ENTRY( pxDelayedTaskList );
 800069a:	6812      	ldr	r2, [r2, #0]
 800069c:	68d2      	ldr	r2, [r2, #12]
 800069e:	6812      	ldr	r2, [r2, #0]
 80006a0:	e7f9      	b.n	8000696 <prvResetNextTaskUnblockTime+0xe>
 80006a2:	bf00      	nop
 80006a4:	2000148c 	.word	0x2000148c
 80006a8:	2000143c 	.word	0x2000143c

080006ac <xTaskCreate>:
    {
 80006ac:	e92d 47f0 	stmdb	sp!, {r4, r5, r6, r7, r8, r9, sl, lr}
            pxStack = pvPortMallocStack( ( ( ( size_t ) usStackDepth ) * sizeof( StackType_t ) ) ); /*lint !e9079 All values returned by pvPortMalloc() have at least the alignment required by the MCU's stack and this allocation is the stack. */
 80006b0:	ea4f 0a82 	mov.w	sl, r2, lsl #2
    {
 80006b4:	4607      	mov	r7, r0
            pxStack = pvPortMallocStack( ( ( ( size_t ) usStackDepth ) * sizeof( StackType_t ) ) ); /*lint !e9079 All values returned by pvPortMalloc() have at least the alignment required by the MCU's stack and this allocation is the stack. */
 80006b6:	4650      	mov	r0, sl
    {
 80006b8:	460e      	mov	r6, r1
 80006ba:	4698      	mov	r8, r3
 80006bc:	f8dd 9024 	ldr.w	r9, [sp, #36]	; 0x24
            pxStack = pvPortMallocStack( ( ( ( size_t ) usStackDepth ) * sizeof( StackType_t ) ) ); /*lint !e9079 All values returned by pvPortMalloc() have at least the alignment required by the MCU's stack and this allocation is the stack. */
 80006c0:	f7ff fe2a 	bl	8000318 <pvPortMalloc>
            if( pxStack != NULL )
 80006c4:	4605      	mov	r5, r0
 80006c6:	b918      	cbnz	r0, 80006d0 <xTaskCreate+0x24>
            xReturn = errCOULD_NOT_ALLOCATE_REQUIRED_MEMORY;
 80006c8:	f04f 30ff 	mov.w	r0, #4294967295	; 0xffffffff
    }
 80006cc:	e8bd 87f0 	ldmia.w	sp!, {r4, r5, r6, r7, r8, r9, sl, pc}
                pxNewTCB = ( TCB_t * ) pvPortMalloc( sizeof( TCB_t ) ); /*lint !e9087 !e9079 All values returned by pvPortMalloc() have at least the alignment required by the MCU's stack, and the first member of TCB_t is always a pointer to the task's stack. */
 80006d0:	2054      	movs	r0, #84	; 0x54
 80006d2:	f7ff fe21 	bl	8000318 <pvPortMalloc>
                if( pxNewTCB != NULL )
 80006d6:	4604      	mov	r4, r0
 80006d8:	2800      	cmp	r0, #0
 80006da:	f000 809f 	beq.w	800081c <xTaskCreate+0x170>
                    memset( ( void * ) pxNewTCB, 0x00, sizeof( TCB_t ) );
 80006de:	2254      	movs	r2, #84	; 0x54
 80006e0:	2100      	movs	r1, #0
        pxTopOfStack = &( pxNewTCB->pxStack[ ulStackDepth - ( uint32_t ) 1 ] );
 80006e2:	f1aa 0a04 	sub.w	sl, sl, #4
                    memset( ( void * ) pxNewTCB, 0x00, sizeof( TCB_t ) );
 80006e6:	f001 f887 	bl	80017f8 <memset>
                    pxNewTCB->pxStack = pxStack;
 80006ea:	6325      	str	r5, [r4, #48]	; 0x30
        pxTopOfStack = &( pxNewTCB->pxStack[ ulStackDepth - ( uint32_t ) 1 ] );
 80006ec:	4455      	add	r5, sl
        pxTopOfStack = ( StackType_t * ) ( ( ( portPOINTER_SIZE_TYPE ) pxTopOfStack ) & ( ~( ( portPOINTER_SIZE_TYPE ) portBYTE_ALIGNMENT_MASK ) ) ); /*lint !e923 !e9033 !e9078 MISRA exception.  Avoiding casts between pointers and integers is not practical.  Size differences accounted for using portPOINTER_SIZE_TYPE type.  Checked by assert(). */
 80006ee:	f025 0507 	bic.w	r5, r5, #7
    if( pcName != NULL )
 80006f2:	b16e      	cbz	r6, 8000710 <xTaskCreate+0x64>
 80006f4:	1e73      	subs	r3, r6, #1
 80006f6:	f104 0233 	add.w	r2, r4, #51	; 0x33
 80006fa:	360f      	adds	r6, #15
            pxNewTCB->pcTaskName[ x ] = pcName[ x ];
 80006fc:	f813 1f01 	ldrb.w	r1, [r3, #1]!
 8000700:	f802 1f01 	strb.w	r1, [r2, #1]!
            if( pcName[ x ] == ( char ) 0x00 )
 8000704:	b109      	cbz	r1, 800070a <xTaskCreate+0x5e>
        for( x = ( UBaseType_t ) 0; x < ( UBaseType_t ) configMAX_TASK_NAME_LEN; x++ )
 8000706:	42b3      	cmp	r3, r6
 8000708:	d1f8      	bne.n	80006fc <xTaskCreate+0x50>
        pxNewTCB->pcTaskName[ configMAX_TASK_NAME_LEN - 1 ] = '\0';
 800070a:	2300      	movs	r3, #0
 800070c:	f884 3043 	strb.w	r3, [r4, #67]	; 0x43
    if( uxPriority >= ( UBaseType_t ) configMAX_PRIORITIES )
 8000710:	9e08      	ldr	r6, [sp, #32]
    vListInitialiseItem( &( pxNewTCB->xStateListItem ) );
 8000712:	f104 0a04 	add.w	sl, r4, #4
    if( uxPriority >= ( UBaseType_t ) configMAX_PRIORITIES )
 8000716:	2e04      	cmp	r6, #4
 8000718:	bf28      	it	cs
 800071a:	2604      	movcs	r6, #4
    vListInitialiseItem( &( pxNewTCB->xStateListItem ) );
 800071c:	4650      	mov	r0, sl
    pxNewTCB->uxPriority = uxPriority;
 800071e:	62e6      	str	r6, [r4, #44]	; 0x2c
        pxNewTCB->uxBasePriority = uxPriority;
 8000720:	6466      	str	r6, [r4, #68]	; 0x44
    vListInitialiseItem( &( pxNewTCB->xStateListItem ) );
 8000722:	f000 fdf7 	bl	8001314 <vListInitialiseItem>
    listSET_LIST_ITEM_VALUE( &( pxNewTCB->xEventListItem ), ( TickType_t ) configMAX_PRIORITIES - ( TickType_t ) uxPriority ); /*lint !e961 MISRA exception as the casts are only redundant for some ports. */
 8000726:	f1c6 0605 	rsb	r6, r6, #5
    vListInitialiseItem( &( pxNewTCB->xEventListItem ) );
 800072a:	f104 0018 	add.w	r0, r4, #24
 800072e:	f000 fdf1 	bl	8001314 <vListInitialiseItem>
            pxNewTCB->pxTopOfStack = pxPortInitialiseStack( pxTopOfStack, pxTaskCode, pvParameters );
 8000732:	4642      	mov	r2, r8
 8000734:	4639      	mov	r1, r7
 8000736:	4628      	mov	r0, r5
    listSET_LIST_ITEM_OWNER( &( pxNewTCB->xStateListItem ), pxNewTCB );
 8000738:	6124      	str	r4, [r4, #16]
    listSET_LIST_ITEM_VALUE( &( pxNewTCB->xEventListItem ), ( TickType_t ) configMAX_PRIORITIES - ( TickType_t ) uxPriority ); /*lint !e961 MISRA exception as the casts are only redundant for some ports. */
 800073a:	61a6      	str	r6, [r4, #24]
    listSET_LIST_ITEM_OWNER( &( pxNewTCB->xEventListItem ), pxNewTCB );
 800073c:	6264      	str	r4, [r4, #36]	; 0x24
            pxNewTCB->pxTopOfStack = pxPortInitialiseStack( pxTopOfStack, pxTaskCode, pvParameters );
 800073e:	f7ff fe99 	bl	8000474 <pxPortInitialiseStack>
 8000742:	6020      	str	r0, [r4, #0]
    if( pxCreatedTask != NULL )
 8000744:	f1b9 0f00 	cmp.w	r9, #0
 8000748:	d001      	beq.n	800074e <xTaskCreate+0xa2>
        *pxCreatedTask = ( TaskHandle_t ) pxNewTCB;
 800074a:	f8c9 4000 	str.w	r4, [r9]
    taskENTER_CRITICAL();
 800074e:	f7ff feb9 	bl	80004c4 <vPortEnterCritical>
        uxCurrentNumberOfTasks++;
 8000752:	4b34      	ldr	r3, [pc, #208]	; (8000824 <xTaskCreate+0x178>)
        if( pxCurrentTCB == NULL )
 8000754:	4e34      	ldr	r6, [pc, #208]	; (8000828 <xTaskCreate+0x17c>)
        uxCurrentNumberOfTasks++;
 8000756:	681a      	ldr	r2, [r3, #0]
 8000758:	4f34      	ldr	r7, [pc, #208]	; (800082c <xTaskCreate+0x180>)
 800075a:	3201      	adds	r2, #1
 800075c:	601a      	str	r2, [r3, #0]
        if( pxCurrentTCB == NULL )
 800075e:	6835      	ldr	r5, [r6, #0]
 8000760:	2d00      	cmp	r5, #0
 8000762:	d150      	bne.n	8000806 <xTaskCreate+0x15a>
            pxCurrentTCB = pxNewTCB;
 8000764:	6034      	str	r4, [r6, #0]
            if( uxCurrentNumberOfTasks == ( UBaseType_t ) 1 )
 8000766:	681b      	ldr	r3, [r3, #0]
 8000768:	2b01      	cmp	r3, #1
 800076a:	d11c      	bne.n	80007a6 <xTaskCreate+0xfa>
 800076c:	46b8      	mov	r8, r7
        vListInitialise( &( pxReadyTasksLists[ uxPriority ] ) );
 800076e:	4640      	mov	r0, r8
    for( uxPriority = ( UBaseType_t ) 0U; uxPriority < ( UBaseType_t ) configMAX_PRIORITIES; uxPriority++ )
 8000770:	3501      	adds	r5, #1
        vListInitialise( &( pxReadyTasksLists[ uxPriority ] ) );
 8000772:	f000 fdc4 	bl	80012fe <vListInitialise>
    for( uxPriority = ( UBaseType_t ) 0U; uxPriority < ( UBaseType_t ) configMAX_PRIORITIES; uxPriority++ )
 8000776:	2d05      	cmp	r5, #5
 8000778:	f108 0814 	add.w	r8, r8, #20
 800077c:	d1f7      	bne.n	800076e <xTaskCreate+0xc2>
    vListInitialise( &xDelayedTaskList1 );
 800077e:	f8df 80b0 	ldr.w	r8, [pc, #176]	; 8000830 <xTaskCreate+0x184>
    vListInitialise( &xDelayedTaskList2 );
 8000782:	4d2c      	ldr	r5, [pc, #176]	; (8000834 <xTaskCreate+0x188>)
    vListInitialise( &xDelayedTaskList1 );
 8000784:	4640      	mov	r0, r8
 8000786:	f000 fdba 	bl	80012fe <vListInitialise>
    vListInitialise( &xDelayedTaskList2 );
 800078a:	4628      	mov	r0, r5
 800078c:	f000 fdb7 	bl	80012fe <vListInitialise>
    vListInitialise( &xPendingReadyList );
 8000790:	4829      	ldr	r0, [pc, #164]	; (8000838 <xTaskCreate+0x18c>)
 8000792:	f000 fdb4 	bl	80012fe <vListInitialise>
        vListInitialise( &xSuspendedTaskList );
 8000796:	4829      	ldr	r0, [pc, #164]	; (800083c <xTaskCreate+0x190>)
 8000798:	f000 fdb1 	bl	80012fe <vListInitialise>
    pxDelayedTaskList = &xDelayedTaskList1;
 800079c:	4b28      	ldr	r3, [pc, #160]	; (8000840 <xTaskCreate+0x194>)
 800079e:	f8c3 8000 	str.w	r8, [r3]
    pxOverflowDelayedTaskList = &xDelayedTaskList2;
 80007a2:	4b28      	ldr	r3, [pc, #160]	; (8000844 <xTaskCreate+0x198>)
 80007a4:	601d      	str	r5, [r3, #0]
        uxTaskNumber++;
 80007a6:	4a28      	ldr	r2, [pc, #160]	; (8000848 <xTaskCreate+0x19c>)
        prvAddTaskToReadyList( pxNewTCB );
 80007a8:	4928      	ldr	r1, [pc, #160]	; (800084c <xTaskCreate+0x1a0>)
        uxTaskNumber++;
 80007aa:	6813      	ldr	r3, [r2, #0]
        prvAddTaskToReadyList( pxNewTCB );
 80007ac:	6808      	ldr	r0, [r1, #0]
        uxTaskNumber++;
 80007ae:	3301      	adds	r3, #1
 80007b0:	6013      	str	r3, [r2, #0]
        prvAddTaskToReadyList( pxNewTCB );
 80007b2:	2201      	movs	r2, #1
 80007b4:	6ae3      	ldr	r3, [r4, #44]	; 0x2c
 80007b6:	409a      	lsls	r2, r3
 80007b8:	4302      	orrs	r2, r0
 80007ba:	600a      	str	r2, [r1, #0]
 80007bc:	2214      	movs	r2, #20
 80007be:	4353      	muls	r3, r2
 80007c0:	18f9      	adds	r1, r7, r3
 80007c2:	684a      	ldr	r2, [r1, #4]
 80007c4:	6890      	ldr	r0, [r2, #8]
 80007c6:	60a2      	str	r2, [r4, #8]
 80007c8:	60e0      	str	r0, [r4, #12]
 80007ca:	f8c0 a004 	str.w	sl, [r0, #4]
 80007ce:	f8c2 a008 	str.w	sl, [r2, #8]
 80007d2:	58fa      	ldr	r2, [r7, r3]
 80007d4:	6161      	str	r1, [r4, #20]
 80007d6:	3201      	adds	r2, #1
 80007d8:	50fa      	str	r2, [r7, r3]
    taskEXIT_CRITICAL();
 80007da:	f7ff fe83 	bl	80004e4 <vPortExitCritical>
    if( xSchedulerRunning != pdFALSE )
 80007de:	4b1c      	ldr	r3, [pc, #112]	; (8000850 <xTaskCreate+0x1a4>)
 80007e0:	681b      	ldr	r3, [r3, #0]
 80007e2:	b173      	cbz	r3, 8000802 <xTaskCreate+0x156>
        if( pxCurrentTCB->uxPriority < pxNewTCB->uxPriority )
 80007e4:	6833      	ldr	r3, [r6, #0]
 80007e6:	6ada      	ldr	r2, [r3, #44]	; 0x2c
 80007e8:	6ae3      	ldr	r3, [r4, #44]	; 0x2c
 80007ea:	429a      	cmp	r2, r3
 80007ec:	d209      	bcs.n	8000802 <xTaskCreate+0x156>
            taskYIELD_IF_USING_PREEMPTION();
 80007ee:	f04f 23e0 	mov.w	r3, #3758153728	; 0xe000e000
 80007f2:	f04f 5280 	mov.w	r2, #268435456	; 0x10000000
 80007f6:	f8c3 2d04 	str.w	r2, [r3, #3332]	; 0xd04
 80007fa:	f3bf 8f4f 	dsb	sy
 80007fe:	f3bf 8f6f 	isb	sy
            xReturn = pdPASS;
 8000802:	2001      	movs	r0, #1
        return xReturn;
 8000804:	e762      	b.n	80006cc <xTaskCreate+0x20>
            if( xSchedulerRunning == pdFALSE )
 8000806:	4b12      	ldr	r3, [pc, #72]	; (8000850 <xTaskCreate+0x1a4>)
 8000808:	681a      	ldr	r2, [r3, #0]
                if( pxCurrentTCB->uxPriority <= pxNewTCB->uxPriority )
 800080a:	6ae3      	ldr	r3, [r4, #44]	; 0x2c
            if( xSchedulerRunning == pdFALSE )
 800080c:	2a00      	cmp	r2, #0
 800080e:	d1ca      	bne.n	80007a6 <xTaskCreate+0xfa>
                if( pxCurrentTCB->uxPriority <= pxNewTCB->uxPriority )
 8000810:	6832      	ldr	r2, [r6, #0]
 8000812:	6ad2      	ldr	r2, [r2, #44]	; 0x2c
 8000814:	429a      	cmp	r2, r3
                    pxCurrentTCB = pxNewTCB;
 8000816:	bf98      	it	ls
 8000818:	6034      	strls	r4, [r6, #0]
 800081a:	e7c4      	b.n	80007a6 <xTaskCreate+0xfa>
                    vPortFreeStack( pxStack );
 800081c:	4628      	mov	r0, r5
 800081e:	f7ff fde1 	bl	80003e4 <vPortFree>
        if( pxNewTCB != NULL )
 8000822:	e751      	b.n	80006c8 <xTaskCreate+0x1c>
 8000824:	2000145c 	.word	0x2000145c
 8000828:	2000151c 	.word	0x2000151c
 800082c:	200014b8 	.word	0x200014b8
 8000830:	200014a4 	.word	0x200014a4
 8000834:	20001490 	.word	0x20001490
 8000838:	20001474 	.word	0x20001474
 800083c:	20001460 	.word	0x20001460
 8000840:	2000148c 	.word	0x2000148c
 8000844:	20001488 	.word	0x20001488
 8000848:	20001440 	.word	0x20001440
 800084c:	20001454 	.word	0x20001454
 8000850:	20001450 	.word	0x20001450

08000854 <vTaskStartScheduler>:
{
 8000854:	b513      	push	{r0, r1, r4, lr}
        xReturn = xTaskCreate( prvIdleTask,
 8000856:	2400      	movs	r4, #0
 8000858:	4b10      	ldr	r3, [pc, #64]	; (800089c <vTaskStartScheduler+0x48>)
 800085a:	220a      	movs	r2, #10
 800085c:	9301      	str	r3, [sp, #4]
 800085e:	4910      	ldr	r1, [pc, #64]	; (80008a0 <vTaskStartScheduler+0x4c>)
 8000860:	4623      	mov	r3, r4
 8000862:	4810      	ldr	r0, [pc, #64]	; (80008a4 <vTaskStartScheduler+0x50>)
 8000864:	9400      	str	r4, [sp, #0]
 8000866:	f7ff ff21 	bl	80006ac <xTaskCreate>
    if( xReturn == pdPASS )
 800086a:	2801      	cmp	r0, #1
 800086c:	d111      	bne.n	8000892 <vTaskStartScheduler+0x3e>

    portFORCE_INLINE static void vPortRaiseBASEPRI( void )
    {
        uint32_t ulNewBASEPRI;

        __asm volatile
 800086e:	f04f 03bf 	mov.w	r3, #191	; 0xbf
 8000872:	f383 8811 	msr	BASEPRI, r3
 8000876:	f3bf 8f6f 	isb	sy
 800087a:	f3bf 8f4f 	dsb	sy
        xNextTaskUnblockTime = portMAX_DELAY;
 800087e:	f04f 32ff 	mov.w	r2, #4294967295	; 0xffffffff
 8000882:	4b09      	ldr	r3, [pc, #36]	; (80008a8 <vTaskStartScheduler+0x54>)
 8000884:	601a      	str	r2, [r3, #0]
        xSchedulerRunning = pdTRUE;
 8000886:	4b09      	ldr	r3, [pc, #36]	; (80008ac <vTaskStartScheduler+0x58>)
 8000888:	6018      	str	r0, [r3, #0]
        xTickCount = ( TickType_t ) configINITIAL_TICK_COUNT;
 800088a:	4b09      	ldr	r3, [pc, #36]	; (80008b0 <vTaskStartScheduler+0x5c>)
 800088c:	601c      	str	r4, [r3, #0]
        xPortStartScheduler();
 800088e:	f7ff fe7b 	bl	8000588 <xPortStartScheduler>
    ( void ) uxTopUsedPriority;
 8000892:	4b08      	ldr	r3, [pc, #32]	; (80008b4 <vTaskStartScheduler+0x60>)
 8000894:	681b      	ldr	r3, [r3, #0]
}
 8000896:	b002      	add	sp, #8
 8000898:	bd10      	pop	{r4, pc}
 800089a:	bf00      	nop
 800089c:	20001438 	.word	0x20001438
 80008a0:	080018bb 	.word	0x080018bb
 80008a4:	080005c5 	.word	0x080005c5
 80008a8:	2000143c 	.word	0x2000143c
 80008ac:	20001450 	.word	0x20001450
 80008b0:	20001458 	.word	0x20001458
 80008b4:	20000008 	.word	0x20000008

080008b8 <vTaskSuspendAll>:
    ++uxSchedulerSuspended;
 80008b8:	4a02      	ldr	r2, [pc, #8]	; (80008c4 <vTaskSuspendAll+0xc>)
 80008ba:	6813      	ldr	r3, [r2, #0]
 80008bc:	3301      	adds	r3, #1
 80008be:	6013      	str	r3, [r2, #0]
}
 80008c0:	4770      	bx	lr
 80008c2:	bf00      	nop
 80008c4:	20001434 	.word	0x20001434

080008c8 <xTaskGetTickCount>:
        xTicks = xTickCount;
 80008c8:	4b01      	ldr	r3, [pc, #4]	; (80008d0 <xTaskGetTickCount+0x8>)
 80008ca:	6818      	ldr	r0, [r3, #0]
}
 80008cc:	4770      	bx	lr
 80008ce:	bf00      	nop
 80008d0:	20001458 	.word	0x20001458

080008d4 <xTaskIncrementTick>:
{
 80008d4:	e92d 4ff8 	stmdb	sp!, {r3, r4, r5, r6, r7, r8, r9, sl, fp, lr}
    if( uxSchedulerSuspended == ( UBaseType_t ) pdFALSE )
 80008d8:	4b48      	ldr	r3, [pc, #288]	; (80009fc <xTaskIncrementTick+0x128>)
 80008da:	681b      	ldr	r3, [r3, #0]
 80008dc:	2b00      	cmp	r3, #0
 80008de:	f040 8086 	bne.w	80009ee <xTaskIncrementTick+0x11a>
        const TickType_t xConstTickCount = xTickCount + ( TickType_t ) 1;
 80008e2:	4b47      	ldr	r3, [pc, #284]	; (8000a00 <xTaskIncrementTick+0x12c>)
 80008e4:	681c      	ldr	r4, [r3, #0]
 80008e6:	3401      	adds	r4, #1
        xTickCount = xConstTickCount;
 80008e8:	601c      	str	r4, [r3, #0]
        if( xConstTickCount == ( TickType_t ) 0U ) /*lint !e774 'if' does not always evaluate to false as it is looking for an overflow. */
 80008ea:	b95c      	cbnz	r4, 8000904 <xTaskIncrementTick+0x30>
            taskSWITCH_DELAYED_LISTS();
 80008ec:	4a45      	ldr	r2, [pc, #276]	; (8000a04 <xTaskIncrementTick+0x130>)
 80008ee:	4b46      	ldr	r3, [pc, #280]	; (8000a08 <xTaskIncrementTick+0x134>)
 80008f0:	6811      	ldr	r1, [r2, #0]
 80008f2:	6818      	ldr	r0, [r3, #0]
 80008f4:	6010      	str	r0, [r2, #0]
 80008f6:	4a45      	ldr	r2, [pc, #276]	; (8000a0c <xTaskIncrementTick+0x138>)
 80008f8:	6019      	str	r1, [r3, #0]
 80008fa:	6813      	ldr	r3, [r2, #0]
 80008fc:	3301      	adds	r3, #1
 80008fe:	6013      	str	r3, [r2, #0]
 8000900:	f7ff fec2 	bl	8000688 <prvResetNextTaskUnblockTime>
        if( xConstTickCount >= xNextTaskUnblockTime )
 8000904:	f8df c108 	ldr.w	ip, [pc, #264]	; 8000a10 <xTaskIncrementTick+0x13c>
    BaseType_t xSwitchRequired = pdFALSE;
 8000908:	2000      	movs	r0, #0
        if( xConstTickCount >= xNextTaskUnblockTime )
 800090a:	f8dc 3000 	ldr.w	r3, [ip]
 800090e:	4a41      	ldr	r2, [pc, #260]	; (8000a14 <xTaskIncrementTick+0x140>)
 8000910:	429c      	cmp	r4, r3
 8000912:	f8df 9104 	ldr.w	r9, [pc, #260]	; 8000a18 <xTaskIncrementTick+0x144>
 8000916:	d20f      	bcs.n	8000938 <xTaskIncrementTick+0x64>
            if( listCURRENT_LIST_LENGTH( &( pxReadyTasksLists[ pxCurrentTCB->uxPriority ] ) ) > ( UBaseType_t ) 1 )
 8000918:	2114      	movs	r1, #20
 800091a:	f8d9 3000 	ldr.w	r3, [r9]
 800091e:	6adb      	ldr	r3, [r3, #44]	; 0x2c
 8000920:	434b      	muls	r3, r1
 8000922:	58d3      	ldr	r3, [r2, r3]
                xSwitchRequired = pdTRUE;
 8000924:	2b02      	cmp	r3, #2
            if( xYieldPending != pdFALSE )
 8000926:	4b3d      	ldr	r3, [pc, #244]	; (8000a1c <xTaskIncrementTick+0x148>)
                xSwitchRequired = pdTRUE;
 8000928:	bf28      	it	cs
 800092a:	2001      	movcs	r0, #1
            if( xYieldPending != pdFALSE )
 800092c:	681b      	ldr	r3, [r3, #0]
                xSwitchRequired = pdTRUE;
 800092e:	2b00      	cmp	r3, #0
 8000930:	bf18      	it	ne
 8000932:	2001      	movne	r0, #1
}
 8000934:	e8bd 8ff8 	ldmia.w	sp!, {r3, r4, r5, r6, r7, r8, r9, sl, fp, pc}
                if( listLIST_IS_EMPTY( pxDelayedTaskList ) != pdFALSE )
 8000938:	f8df 80c8 	ldr.w	r8, [pc, #200]	; 8000a04 <xTaskIncrementTick+0x130>
                    prvAddTaskToReadyList( pxTCB );
 800093c:	f8df e0e0 	ldr.w	lr, [pc, #224]	; 8000a20 <xTaskIncrementTick+0x14c>
                if( listLIST_IS_EMPTY( pxDelayedTaskList ) != pdFALSE )
 8000940:	f8d8 3000 	ldr.w	r3, [r8]
 8000944:	681b      	ldr	r3, [r3, #0]
 8000946:	b923      	cbnz	r3, 8000952 <xTaskIncrementTick+0x7e>
                    xNextTaskUnblockTime = portMAX_DELAY; /*lint !e961 MISRA exception as the casts are only redundant for some ports. */
 8000948:	f04f 33ff 	mov.w	r3, #4294967295	; 0xffffffff
 800094c:	f8cc 3000 	str.w	r3, [ip]
                    break;
 8000950:	e7e2      	b.n	8000918 <xTaskIncrementTick+0x44>
                    pxTCB = listGET_OWNER_OF_HEAD_ENTRY( pxDelayedTaskList ); /*lint !e9079 void * is used as this macro is used with timers and co-routines too.  Alignment is known to be fine as the type of the pointer stored and retrieved is the same. */
 8000952:	f8d8 3000 	ldr.w	r3, [r8]
 8000956:	68db      	ldr	r3, [r3, #12]
 8000958:	68db      	ldr	r3, [r3, #12]
                    xItemValue = listGET_LIST_ITEM_VALUE( &( pxTCB->xStateListItem ) );
 800095a:	6859      	ldr	r1, [r3, #4]
                    if( xConstTickCount < xItemValue )
 800095c:	428c      	cmp	r4, r1
 800095e:	d202      	bcs.n	8000966 <xTaskIncrementTick+0x92>
                        xNextTaskUnblockTime = xItemValue;
 8000960:	f8cc 1000 	str.w	r1, [ip]
                        break; /*lint !e9011 Code structure here is deemed easier to understand with multiple breaks. */
 8000964:	e7d8      	b.n	8000918 <xTaskIncrementTick+0x44>
                    listREMOVE_ITEM( &( pxTCB->xStateListItem ) );
 8000966:	695d      	ldr	r5, [r3, #20]
 8000968:	e9d3 1602 	ldrd	r1, r6, [r3, #8]
 800096c:	608e      	str	r6, [r1, #8]
 800096e:	6071      	str	r1, [r6, #4]
 8000970:	6869      	ldr	r1, [r5, #4]
 8000972:	1d1f      	adds	r7, r3, #4
 8000974:	42b9      	cmp	r1, r7
 8000976:	f04f 0100 	mov.w	r1, #0
 800097a:	bf08      	it	eq
 800097c:	606e      	streq	r6, [r5, #4]
 800097e:	6159      	str	r1, [r3, #20]
 8000980:	6829      	ldr	r1, [r5, #0]
 8000982:	3901      	subs	r1, #1
 8000984:	6029      	str	r1, [r5, #0]
                    if( listLIST_ITEM_CONTAINER( &( pxTCB->xEventListItem ) ) != NULL )
 8000986:	6a9d      	ldr	r5, [r3, #40]	; 0x28
 8000988:	b17d      	cbz	r5, 80009aa <xTaskIncrementTick+0xd6>
                        listREMOVE_ITEM( &( pxTCB->xEventListItem ) );
 800098a:	e9d3 1607 	ldrd	r1, r6, [r3, #28]
 800098e:	608e      	str	r6, [r1, #8]
 8000990:	6071      	str	r1, [r6, #4]
 8000992:	6869      	ldr	r1, [r5, #4]
 8000994:	f103 0a18 	add.w	sl, r3, #24
 8000998:	4551      	cmp	r1, sl
 800099a:	f04f 0100 	mov.w	r1, #0
 800099e:	bf08      	it	eq
 80009a0:	606e      	streq	r6, [r5, #4]
 80009a2:	6299      	str	r1, [r3, #40]	; 0x28
 80009a4:	6829      	ldr	r1, [r5, #0]
 80009a6:	3901      	subs	r1, #1
 80009a8:	6029      	str	r1, [r5, #0]
                    prvAddTaskToReadyList( pxTCB );
 80009aa:	2501      	movs	r5, #1
 80009ac:	6ad9      	ldr	r1, [r3, #44]	; 0x2c
 80009ae:	f8de 6000 	ldr.w	r6, [lr]
 80009b2:	408d      	lsls	r5, r1
 80009b4:	4335      	orrs	r5, r6
 80009b6:	f8ce 5000 	str.w	r5, [lr]
 80009ba:	2514      	movs	r5, #20
 80009bc:	434d      	muls	r5, r1
 80009be:	eb02 0a05 	add.w	sl, r2, r5
 80009c2:	f8da 6004 	ldr.w	r6, [sl, #4]
 80009c6:	f8d6 b008 	ldr.w	fp, [r6, #8]
 80009ca:	609e      	str	r6, [r3, #8]
 80009cc:	f8c3 b00c 	str.w	fp, [r3, #12]
 80009d0:	f8cb 7004 	str.w	r7, [fp, #4]
 80009d4:	60b7      	str	r7, [r6, #8]
 80009d6:	f8c3 a014 	str.w	sl, [r3, #20]
 80009da:	5953      	ldr	r3, [r2, r5]
 80009dc:	3301      	adds	r3, #1
 80009de:	5153      	str	r3, [r2, r5]
                        if( pxTCB->uxPriority > pxCurrentTCB->uxPriority )
 80009e0:	f8d9 3000 	ldr.w	r3, [r9]
 80009e4:	6adb      	ldr	r3, [r3, #44]	; 0x2c
                            xSwitchRequired = pdTRUE;
 80009e6:	4299      	cmp	r1, r3
 80009e8:	bf88      	it	hi
 80009ea:	2001      	movhi	r0, #1
 80009ec:	e7a8      	b.n	8000940 <xTaskIncrementTick+0x6c>
        ++xPendedTicks;
 80009ee:	4a0d      	ldr	r2, [pc, #52]	; (8000a24 <xTaskIncrementTick+0x150>)
    BaseType_t xSwitchRequired = pdFALSE;
 80009f0:	2000      	movs	r0, #0
        ++xPendedTicks;
 80009f2:	6813      	ldr	r3, [r2, #0]
 80009f4:	3301      	adds	r3, #1
 80009f6:	6013      	str	r3, [r2, #0]
 80009f8:	e79c      	b.n	8000934 <xTaskIncrementTick+0x60>
 80009fa:	bf00      	nop
 80009fc:	20001434 	.word	0x20001434
 8000a00:	20001458 	.word	0x20001458
 8000a04:	2000148c 	.word	0x2000148c
 8000a08:	20001488 	.word	0x20001488
 8000a0c:	20001444 	.word	0x20001444
 8000a10:	2000143c 	.word	0x2000143c
 8000a14:	200014b8 	.word	0x200014b8
 8000a18:	2000151c 	.word	0x2000151c
 8000a1c:	20001448 	.word	0x20001448
 8000a20:	20001454 	.word	0x20001454
 8000a24:	2000144c 	.word	0x2000144c

08000a28 <xTaskResumeAll>:
{
 8000a28:	e92d 4ff8 	stmdb	sp!, {r3, r4, r5, r6, r7, r8, r9, sl, fp, lr}
    taskENTER_CRITICAL();
 8000a2c:	f7ff fd4a 	bl	80004c4 <vPortEnterCritical>
        --uxSchedulerSuspended;
 8000a30:	4b3e      	ldr	r3, [pc, #248]	; (8000b2c <xTaskResumeAll+0x104>)
 8000a32:	681a      	ldr	r2, [r3, #0]
 8000a34:	3a01      	subs	r2, #1
 8000a36:	601a      	str	r2, [r3, #0]
        if( uxSchedulerSuspended == ( UBaseType_t ) pdFALSE )
 8000a38:	681b      	ldr	r3, [r3, #0]
 8000a3a:	b12b      	cbz	r3, 8000a48 <xTaskResumeAll+0x20>
    BaseType_t xAlreadyYielded = pdFALSE;
 8000a3c:	2400      	movs	r4, #0
    taskEXIT_CRITICAL();
 8000a3e:	f7ff fd51 	bl	80004e4 <vPortExitCritical>
}
 8000a42:	4620      	mov	r0, r4
 8000a44:	e8bd 8ff8 	ldmia.w	sp!, {r3, r4, r5, r6, r7, r8, r9, sl, fp, pc}
            if( uxCurrentNumberOfTasks > ( UBaseType_t ) 0U )
 8000a48:	4a39      	ldr	r2, [pc, #228]	; (8000b30 <xTaskResumeAll+0x108>)
 8000a4a:	6812      	ldr	r2, [r2, #0]
 8000a4c:	2a00      	cmp	r2, #0
 8000a4e:	d0f5      	beq.n	8000a3c <xTaskResumeAll+0x14>
                    prvAddTaskToReadyList( pxTCB );
 8000a50:	f04f 0c01 	mov.w	ip, #1
 8000a54:	f04f 0e14 	mov.w	lr, #20
                while( listLIST_IS_EMPTY( &xPendingReadyList ) == pdFALSE )
 8000a58:	4e36      	ldr	r6, [pc, #216]	; (8000b34 <xTaskResumeAll+0x10c>)
                    prvAddTaskToReadyList( pxTCB );
 8000a5a:	4f37      	ldr	r7, [pc, #220]	; (8000b38 <xTaskResumeAll+0x110>)
 8000a5c:	4a37      	ldr	r2, [pc, #220]	; (8000b3c <xTaskResumeAll+0x114>)
                    if( pxTCB->uxPriority >= pxCurrentTCB->uxPriority )
 8000a5e:	f8df 80e0 	ldr.w	r8, [pc, #224]	; 8000b40 <xTaskResumeAll+0x118>
                        xYieldPending = pdTRUE;
 8000a62:	f8df 90e0 	ldr.w	r9, [pc, #224]	; 8000b44 <xTaskResumeAll+0x11c>
 8000a66:	e03f      	b.n	8000ae8 <xTaskResumeAll+0xc0>
                    pxTCB = listGET_OWNER_OF_HEAD_ENTRY( ( &xPendingReadyList ) ); /*lint !e9079 void * is used as this macro is used with timers and co-routines too.  Alignment is known to be fine as the type of the pointer stored and retrieved is the same. */
 8000a68:	68f3      	ldr	r3, [r6, #12]
 8000a6a:	68db      	ldr	r3, [r3, #12]
                    listREMOVE_ITEM( &( pxTCB->xEventListItem ) );
 8000a6c:	6a98      	ldr	r0, [r3, #40]	; 0x28
 8000a6e:	e9d3 1407 	ldrd	r1, r4, [r3, #28]
 8000a72:	608c      	str	r4, [r1, #8]
 8000a74:	6061      	str	r1, [r4, #4]
 8000a76:	6841      	ldr	r1, [r0, #4]
 8000a78:	f103 0518 	add.w	r5, r3, #24
 8000a7c:	42a9      	cmp	r1, r5
 8000a7e:	f04f 0100 	mov.w	r1, #0
 8000a82:	bf08      	it	eq
 8000a84:	6044      	streq	r4, [r0, #4]
 8000a86:	6299      	str	r1, [r3, #40]	; 0x28
 8000a88:	6801      	ldr	r1, [r0, #0]
 8000a8a:	3901      	subs	r1, #1
 8000a8c:	6001      	str	r1, [r0, #0]
                    listREMOVE_ITEM( &( pxTCB->xStateListItem ) );
 8000a8e:	6958      	ldr	r0, [r3, #20]
 8000a90:	e9d3 1402 	ldrd	r1, r4, [r3, #8]
 8000a94:	608c      	str	r4, [r1, #8]
 8000a96:	6061      	str	r1, [r4, #4]
 8000a98:	6841      	ldr	r1, [r0, #4]
 8000a9a:	1d1d      	adds	r5, r3, #4
 8000a9c:	42a9      	cmp	r1, r5
 8000a9e:	6801      	ldr	r1, [r0, #0]
 8000aa0:	bf08      	it	eq
 8000aa2:	6044      	streq	r4, [r0, #4]
 8000aa4:	3901      	subs	r1, #1
 8000aa6:	6001      	str	r1, [r0, #0]
                    prvAddTaskToReadyList( pxTCB );
 8000aa8:	6ad9      	ldr	r1, [r3, #44]	; 0x2c
 8000aaa:	683c      	ldr	r4, [r7, #0]
 8000aac:	fa0c f001 	lsl.w	r0, ip, r1
 8000ab0:	4320      	orrs	r0, r4
 8000ab2:	6038      	str	r0, [r7, #0]
 8000ab4:	fb0e f001 	mul.w	r0, lr, r1
 8000ab8:	eb02 0a00 	add.w	sl, r2, r0
 8000abc:	f8da 4004 	ldr.w	r4, [sl, #4]
 8000ac0:	f8d4 b008 	ldr.w	fp, [r4, #8]
 8000ac4:	609c      	str	r4, [r3, #8]
 8000ac6:	f8c3 b00c 	str.w	fp, [r3, #12]
 8000aca:	f8cb 5004 	str.w	r5, [fp, #4]
 8000ace:	60a5      	str	r5, [r4, #8]
 8000ad0:	5814      	ldr	r4, [r2, r0]
 8000ad2:	f8c3 a014 	str.w	sl, [r3, #20]
 8000ad6:	3401      	adds	r4, #1
 8000ad8:	5014      	str	r4, [r2, r0]
                    if( pxTCB->uxPriority >= pxCurrentTCB->uxPriority )
 8000ada:	f8d8 0000 	ldr.w	r0, [r8]
 8000ade:	6ac0      	ldr	r0, [r0, #44]	; 0x2c
 8000ae0:	4281      	cmp	r1, r0
 8000ae2:	d301      	bcc.n	8000ae8 <xTaskResumeAll+0xc0>
                        xYieldPending = pdTRUE;
 8000ae4:	f8c9 c000 	str.w	ip, [r9]
                while( listLIST_IS_EMPTY( &xPendingReadyList ) == pdFALSE )
 8000ae8:	6831      	ldr	r1, [r6, #0]
 8000aea:	2900      	cmp	r1, #0
 8000aec:	d1bc      	bne.n	8000a68 <xTaskResumeAll+0x40>
                if( pxTCB != NULL )
 8000aee:	b10b      	cbz	r3, 8000af4 <xTaskResumeAll+0xcc>
                    prvResetNextTaskUnblockTime();
 8000af0:	f7ff fdca 	bl	8000688 <prvResetNextTaskUnblockTime>
                    TickType_t xPendedCounts = xPendedTicks; /* Non-volatile copy. */
 8000af4:	4d14      	ldr	r5, [pc, #80]	; (8000b48 <xTaskResumeAll+0x120>)
 8000af6:	682c      	ldr	r4, [r5, #0]
                    if( xPendedCounts > ( TickType_t ) 0U )
 8000af8:	b144      	cbz	r4, 8000b0c <xTaskResumeAll+0xe4>
                                xYieldPending = pdTRUE;
 8000afa:	2701      	movs	r7, #1
 8000afc:	4e11      	ldr	r6, [pc, #68]	; (8000b44 <xTaskResumeAll+0x11c>)
                            if( xTaskIncrementTick() != pdFALSE )
 8000afe:	f7ff fee9 	bl	80008d4 <xTaskIncrementTick>
 8000b02:	b100      	cbz	r0, 8000b06 <xTaskResumeAll+0xde>
                                xYieldPending = pdTRUE;
 8000b04:	6037      	str	r7, [r6, #0]
                        } while( xPendedCounts > ( TickType_t ) 0U );
 8000b06:	3c01      	subs	r4, #1
 8000b08:	d1f9      	bne.n	8000afe <xTaskResumeAll+0xd6>
                        xPendedTicks = 0;
 8000b0a:	602c      	str	r4, [r5, #0]
                if( xYieldPending != pdFALSE )
 8000b0c:	4b0d      	ldr	r3, [pc, #52]	; (8000b44 <xTaskResumeAll+0x11c>)
 8000b0e:	681b      	ldr	r3, [r3, #0]
 8000b10:	2b00      	cmp	r3, #0
 8000b12:	d093      	beq.n	8000a3c <xTaskResumeAll+0x14>
                    taskYIELD_IF_USING_PREEMPTION();
 8000b14:	f04f 23e0 	mov.w	r3, #3758153728	; 0xe000e000
 8000b18:	f04f 5280 	mov.w	r2, #268435456	; 0x10000000
 8000b1c:	f8c3 2d04 	str.w	r2, [r3, #3332]	; 0xd04
 8000b20:	f3bf 8f4f 	dsb	sy
 8000b24:	f3bf 8f6f 	isb	sy
                        xAlreadyYielded = pdTRUE;
 8000b28:	2401      	movs	r4, #1
 8000b2a:	e788      	b.n	8000a3e <xTaskResumeAll+0x16>
 8000b2c:	20001434 	.word	0x20001434
 8000b30:	2000145c 	.word	0x2000145c
 8000b34:	20001474 	.word	0x20001474
 8000b38:	20001454 	.word	0x20001454
 8000b3c:	200014b8 	.word	0x200014b8
 8000b40:	2000151c 	.word	0x2000151c
 8000b44:	20001448 	.word	0x20001448
 8000b48:	2000144c 	.word	0x2000144c

08000b4c <xTaskDelayUntil>:
    {
 8000b4c:	b510      	push	{r4, lr}
        vTaskSuspendAll();
 8000b4e:	f7ff feb3 	bl	80008b8 <vTaskSuspendAll>
            const TickType_t xConstTickCount = xTickCount;
 8000b52:	4b13      	ldr	r3, [pc, #76]	; (8000ba0 <xTaskDelayUntil+0x54>)
            xTimeToWake = *pxPreviousWakeTime + xTimeIncrement;
 8000b54:	6804      	ldr	r4, [r0, #0]
            const TickType_t xConstTickCount = xTickCount;
 8000b56:	681a      	ldr	r2, [r3, #0]
            xTimeToWake = *pxPreviousWakeTime + xTimeIncrement;
 8000b58:	1863      	adds	r3, r4, r1
 8000b5a:	bf2c      	ite	cs
 8000b5c:	2101      	movcs	r1, #1
 8000b5e:	2100      	movcc	r1, #0
            if( xConstTickCount < *pxPreviousWakeTime )
 8000b60:	4294      	cmp	r4, r2
 8000b62:	d913      	bls.n	8000b8c <xTaskDelayUntil+0x40>
                if( ( xTimeToWake < *pxPreviousWakeTime ) && ( xTimeToWake > xConstTickCount ) )
 8000b64:	b109      	cbz	r1, 8000b6a <xTaskDelayUntil+0x1e>
 8000b66:	429a      	cmp	r2, r3
 8000b68:	d312      	bcc.n	8000b90 <xTaskDelayUntil+0x44>
        BaseType_t xAlreadyYielded, xShouldDelay = pdFALSE;
 8000b6a:	2400      	movs	r4, #0
            *pxPreviousWakeTime = xTimeToWake;
 8000b6c:	6003      	str	r3, [r0, #0]
        xAlreadyYielded = xTaskResumeAll();
 8000b6e:	f7ff ff5b 	bl	8000a28 <xTaskResumeAll>
        if( xAlreadyYielded == pdFALSE )
 8000b72:	b948      	cbnz	r0, 8000b88 <xTaskDelayUntil+0x3c>
            portYIELD_WITHIN_API();
 8000b74:	f04f 23e0 	mov.w	r3, #3758153728	; 0xe000e000
 8000b78:	f04f 5280 	mov.w	r2, #268435456	; 0x10000000
 8000b7c:	f8c3 2d04 	str.w	r2, [r3, #3332]	; 0xd04
 8000b80:	f3bf 8f4f 	dsb	sy
 8000b84:	f3bf 8f6f 	isb	sy
    }
 8000b88:	4620      	mov	r0, r4
 8000b8a:	bd10      	pop	{r4, pc}
                if( ( xTimeToWake < *pxPreviousWakeTime ) || ( xTimeToWake > xConstTickCount ) )
 8000b8c:	2900      	cmp	r1, #0
 8000b8e:	d0ea      	beq.n	8000b66 <xTaskDelayUntil+0x1a>
            *pxPreviousWakeTime = xTimeToWake;
 8000b90:	6003      	str	r3, [r0, #0]
                prvAddCurrentTaskToDelayedList( xTimeToWake - xConstTickCount, pdFALSE );
 8000b92:	2100      	movs	r1, #0
 8000b94:	1a98      	subs	r0, r3, r2
 8000b96:	f7ff fd27 	bl	80005e8 <prvAddCurrentTaskToDelayedList>
 8000b9a:	2401      	movs	r4, #1
 8000b9c:	e7e7      	b.n	8000b6e <xTaskDelayUntil+0x22>
 8000b9e:	bf00      	nop
 8000ba0:	20001458 	.word	0x20001458

08000ba4 <vTaskSwitchContext>:
    if( uxSchedulerSuspended != ( UBaseType_t ) pdFALSE )
 8000ba4:	4b12      	ldr	r3, [pc, #72]	; (8000bf0 <vTaskSwitchContext+0x4c>)
{
 8000ba6:	b530      	push	{r4, r5, lr}
    if( uxSchedulerSuspended != ( UBaseType_t ) pdFALSE )
 8000ba8:	681a      	ldr	r2, [r3, #0]
 8000baa:	4b12      	ldr	r3, [pc, #72]	; (8000bf4 <vTaskSwitchContext+0x50>)
 8000bac:	b112      	cbz	r2, 8000bb4 <vTaskSwitchContext+0x10>
        xYieldPending = pdTRUE;
 8000bae:	2201      	movs	r2, #1
        taskSELECT_HIGHEST_PRIORITY_TASK(); /*lint !e9079 void * is used as this macro is used with timers and co-routines too.  Alignment is known to be fine as the type of the pointer stored and retrieved is the same. */
 8000bb0:	601a      	str	r2, [r3, #0]
}
 8000bb2:	bd30      	pop	{r4, r5, pc}
        xYieldPending = pdFALSE;
 8000bb4:	601a      	str	r2, [r3, #0]
        taskSELECT_HIGHEST_PRIORITY_TASK(); /*lint !e9079 void * is used as this macro is used with timers and co-routines too.  Alignment is known to be fine as the type of the pointer stored and retrieved is the same. */
 8000bb6:	4b10      	ldr	r3, [pc, #64]	; (8000bf8 <vTaskSwitchContext+0x54>)
 8000bb8:	681b      	ldr	r3, [r3, #0]
            __asm volatile ( "clz %0, %1" : "=r" ( ucReturn ) : "r" ( ulBitmap ) : "memory" );
 8000bba:	fab3 f383 	clz	r3, r3
 8000bbe:	2514      	movs	r5, #20
 8000bc0:	b2db      	uxtb	r3, r3
 8000bc2:	f1c3 031f 	rsb	r3, r3, #31
 8000bc6:	fb05 f203 	mul.w	r2, r5, r3
 8000bca:	490c      	ldr	r1, [pc, #48]	; (8000bfc <vTaskSwitchContext+0x58>)
 8000bcc:	1888      	adds	r0, r1, r2
 8000bce:	6844      	ldr	r4, [r0, #4]
 8000bd0:	3208      	adds	r2, #8
 8000bd2:	6864      	ldr	r4, [r4, #4]
 8000bd4:	440a      	add	r2, r1
 8000bd6:	4294      	cmp	r4, r2
 8000bd8:	fb05 1103 	mla	r1, r5, r3, r1
 8000bdc:	bf08      	it	eq
 8000bde:	6862      	ldreq	r2, [r4, #4]
 8000be0:	6044      	str	r4, [r0, #4]
 8000be2:	bf08      	it	eq
 8000be4:	6042      	streq	r2, [r0, #4]
 8000be6:	684b      	ldr	r3, [r1, #4]
 8000be8:	68da      	ldr	r2, [r3, #12]
 8000bea:	4b05      	ldr	r3, [pc, #20]	; (8000c00 <vTaskSwitchContext+0x5c>)
 8000bec:	e7e0      	b.n	8000bb0 <vTaskSwitchContext+0xc>
 8000bee:	bf00      	nop
 8000bf0:	20001434 	.word	0x20001434
 8000bf4:	20001448 	.word	0x20001448
 8000bf8:	20001454 	.word	0x20001454
 8000bfc:	200014b8 	.word	0x200014b8
 8000c00:	2000151c 	.word	0x2000151c

08000c04 <vTaskPlaceOnEventList>:
{
 8000c04:	b510      	push	{r4, lr}
 8000c06:	460c      	mov	r4, r1
    vListInsert( pxEventList, &( pxCurrentTCB->xEventListItem ) );
 8000c08:	4b05      	ldr	r3, [pc, #20]	; (8000c20 <vTaskPlaceOnEventList+0x1c>)
 8000c0a:	6819      	ldr	r1, [r3, #0]
 8000c0c:	3118      	adds	r1, #24
 8000c0e:	f000 fb84 	bl	800131a <vListInsert>
    prvAddCurrentTaskToDelayedList( xTicksToWait, pdTRUE );
 8000c12:	4620      	mov	r0, r4
}
 8000c14:	e8bd 4010 	ldmia.w	sp!, {r4, lr}
    prvAddCurrentTaskToDelayedList( xTicksToWait, pdTRUE );
 8000c18:	2101      	movs	r1, #1
 8000c1a:	f7ff bce5 	b.w	80005e8 <prvAddCurrentTaskToDelayedList>
 8000c1e:	bf00      	nop
 8000c20:	2000151c 	.word	0x2000151c

08000c24 <xTaskRemoveFromEventList>:
    pxUnblockedTCB = listGET_OWNER_OF_HEAD_ENTRY( pxEventList ); /*lint !e9079 void * is used as this macro is used with timers and co-routines too.  Alignment is known to be fine as the type of the pointer stored and retrieved is the same. */
 8000c24:	68c3      	ldr	r3, [r0, #12]
{
 8000c26:	b5f0      	push	{r4, r5, r6, r7, lr}
    pxUnblockedTCB = listGET_OWNER_OF_HEAD_ENTRY( pxEventList ); /*lint !e9079 void * is used as this macro is used with timers and co-routines too.  Alignment is known to be fine as the type of the pointer stored and retrieved is the same. */
 8000c28:	68db      	ldr	r3, [r3, #12]
    listREMOVE_ITEM( &( pxUnblockedTCB->xEventListItem ) );
 8000c2a:	6a9a      	ldr	r2, [r3, #40]	; 0x28
 8000c2c:	e9d3 0107 	ldrd	r0, r1, [r3, #28]
 8000c30:	6081      	str	r1, [r0, #8]
 8000c32:	6048      	str	r0, [r1, #4]
 8000c34:	6850      	ldr	r0, [r2, #4]
 8000c36:	f103 0418 	add.w	r4, r3, #24
 8000c3a:	42a0      	cmp	r0, r4
 8000c3c:	bf08      	it	eq
 8000c3e:	6051      	streq	r1, [r2, #4]
 8000c40:	2100      	movs	r1, #0
 8000c42:	6299      	str	r1, [r3, #40]	; 0x28
 8000c44:	6811      	ldr	r1, [r2, #0]
 8000c46:	3901      	subs	r1, #1
 8000c48:	6011      	str	r1, [r2, #0]
    if( uxSchedulerSuspended == ( UBaseType_t ) pdFALSE )
 8000c4a:	4a1e      	ldr	r2, [pc, #120]	; (8000cc4 <xTaskRemoveFromEventList+0xa0>)
 8000c4c:	6ad9      	ldr	r1, [r3, #44]	; 0x2c
 8000c4e:	6812      	ldr	r2, [r2, #0]
 8000c50:	2a00      	cmp	r2, #0
 8000c52:	d12a      	bne.n	8000caa <xTaskRemoveFromEventList+0x86>
        listREMOVE_ITEM( &( pxUnblockedTCB->xStateListItem ) );
 8000c54:	e9d3 4002 	ldrd	r4, r0, [r3, #8]
 8000c58:	695a      	ldr	r2, [r3, #20]
 8000c5a:	60a0      	str	r0, [r4, #8]
 8000c5c:	6044      	str	r4, [r0, #4]
 8000c5e:	6854      	ldr	r4, [r2, #4]
 8000c60:	1d1d      	adds	r5, r3, #4
 8000c62:	42ac      	cmp	r4, r5
 8000c64:	bf08      	it	eq
 8000c66:	6050      	streq	r0, [r2, #4]
 8000c68:	6810      	ldr	r0, [r2, #0]
 8000c6a:	3801      	subs	r0, #1
 8000c6c:	6010      	str	r0, [r2, #0]
        prvAddTaskToReadyList( pxUnblockedTCB );
 8000c6e:	2201      	movs	r2, #1
 8000c70:	4815      	ldr	r0, [pc, #84]	; (8000cc8 <xTaskRemoveFromEventList+0xa4>)
 8000c72:	408a      	lsls	r2, r1
 8000c74:	6804      	ldr	r4, [r0, #0]
 8000c76:	4322      	orrs	r2, r4
 8000c78:	6002      	str	r2, [r0, #0]
 8000c7a:	2214      	movs	r2, #20
 8000c7c:	434a      	muls	r2, r1
 8000c7e:	4813      	ldr	r0, [pc, #76]	; (8000ccc <xTaskRemoveFromEventList+0xa8>)
 8000c80:	1886      	adds	r6, r0, r2
 8000c82:	6874      	ldr	r4, [r6, #4]
 8000c84:	68a7      	ldr	r7, [r4, #8]
 8000c86:	609c      	str	r4, [r3, #8]
 8000c88:	60df      	str	r7, [r3, #12]
 8000c8a:	607d      	str	r5, [r7, #4]
 8000c8c:	60a5      	str	r5, [r4, #8]
 8000c8e:	615e      	str	r6, [r3, #20]
 8000c90:	5883      	ldr	r3, [r0, r2]
 8000c92:	3301      	adds	r3, #1
 8000c94:	5083      	str	r3, [r0, r2]
    if( pxUnblockedTCB->uxPriority > pxCurrentTCB->uxPriority )
 8000c96:	4b0e      	ldr	r3, [pc, #56]	; (8000cd0 <xTaskRemoveFromEventList+0xac>)
 8000c98:	681b      	ldr	r3, [r3, #0]
 8000c9a:	6adb      	ldr	r3, [r3, #44]	; 0x2c
 8000c9c:	4299      	cmp	r1, r3
        xYieldPending = pdTRUE;
 8000c9e:	bf85      	ittet	hi
 8000ca0:	2001      	movhi	r0, #1
 8000ca2:	4b0c      	ldrhi	r3, [pc, #48]	; (8000cd4 <xTaskRemoveFromEventList+0xb0>)
        xReturn = pdFALSE;
 8000ca4:	2000      	movls	r0, #0
        xYieldPending = pdTRUE;
 8000ca6:	6018      	strhi	r0, [r3, #0]
}
 8000ca8:	bdf0      	pop	{r4, r5, r6, r7, pc}
        listINSERT_END( &( xPendingReadyList ), &( pxUnblockedTCB->xEventListItem ) );
 8000caa:	4a0b      	ldr	r2, [pc, #44]	; (8000cd8 <xTaskRemoveFromEventList+0xb4>)
 8000cac:	6850      	ldr	r0, [r2, #4]
 8000cae:	6885      	ldr	r5, [r0, #8]
 8000cb0:	61d8      	str	r0, [r3, #28]
 8000cb2:	621d      	str	r5, [r3, #32]
 8000cb4:	606c      	str	r4, [r5, #4]
 8000cb6:	6084      	str	r4, [r0, #8]
 8000cb8:	629a      	str	r2, [r3, #40]	; 0x28
 8000cba:	6813      	ldr	r3, [r2, #0]
 8000cbc:	3301      	adds	r3, #1
 8000cbe:	6013      	str	r3, [r2, #0]
 8000cc0:	e7e9      	b.n	8000c96 <xTaskRemoveFromEventList+0x72>
 8000cc2:	bf00      	nop
 8000cc4:	20001434 	.word	0x20001434
 8000cc8:	20001454 	.word	0x20001454
 8000ccc:	200014b8 	.word	0x200014b8
 8000cd0:	2000151c 	.word	0x2000151c
 8000cd4:	20001448 	.word	0x20001448
 8000cd8:	20001474 	.word	0x20001474

08000cdc <vTaskInternalSetTimeOutState>:
    pxTimeOut->xOverflowCount = xNumOfOverflows;
 8000cdc:	4b03      	ldr	r3, [pc, #12]	; (8000cec <vTaskInternalSetTimeOutState+0x10>)
 8000cde:	681b      	ldr	r3, [r3, #0]
 8000ce0:	6003      	str	r3, [r0, #0]
    pxTimeOut->xTimeOnEntering = xTickCount;
 8000ce2:	4b03      	ldr	r3, [pc, #12]	; (8000cf0 <vTaskInternalSetTimeOutState+0x14>)
 8000ce4:	681b      	ldr	r3, [r3, #0]
 8000ce6:	6043      	str	r3, [r0, #4]
}
 8000ce8:	4770      	bx	lr
 8000cea:	bf00      	nop
 8000cec:	20001444 	.word	0x20001444
 8000cf0:	20001458 	.word	0x20001458

08000cf4 <xTaskCheckForTimeOut>:
{
 8000cf4:	b570      	push	{r4, r5, r6, lr}
 8000cf6:	460d      	mov	r5, r1
 8000cf8:	4604      	mov	r4, r0
    taskENTER_CRITICAL();
 8000cfa:	f7ff fbe3 	bl	80004c4 <vPortEnterCritical>
        const TickType_t xConstTickCount = xTickCount;
 8000cfe:	4b0f      	ldr	r3, [pc, #60]	; (8000d3c <xTaskCheckForTimeOut+0x48>)
 8000d00:	6819      	ldr	r1, [r3, #0]
            if( *pxTicksToWait == portMAX_DELAY )
 8000d02:	682b      	ldr	r3, [r5, #0]
 8000d04:	1c5a      	adds	r2, r3, #1
 8000d06:	d017      	beq.n	8000d38 <xTaskCheckForTimeOut+0x44>
        if( ( xNumOfOverflows != pxTimeOut->xOverflowCount ) && ( xConstTickCount >= pxTimeOut->xTimeOnEntering ) ) /*lint !e525 Indentation preferred as is to make code within pre-processor directives clearer. */
 8000d08:	480d      	ldr	r0, [pc, #52]	; (8000d40 <xTaskCheckForTimeOut+0x4c>)
 8000d0a:	6826      	ldr	r6, [r4, #0]
 8000d0c:	6800      	ldr	r0, [r0, #0]
        const TickType_t xElapsedTime = xConstTickCount - pxTimeOut->xTimeOnEntering;
 8000d0e:	6862      	ldr	r2, [r4, #4]
        if( ( xNumOfOverflows != pxTimeOut->xOverflowCount ) && ( xConstTickCount >= pxTimeOut->xTimeOnEntering ) ) /*lint !e525 Indentation preferred as is to make code within pre-processor directives clearer. */
 8000d10:	4286      	cmp	r6, r0
 8000d12:	d008      	beq.n	8000d26 <xTaskCheckForTimeOut+0x32>
 8000d14:	428a      	cmp	r2, r1
 8000d16:	d806      	bhi.n	8000d26 <xTaskCheckForTimeOut+0x32>
            *pxTicksToWait = ( TickType_t ) 0;
 8000d18:	2300      	movs	r3, #0
            xReturn = pdTRUE;
 8000d1a:	2401      	movs	r4, #1
            *pxTicksToWait = ( TickType_t ) 0;
 8000d1c:	602b      	str	r3, [r5, #0]
    taskEXIT_CRITICAL();
 8000d1e:	f7ff fbe1 	bl	80004e4 <vPortExitCritical>
}
 8000d22:	4620      	mov	r0, r4
 8000d24:	bd70      	pop	{r4, r5, r6, pc}
        const TickType_t xElapsedTime = xConstTickCount - pxTimeOut->xTimeOnEntering;
 8000d26:	1a88      	subs	r0, r1, r2
        else if( xElapsedTime < *pxTicksToWait ) /*lint !e961 Explicit casting is only redundant with some compilers, whereas others require it to prevent integer conversion errors. */
 8000d28:	4283      	cmp	r3, r0
 8000d2a:	d9f5      	bls.n	8000d18 <xTaskCheckForTimeOut+0x24>
            *pxTicksToWait -= xElapsedTime;
 8000d2c:	1a5b      	subs	r3, r3, r1
 8000d2e:	4413      	add	r3, r2
            vTaskInternalSetTimeOutState( pxTimeOut );
 8000d30:	4620      	mov	r0, r4
            *pxTicksToWait -= xElapsedTime;
 8000d32:	602b      	str	r3, [r5, #0]
            vTaskInternalSetTimeOutState( pxTimeOut );
 8000d34:	f7ff ffd2 	bl	8000cdc <vTaskInternalSetTimeOutState>
                xReturn = pdFALSE;
 8000d38:	2400      	movs	r4, #0
 8000d3a:	e7f0      	b.n	8000d1e <xTaskCheckForTimeOut+0x2a>
 8000d3c:	20001458 	.word	0x20001458
 8000d40:	20001444 	.word	0x20001444

08000d44 <vTaskMissedYield>:
    xYieldPending = pdTRUE;
 8000d44:	2201      	movs	r2, #1
 8000d46:	4b01      	ldr	r3, [pc, #4]	; (8000d4c <vTaskMissedYield+0x8>)
 8000d48:	601a      	str	r2, [r3, #0]
}
 8000d4a:	4770      	bx	lr
 8000d4c:	20001448 	.word	0x20001448

08000d50 <xTaskPriorityInherit>:
    {
 8000d50:	b5f8      	push	{r3, r4, r5, r6, r7, lr}
        if( pxMutexHolder != NULL )
 8000d52:	4604      	mov	r4, r0
 8000d54:	2800      	cmp	r0, #0
 8000d56:	d037      	beq.n	8000dc8 <xTaskPriorityInherit+0x78>
            if( pxMutexHolderTCB->uxPriority < pxCurrentTCB->uxPriority )
 8000d58:	4d22      	ldr	r5, [pc, #136]	; (8000de4 <xTaskPriorityInherit+0x94>)
 8000d5a:	6ac3      	ldr	r3, [r0, #44]	; 0x2c
 8000d5c:	682a      	ldr	r2, [r5, #0]
 8000d5e:	6ad2      	ldr	r2, [r2, #44]	; 0x2c
 8000d60:	4293      	cmp	r3, r2
 8000d62:	d236      	bcs.n	8000dd2 <xTaskPriorityInherit+0x82>
                if( ( listGET_LIST_ITEM_VALUE( &( pxMutexHolderTCB->xEventListItem ) ) & taskEVENT_LIST_ITEM_VALUE_IN_USE ) == 0UL )
 8000d64:	6982      	ldr	r2, [r0, #24]
                if( listIS_CONTAINED_WITHIN( &( pxReadyTasksLists[ pxMutexHolderTCB->uxPriority ] ), &( pxMutexHolderTCB->xStateListItem ) ) != pdFALSE )
 8000d66:	4e20      	ldr	r6, [pc, #128]	; (8000de8 <xTaskPriorityInherit+0x98>)
                if( ( listGET_LIST_ITEM_VALUE( &( pxMutexHolderTCB->xEventListItem ) ) & taskEVENT_LIST_ITEM_VALUE_IN_USE ) == 0UL )
 8000d68:	2a00      	cmp	r2, #0
                    listSET_LIST_ITEM_VALUE( &( pxMutexHolderTCB->xEventListItem ), ( TickType_t ) configMAX_PRIORITIES - ( TickType_t ) pxCurrentTCB->uxPriority ); /*lint !e961 MISRA exception as the casts are only redundant for some ports. */
 8000d6a:	bfa1      	itttt	ge
 8000d6c:	682a      	ldrge	r2, [r5, #0]
 8000d6e:	6ad2      	ldrge	r2, [r2, #44]	; 0x2c
 8000d70:	f1c2 0205 	rsbge	r2, r2, #5
 8000d74:	6182      	strge	r2, [r0, #24]
                if( listIS_CONTAINED_WITHIN( &( pxReadyTasksLists[ pxMutexHolderTCB->uxPriority ] ), &( pxMutexHolderTCB->xStateListItem ) ) != pdFALSE )
 8000d76:	2214      	movs	r2, #20
 8000d78:	fb02 6303 	mla	r3, r2, r3, r6
 8000d7c:	6942      	ldr	r2, [r0, #20]
 8000d7e:	429a      	cmp	r2, r3
 8000d80:	d123      	bne.n	8000dca <xTaskPriorityInherit+0x7a>
                    if( uxListRemove( &( pxMutexHolderTCB->xStateListItem ) ) == ( UBaseType_t ) 0 )
 8000d82:	1d07      	adds	r7, r0, #4
 8000d84:	4638      	mov	r0, r7
 8000d86:	f000 fadf 	bl	8001348 <uxListRemove>
 8000d8a:	4918      	ldr	r1, [pc, #96]	; (8000dec <xTaskPriorityInherit+0x9c>)
 8000d8c:	b930      	cbnz	r0, 8000d9c <xTaskPriorityInherit+0x4c>
                        portRESET_READY_PRIORITY( pxMutexHolderTCB->uxPriority, uxTopReadyPriority );
 8000d8e:	2201      	movs	r2, #1
 8000d90:	6ae0      	ldr	r0, [r4, #44]	; 0x2c
 8000d92:	680b      	ldr	r3, [r1, #0]
 8000d94:	4082      	lsls	r2, r0
 8000d96:	ea23 0302 	bic.w	r3, r3, r2
 8000d9a:	600b      	str	r3, [r1, #0]
                    prvAddTaskToReadyList( pxMutexHolderTCB );
 8000d9c:	2201      	movs	r2, #1
                    pxMutexHolderTCB->uxPriority = pxCurrentTCB->uxPriority;
 8000d9e:	682b      	ldr	r3, [r5, #0]
                    prvAddTaskToReadyList( pxMutexHolderTCB );
 8000da0:	6808      	ldr	r0, [r1, #0]
                    pxMutexHolderTCB->uxPriority = pxCurrentTCB->uxPriority;
 8000da2:	6adb      	ldr	r3, [r3, #44]	; 0x2c
                    prvAddTaskToReadyList( pxMutexHolderTCB );
 8000da4:	409a      	lsls	r2, r3
 8000da6:	4302      	orrs	r2, r0
 8000da8:	600a      	str	r2, [r1, #0]
 8000daa:	2214      	movs	r2, #20
                    pxMutexHolderTCB->uxPriority = pxCurrentTCB->uxPriority;
 8000dac:	62e3      	str	r3, [r4, #44]	; 0x2c
                    prvAddTaskToReadyList( pxMutexHolderTCB );
 8000dae:	4353      	muls	r3, r2
 8000db0:	18f1      	adds	r1, r6, r3
 8000db2:	684a      	ldr	r2, [r1, #4]
 8000db4:	6890      	ldr	r0, [r2, #8]
 8000db6:	60a2      	str	r2, [r4, #8]
 8000db8:	60e0      	str	r0, [r4, #12]
 8000dba:	6047      	str	r7, [r0, #4]
 8000dbc:	6097      	str	r7, [r2, #8]
 8000dbe:	58f2      	ldr	r2, [r6, r3]
 8000dc0:	6161      	str	r1, [r4, #20]
 8000dc2:	3201      	adds	r2, #1
 8000dc4:	50f2      	str	r2, [r6, r3]
                xReturn = pdTRUE;
 8000dc6:	2001      	movs	r0, #1
    }
 8000dc8:	bdf8      	pop	{r3, r4, r5, r6, r7, pc}
                    pxMutexHolderTCB->uxPriority = pxCurrentTCB->uxPriority;
 8000dca:	682b      	ldr	r3, [r5, #0]
 8000dcc:	6adb      	ldr	r3, [r3, #44]	; 0x2c
 8000dce:	62c3      	str	r3, [r0, #44]	; 0x2c
 8000dd0:	e7f9      	b.n	8000dc6 <xTaskPriorityInherit+0x76>
                if( pxMutexHolderTCB->uxBasePriority < pxCurrentTCB->uxPriority )
 8000dd2:	682b      	ldr	r3, [r5, #0]
 8000dd4:	6c40      	ldr	r0, [r0, #68]	; 0x44
 8000dd6:	6adb      	ldr	r3, [r3, #44]	; 0x2c
 8000dd8:	4298      	cmp	r0, r3
 8000dda:	bf2c      	ite	cs
 8000ddc:	2000      	movcs	r0, #0
 8000dde:	2001      	movcc	r0, #1
 8000de0:	e7f2      	b.n	8000dc8 <xTaskPriorityInherit+0x78>
 8000de2:	bf00      	nop
 8000de4:	2000151c 	.word	0x2000151c
 8000de8:	200014b8 	.word	0x200014b8
 8000dec:	20001454 	.word	0x20001454

08000df0 <xTaskPriorityDisinherit>:
    {
 8000df0:	b5f8      	push	{r3, r4, r5, r6, r7, lr}
        if( pxMutexHolder != NULL )
 8000df2:	4604      	mov	r4, r0
 8000df4:	b908      	cbnz	r0, 8000dfa <xTaskPriorityDisinherit+0xa>
        BaseType_t xReturn = pdFALSE;
 8000df6:	2000      	movs	r0, #0
    }
 8000df8:	bdf8      	pop	{r3, r4, r5, r6, r7, pc}
            ( pxTCB->uxMutexesHeld )--;
 8000dfa:	6c83      	ldr	r3, [r0, #72]	; 0x48
            if( pxTCB->uxPriority != pxTCB->uxBasePriority )
 8000dfc:	6ac1      	ldr	r1, [r0, #44]	; 0x2c
 8000dfe:	6c42      	ldr	r2, [r0, #68]	; 0x44
            ( pxTCB->uxMutexesHeld )--;
 8000e00:	3b01      	subs	r3, #1
            if( pxTCB->uxPriority != pxTCB->uxBasePriority )
 8000e02:	4291      	cmp	r1, r2
            ( pxTCB->uxMutexesHeld )--;
 8000e04:	6483      	str	r3, [r0, #72]	; 0x48
            if( pxTCB->uxPriority != pxTCB->uxBasePriority )
 8000e06:	d0f6      	beq.n	8000df6 <xTaskPriorityDisinherit+0x6>
                if( pxTCB->uxMutexesHeld == ( UBaseType_t ) 0 )
 8000e08:	2b00      	cmp	r3, #0
 8000e0a:	d1f4      	bne.n	8000df6 <xTaskPriorityDisinherit+0x6>
                    if( uxListRemove( &( pxTCB->xStateListItem ) ) == ( UBaseType_t ) 0 )
 8000e0c:	1d05      	adds	r5, r0, #4
 8000e0e:	4628      	mov	r0, r5
 8000e10:	f000 fa9a 	bl	8001348 <uxListRemove>
 8000e14:	4a11      	ldr	r2, [pc, #68]	; (8000e5c <xTaskPriorityDisinherit+0x6c>)
 8000e16:	b930      	cbnz	r0, 8000e26 <xTaskPriorityDisinherit+0x36>
                        portRESET_READY_PRIORITY( pxTCB->uxPriority, uxTopReadyPriority );
 8000e18:	2101      	movs	r1, #1
 8000e1a:	6ae0      	ldr	r0, [r4, #44]	; 0x2c
 8000e1c:	6813      	ldr	r3, [r2, #0]
 8000e1e:	4081      	lsls	r1, r0
 8000e20:	ea23 0301 	bic.w	r3, r3, r1
 8000e24:	6013      	str	r3, [r2, #0]
                    prvAddTaskToReadyList( pxTCB );
 8000e26:	2001      	movs	r0, #1
                    pxTCB->uxPriority = pxTCB->uxBasePriority;
 8000e28:	6c63      	ldr	r3, [r4, #68]	; 0x44
                    prvAddTaskToReadyList( pxTCB );
 8000e2a:	6816      	ldr	r6, [r2, #0]
                    listSET_LIST_ITEM_VALUE( &( pxTCB->xEventListItem ), ( TickType_t ) configMAX_PRIORITIES - ( TickType_t ) pxTCB->uxPriority ); /*lint !e961 MISRA exception as the casts are only redundant for some ports. */
 8000e2c:	f1c3 0105 	rsb	r1, r3, #5
 8000e30:	61a1      	str	r1, [r4, #24]
                    prvAddTaskToReadyList( pxTCB );
 8000e32:	fa00 f103 	lsl.w	r1, r0, r3
 8000e36:	4331      	orrs	r1, r6
 8000e38:	6011      	str	r1, [r2, #0]
 8000e3a:	2114      	movs	r1, #20
                    pxTCB->uxPriority = pxTCB->uxBasePriority;
 8000e3c:	62e3      	str	r3, [r4, #44]	; 0x2c
                    prvAddTaskToReadyList( pxTCB );
 8000e3e:	434b      	muls	r3, r1
 8000e40:	4a07      	ldr	r2, [pc, #28]	; (8000e60 <xTaskPriorityDisinherit+0x70>)
 8000e42:	18d6      	adds	r6, r2, r3
 8000e44:	6871      	ldr	r1, [r6, #4]
 8000e46:	688f      	ldr	r7, [r1, #8]
 8000e48:	60a1      	str	r1, [r4, #8]
 8000e4a:	60e7      	str	r7, [r4, #12]
 8000e4c:	607d      	str	r5, [r7, #4]
 8000e4e:	608d      	str	r5, [r1, #8]
 8000e50:	58d1      	ldr	r1, [r2, r3]
 8000e52:	6166      	str	r6, [r4, #20]
 8000e54:	4401      	add	r1, r0
 8000e56:	50d1      	str	r1, [r2, r3]
        return xReturn;
 8000e58:	e7ce      	b.n	8000df8 <xTaskPriorityDisinherit+0x8>
 8000e5a:	bf00      	nop
 8000e5c:	20001454 	.word	0x20001454
 8000e60:	200014b8 	.word	0x200014b8

08000e64 <vTaskPriorityDisinheritAfterTimeout>:
    {
 8000e64:	b570      	push	{r4, r5, r6, lr}
        if( pxMutexHolder != NULL )
 8000e66:	4604      	mov	r4, r0
 8000e68:	2800      	cmp	r0, #0
 8000e6a:	d037      	beq.n	8000edc <vTaskPriorityDisinheritAfterTimeout+0x78>
            if( pxTCB->uxBasePriority < uxHighestPriorityWaitingTask )
 8000e6c:	6c43      	ldr	r3, [r0, #68]	; 0x44
 8000e6e:	4299      	cmp	r1, r3
 8000e70:	bf38      	it	cc
 8000e72:	4619      	movcc	r1, r3
            if( pxTCB->uxPriority != uxPriorityToUse )
 8000e74:	6ac3      	ldr	r3, [r0, #44]	; 0x2c
 8000e76:	428b      	cmp	r3, r1
 8000e78:	d030      	beq.n	8000edc <vTaskPriorityDisinheritAfterTimeout+0x78>
                if( pxTCB->uxMutexesHeld == uxOnlyOneMutexHeld )
 8000e7a:	6c82      	ldr	r2, [r0, #72]	; 0x48
 8000e7c:	2a01      	cmp	r2, #1
 8000e7e:	d12d      	bne.n	8000edc <vTaskPriorityDisinheritAfterTimeout+0x78>
                    if( ( listGET_LIST_ITEM_VALUE( &( pxTCB->xEventListItem ) ) & taskEVENT_LIST_ITEM_VALUE_IN_USE ) == 0UL )
 8000e80:	6982      	ldr	r2, [r0, #24]
                    if( listIS_CONTAINED_WITHIN( &( pxReadyTasksLists[ uxPriorityUsedOnEntry ] ), &( pxTCB->xStateListItem ) ) != pdFALSE )
 8000e82:	4d17      	ldr	r5, [pc, #92]	; (8000ee0 <vTaskPriorityDisinheritAfterTimeout+0x7c>)
                    if( ( listGET_LIST_ITEM_VALUE( &( pxTCB->xEventListItem ) ) & taskEVENT_LIST_ITEM_VALUE_IN_USE ) == 0UL )
 8000e84:	2a00      	cmp	r2, #0
                    if( listIS_CONTAINED_WITHIN( &( pxReadyTasksLists[ uxPriorityUsedOnEntry ] ), &( pxTCB->xStateListItem ) ) != pdFALSE )
 8000e86:	f04f 0214 	mov.w	r2, #20
 8000e8a:	fb02 5303 	mla	r3, r2, r3, r5
 8000e8e:	6942      	ldr	r2, [r0, #20]
                    pxTCB->uxPriority = uxPriorityToUse;
 8000e90:	62c1      	str	r1, [r0, #44]	; 0x2c
                        listSET_LIST_ITEM_VALUE( &( pxTCB->xEventListItem ), ( TickType_t ) configMAX_PRIORITIES - ( TickType_t ) uxPriorityToUse ); /*lint !e961 MISRA exception as the casts are only redundant for some ports. */
 8000e92:	bfa4      	itt	ge
 8000e94:	f1c1 0105 	rsbge	r1, r1, #5
 8000e98:	6181      	strge	r1, [r0, #24]
                    if( listIS_CONTAINED_WITHIN( &( pxReadyTasksLists[ uxPriorityUsedOnEntry ] ), &( pxTCB->xStateListItem ) ) != pdFALSE )
 8000e9a:	429a      	cmp	r2, r3
 8000e9c:	d11e      	bne.n	8000edc <vTaskPriorityDisinheritAfterTimeout+0x78>
                        if( uxListRemove( &( pxTCB->xStateListItem ) ) == ( UBaseType_t ) 0 )
 8000e9e:	1d06      	adds	r6, r0, #4
 8000ea0:	4630      	mov	r0, r6
 8000ea2:	f000 fa51 	bl	8001348 <uxListRemove>
 8000ea6:	6ae3      	ldr	r3, [r4, #44]	; 0x2c
 8000ea8:	490e      	ldr	r1, [pc, #56]	; (8000ee4 <vTaskPriorityDisinheritAfterTimeout+0x80>)
 8000eaa:	b928      	cbnz	r0, 8000eb8 <vTaskPriorityDisinheritAfterTimeout+0x54>
                            portRESET_READY_PRIORITY( pxTCB->uxPriority, uxTopReadyPriority );
 8000eac:	2001      	movs	r0, #1
 8000eae:	680a      	ldr	r2, [r1, #0]
 8000eb0:	4098      	lsls	r0, r3
 8000eb2:	ea22 0200 	bic.w	r2, r2, r0
 8000eb6:	600a      	str	r2, [r1, #0]
                        prvAddTaskToReadyList( pxTCB );
 8000eb8:	2201      	movs	r2, #1
 8000eba:	6808      	ldr	r0, [r1, #0]
 8000ebc:	409a      	lsls	r2, r3
 8000ebe:	4302      	orrs	r2, r0
 8000ec0:	600a      	str	r2, [r1, #0]
 8000ec2:	2214      	movs	r2, #20
 8000ec4:	4353      	muls	r3, r2
 8000ec6:	18e9      	adds	r1, r5, r3
 8000ec8:	684a      	ldr	r2, [r1, #4]
 8000eca:	6890      	ldr	r0, [r2, #8]
 8000ecc:	60a2      	str	r2, [r4, #8]
 8000ece:	60e0      	str	r0, [r4, #12]
 8000ed0:	6046      	str	r6, [r0, #4]
 8000ed2:	6096      	str	r6, [r2, #8]
 8000ed4:	58ea      	ldr	r2, [r5, r3]
 8000ed6:	6161      	str	r1, [r4, #20]
 8000ed8:	3201      	adds	r2, #1
 8000eda:	50ea      	str	r2, [r5, r3]
    }
 8000edc:	bd70      	pop	{r4, r5, r6, pc}
 8000ede:	bf00      	nop
 8000ee0:	200014b8 	.word	0x200014b8
 8000ee4:	20001454 	.word	0x20001454

08000ee8 <pvTaskIncrementMutexHeldCount>:
        if( pxCurrentTCB != NULL )
 8000ee8:	4b04      	ldr	r3, [pc, #16]	; (8000efc <pvTaskIncrementMutexHeldCount+0x14>)
 8000eea:	681a      	ldr	r2, [r3, #0]
 8000eec:	b11a      	cbz	r2, 8000ef6 <pvTaskIncrementMutexHeldCount+0xe>
            ( pxCurrentTCB->uxMutexesHeld )++;
 8000eee:	6819      	ldr	r1, [r3, #0]
 8000ef0:	6c8a      	ldr	r2, [r1, #72]	; 0x48
 8000ef2:	3201      	adds	r2, #1
 8000ef4:	648a      	str	r2, [r1, #72]	; 0x48
        return pxCurrentTCB;
 8000ef6:	6818      	ldr	r0, [r3, #0]
    }
 8000ef8:	4770      	bx	lr
 8000efa:	bf00      	nop
 8000efc:	2000151c 	.word	0x2000151c

08000f00 <prvIsQueueEmpty>:
    taskEXIT_CRITICAL();
}
/*-----------------------------------------------------------*/

static BaseType_t prvIsQueueEmpty( const Queue_t * pxQueue )
{
 8000f00:	b510      	push	{r4, lr}
 8000f02:	4604      	mov	r4, r0
    BaseType_t xReturn;

    taskENTER_CRITICAL();
 8000f04:	f7ff fade 	bl	80004c4 <vPortEnterCritical>
    {
        if( pxQueue->uxMessagesWaiting == ( UBaseType_t ) 0 )
 8000f08:	6ba4      	ldr	r4, [r4, #56]	; 0x38
        else
        {
            xReturn = pdFALSE;
        }
    }
    taskEXIT_CRITICAL();
 8000f0a:	f7ff faeb 	bl	80004e4 <vPortExitCritical>

    return xReturn;
}
 8000f0e:	fab4 f084 	clz	r0, r4
 8000f12:	0940      	lsrs	r0, r0, #5
 8000f14:	bd10      	pop	{r4, pc}

08000f16 <prvCopyDataToQueue>:
{
 8000f16:	b570      	push	{r4, r5, r6, lr}
 8000f18:	4616      	mov	r6, r2
    if( pxQueue->uxItemSize == ( UBaseType_t ) 0 )
 8000f1a:	6c02      	ldr	r2, [r0, #64]	; 0x40
{
 8000f1c:	4604      	mov	r4, r0
    uxMessagesWaiting = pxQueue->uxMessagesWaiting;
 8000f1e:	6b85      	ldr	r5, [r0, #56]	; 0x38
    if( pxQueue->uxItemSize == ( UBaseType_t ) 0 )
 8000f20:	b942      	cbnz	r2, 8000f34 <prvCopyDataToQueue+0x1e>
            if( pxQueue->uxQueueType == queueQUEUE_IS_MUTEX )
 8000f22:	6806      	ldr	r6, [r0, #0]
 8000f24:	b99e      	cbnz	r6, 8000f4e <prvCopyDataToQueue+0x38>
                xReturn = xTaskPriorityDisinherit( pxQueue->u.xSemaphore.xMutexHolder );
 8000f26:	6880      	ldr	r0, [r0, #8]
 8000f28:	f7ff ff62 	bl	8000df0 <xTaskPriorityDisinherit>
                pxQueue->u.xSemaphore.xMutexHolder = NULL;
 8000f2c:	60a6      	str	r6, [r4, #8]
    pxQueue->uxMessagesWaiting = uxMessagesWaiting + ( UBaseType_t ) 1;
 8000f2e:	3501      	adds	r5, #1
 8000f30:	63a5      	str	r5, [r4, #56]	; 0x38
}
 8000f32:	bd70      	pop	{r4, r5, r6, pc}
    else if( xPosition == queueSEND_TO_BACK )
 8000f34:	b96e      	cbnz	r6, 8000f52 <prvCopyDataToQueue+0x3c>
        ( void ) memcpy( ( void * ) pxQueue->pcWriteTo, pvItemToQueue, ( size_t ) pxQueue->uxItemSize ); /*lint !e961 !e418 !e9087 MISRA exception as the casts are only redundant for some ports, plus previous logic ensures a null pointer can only be passed to memcpy() if the copy size is 0.  Cast to void required by function signature and safe as no alignment requirement and copy length specified in bytes. */
 8000f36:	6840      	ldr	r0, [r0, #4]
 8000f38:	f000 fbe8 	bl	800170c <memcpy>
        pxQueue->pcWriteTo += pxQueue->uxItemSize;                                                       /*lint !e9016 Pointer arithmetic on char types ok, especially in this use case where it is the clearest way of conveying intent. */
 8000f3c:	6863      	ldr	r3, [r4, #4]
 8000f3e:	6c22      	ldr	r2, [r4, #64]	; 0x40
 8000f40:	4413      	add	r3, r2
        if( pxQueue->pcWriteTo >= pxQueue->u.xQueue.pcTail )                                             /*lint !e946 MISRA exception justified as comparison of pointers is the cleanest solution. */
 8000f42:	68a2      	ldr	r2, [r4, #8]
        pxQueue->pcWriteTo += pxQueue->uxItemSize;                                                       /*lint !e9016 Pointer arithmetic on char types ok, especially in this use case where it is the clearest way of conveying intent. */
 8000f44:	6063      	str	r3, [r4, #4]
        if( pxQueue->pcWriteTo >= pxQueue->u.xQueue.pcTail )                                             /*lint !e946 MISRA exception justified as comparison of pointers is the cleanest solution. */
 8000f46:	4293      	cmp	r3, r2
            pxQueue->pcWriteTo = pxQueue->pcHead;
 8000f48:	bf24      	itt	cs
 8000f4a:	6823      	ldrcs	r3, [r4, #0]
 8000f4c:	6063      	strcs	r3, [r4, #4]
    BaseType_t xReturn = pdFALSE;
 8000f4e:	2000      	movs	r0, #0
 8000f50:	e7ed      	b.n	8000f2e <prvCopyDataToQueue+0x18>
        ( void ) memcpy( ( void * ) pxQueue->u.xQueue.pcReadFrom, pvItemToQueue, ( size_t ) pxQueue->uxItemSize ); /*lint !e961 !e9087 !e418 MISRA exception as the casts are only redundant for some ports.  Cast to void required by function signature and safe as no alignment requirement and copy length specified in bytes.  Assert checks null pointer only used when length is 0. */
 8000f52:	68c0      	ldr	r0, [r0, #12]
 8000f54:	f000 fbda 	bl	800170c <memcpy>
        pxQueue->u.xQueue.pcReadFrom -= pxQueue->uxItemSize;
 8000f58:	6c22      	ldr	r2, [r4, #64]	; 0x40
 8000f5a:	68e3      	ldr	r3, [r4, #12]
 8000f5c:	4251      	negs	r1, r2
 8000f5e:	1a9b      	subs	r3, r3, r2
        if( pxQueue->u.xQueue.pcReadFrom < pxQueue->pcHead ) /*lint !e946 MISRA exception justified as comparison of pointers is the cleanest solution. */
 8000f60:	6822      	ldr	r2, [r4, #0]
        pxQueue->u.xQueue.pcReadFrom -= pxQueue->uxItemSize;
 8000f62:	60e3      	str	r3, [r4, #12]
        if( pxQueue->u.xQueue.pcReadFrom < pxQueue->pcHead ) /*lint !e946 MISRA exception justified as comparison of pointers is the cleanest solution. */
 8000f64:	4293      	cmp	r3, r2
            pxQueue->u.xQueue.pcReadFrom = ( pxQueue->u.xQueue.pcTail - pxQueue->uxItemSize );
 8000f66:	bf3e      	ittt	cc
 8000f68:	68a3      	ldrcc	r3, [r4, #8]
 8000f6a:	185b      	addcc	r3, r3, r1
 8000f6c:	60e3      	strcc	r3, [r4, #12]
        if( xPosition == queueOVERWRITE )
 8000f6e:	2e02      	cmp	r6, #2
 8000f70:	d1ed      	bne.n	8000f4e <prvCopyDataToQueue+0x38>
            if( uxMessagesWaiting > ( UBaseType_t ) 0 )
 8000f72:	b10d      	cbz	r5, 8000f78 <prvCopyDataToQueue+0x62>
                --uxMessagesWaiting;
 8000f74:	3d01      	subs	r5, #1
 8000f76:	e7ea      	b.n	8000f4e <prvCopyDataToQueue+0x38>
    BaseType_t xReturn = pdFALSE;
 8000f78:	4628      	mov	r0, r5
 8000f7a:	e7d8      	b.n	8000f2e <prvCopyDataToQueue+0x18>

08000f7c <prvUnlockQueue>:
{
 8000f7c:	b570      	push	{r4, r5, r6, lr}
 8000f7e:	4604      	mov	r4, r0
    taskENTER_CRITICAL();
 8000f80:	f7ff faa0 	bl	80004c4 <vPortEnterCritical>
        int8_t cTxLock = pxQueue->cTxLock;
 8000f84:	f894 5045 	ldrb.w	r5, [r4, #69]	; 0x45
                    if( xTaskRemoveFromEventList( &( pxQueue->xTasksWaitingToReceive ) ) != pdFALSE )
 8000f88:	f104 0624 	add.w	r6, r4, #36	; 0x24
        int8_t cTxLock = pxQueue->cTxLock;
 8000f8c:	b26d      	sxtb	r5, r5
        while( cTxLock > queueLOCKED_UNMODIFIED )
 8000f8e:	2d00      	cmp	r5, #0
 8000f90:	dc14      	bgt.n	8000fbc <prvUnlockQueue+0x40>
        pxQueue->cTxLock = queueUNLOCKED;
 8000f92:	23ff      	movs	r3, #255	; 0xff
 8000f94:	f884 3045 	strb.w	r3, [r4, #69]	; 0x45
    taskEXIT_CRITICAL();
 8000f98:	f7ff faa4 	bl	80004e4 <vPortExitCritical>
    taskENTER_CRITICAL();
 8000f9c:	f7ff fa92 	bl	80004c4 <vPortEnterCritical>
        int8_t cRxLock = pxQueue->cRxLock;
 8000fa0:	f894 5044 	ldrb.w	r5, [r4, #68]	; 0x44
                if( xTaskRemoveFromEventList( &( pxQueue->xTasksWaitingToSend ) ) != pdFALSE )
 8000fa4:	f104 0610 	add.w	r6, r4, #16
        int8_t cRxLock = pxQueue->cRxLock;
 8000fa8:	b26d      	sxtb	r5, r5
        while( cRxLock > queueLOCKED_UNMODIFIED )
 8000faa:	2d00      	cmp	r5, #0
 8000fac:	dc12      	bgt.n	8000fd4 <prvUnlockQueue+0x58>
        pxQueue->cRxLock = queueUNLOCKED;
 8000fae:	23ff      	movs	r3, #255	; 0xff
 8000fb0:	f884 3044 	strb.w	r3, [r4, #68]	; 0x44
}
 8000fb4:	e8bd 4070 	ldmia.w	sp!, {r4, r5, r6, lr}
    taskEXIT_CRITICAL();
 8000fb8:	f7ff ba94 	b.w	80004e4 <vPortExitCritical>
                if( listLIST_IS_EMPTY( &( pxQueue->xTasksWaitingToReceive ) ) == pdFALSE )
 8000fbc:	6a63      	ldr	r3, [r4, #36]	; 0x24
 8000fbe:	2b00      	cmp	r3, #0
 8000fc0:	d0e7      	beq.n	8000f92 <prvUnlockQueue+0x16>
                    if( xTaskRemoveFromEventList( &( pxQueue->xTasksWaitingToReceive ) ) != pdFALSE )
 8000fc2:	4630      	mov	r0, r6
 8000fc4:	f7ff fe2e 	bl	8000c24 <xTaskRemoveFromEventList>
 8000fc8:	b108      	cbz	r0, 8000fce <prvUnlockQueue+0x52>
                        vTaskMissedYield();
 8000fca:	f7ff febb 	bl	8000d44 <vTaskMissedYield>
            --cTxLock;
 8000fce:	3d01      	subs	r5, #1
 8000fd0:	b26d      	sxtb	r5, r5
 8000fd2:	e7dc      	b.n	8000f8e <prvUnlockQueue+0x12>
            if( listLIST_IS_EMPTY( &( pxQueue->xTasksWaitingToSend ) ) == pdFALSE )
 8000fd4:	6923      	ldr	r3, [r4, #16]
 8000fd6:	2b00      	cmp	r3, #0
 8000fd8:	d0e9      	beq.n	8000fae <prvUnlockQueue+0x32>
                if( xTaskRemoveFromEventList( &( pxQueue->xTasksWaitingToSend ) ) != pdFALSE )
 8000fda:	4630      	mov	r0, r6
 8000fdc:	f7ff fe22 	bl	8000c24 <xTaskRemoveFromEventList>
 8000fe0:	b108      	cbz	r0, 8000fe6 <prvUnlockQueue+0x6a>
                    vTaskMissedYield();
 8000fe2:	f7ff feaf 	bl	8000d44 <vTaskMissedYield>
                --cRxLock;
 8000fe6:	3d01      	subs	r5, #1
 8000fe8:	b26d      	sxtb	r5, r5
 8000fea:	e7de      	b.n	8000faa <prvUnlockQueue+0x2e>

08000fec <xQueueGenericReset>:
{
 8000fec:	b570      	push	{r4, r5, r6, lr}
 8000fee:	460e      	mov	r6, r1
    if( ( pxQueue != NULL ) &&
 8000ff0:	4604      	mov	r4, r0
 8000ff2:	b310      	cbz	r0, 800103a <xQueueGenericReset+0x4e>
        ( pxQueue->uxLength >= 1U ) &&
 8000ff4:	6bc0      	ldr	r0, [r0, #60]	; 0x3c
    if( ( pxQueue != NULL ) &&
 8000ff6:	b300      	cbz	r0, 800103a <xQueueGenericReset+0x4e>
        ( ( SIZE_MAX / pxQueue->uxLength ) >= pxQueue->uxItemSize ) )
 8000ff8:	6c23      	ldr	r3, [r4, #64]	; 0x40
 8000ffa:	fba3 3500 	umull	r3, r5, r3, r0
 8000ffe:	b9dd      	cbnz	r5, 8001038 <xQueueGenericReset+0x4c>
        taskENTER_CRITICAL();
 8001000:	f7ff fa60 	bl	80004c4 <vPortEnterCritical>
            pxQueue->u.xQueue.pcTail = pxQueue->pcHead + ( pxQueue->uxLength * pxQueue->uxItemSize ); /*lint !e9016 Pointer arithmetic allowed on char types, especially when it assists conveying intent. */
 8001004:	e9d4 310f 	ldrd	r3, r1, [r4, #60]	; 0x3c
 8001008:	434b      	muls	r3, r1
 800100a:	6822      	ldr	r2, [r4, #0]
            pxQueue->uxMessagesWaiting = ( UBaseType_t ) 0U;
 800100c:	63a5      	str	r5, [r4, #56]	; 0x38
            pxQueue->u.xQueue.pcTail = pxQueue->pcHead + ( pxQueue->uxLength * pxQueue->uxItemSize ); /*lint !e9016 Pointer arithmetic allowed on char types, especially when it assists conveying intent. */
 800100e:	18d0      	adds	r0, r2, r3
            pxQueue->u.xQueue.pcReadFrom = pxQueue->pcHead + ( ( pxQueue->uxLength - 1U ) * pxQueue->uxItemSize ); /*lint !e9016 Pointer arithmetic allowed on char types, especially when it assists conveying intent. */
 8001010:	1a5b      	subs	r3, r3, r1
            pxQueue->pcWriteTo = pxQueue->pcHead;
 8001012:	6062      	str	r2, [r4, #4]
            pxQueue->u.xQueue.pcReadFrom = pxQueue->pcHead + ( ( pxQueue->uxLength - 1U ) * pxQueue->uxItemSize ); /*lint !e9016 Pointer arithmetic allowed on char types, especially when it assists conveying intent. */
 8001014:	441a      	add	r2, r3
            pxQueue->cRxLock = queueUNLOCKED;
 8001016:	23ff      	movs	r3, #255	; 0xff
            pxQueue->u.xQueue.pcTail = pxQueue->pcHead + ( pxQueue->uxLength * pxQueue->uxItemSize ); /*lint !e9016 Pointer arithmetic allowed on char types, especially when it assists conveying intent. */
 8001018:	60a0      	str	r0, [r4, #8]
            pxQueue->cRxLock = queueUNLOCKED;
 800101a:	f884 3044 	strb.w	r3, [r4, #68]	; 0x44
            pxQueue->u.xQueue.pcReadFrom = pxQueue->pcHead + ( ( pxQueue->uxLength - 1U ) * pxQueue->uxItemSize ); /*lint !e9016 Pointer arithmetic allowed on char types, especially when it assists conveying intent. */
 800101e:	60e2      	str	r2, [r4, #12]
            pxQueue->cTxLock = queueUNLOCKED;
 8001020:	f884 3045 	strb.w	r3, [r4, #69]	; 0x45
            if( xNewQueue == pdFALSE )
 8001024:	b156      	cbz	r6, 800103c <xQueueGenericReset+0x50>
                vListInitialise( &( pxQueue->xTasksWaitingToSend ) );
 8001026:	f104 0010 	add.w	r0, r4, #16
 800102a:	f000 f968 	bl	80012fe <vListInitialise>
                vListInitialise( &( pxQueue->xTasksWaitingToReceive ) );
 800102e:	f104 0024 	add.w	r0, r4, #36	; 0x24
 8001032:	f000 f964 	bl	80012fe <vListInitialise>
 8001036:	e012      	b.n	800105e <xQueueGenericReset+0x72>
        xReturn = pdFAIL;
 8001038:	2000      	movs	r0, #0
}
 800103a:	bd70      	pop	{r4, r5, r6, pc}
                if( listLIST_IS_EMPTY( &( pxQueue->xTasksWaitingToSend ) ) == pdFALSE )
 800103c:	6923      	ldr	r3, [r4, #16]
 800103e:	b173      	cbz	r3, 800105e <xQueueGenericReset+0x72>
                    if( xTaskRemoveFromEventList( &( pxQueue->xTasksWaitingToSend ) ) != pdFALSE )
 8001040:	f104 0010 	add.w	r0, r4, #16
 8001044:	f7ff fdee 	bl	8000c24 <xTaskRemoveFromEventList>
 8001048:	b148      	cbz	r0, 800105e <xQueueGenericReset+0x72>
                        queueYIELD_IF_USING_PREEMPTION();
 800104a:	f04f 23e0 	mov.w	r3, #3758153728	; 0xe000e000
 800104e:	f04f 5280 	mov.w	r2, #268435456	; 0x10000000
 8001052:	f8c3 2d04 	str.w	r2, [r3, #3332]	; 0xd04
 8001056:	f3bf 8f4f 	dsb	sy
 800105a:	f3bf 8f6f 	isb	sy
        taskEXIT_CRITICAL();
 800105e:	f7ff fa41 	bl	80004e4 <vPortExitCritical>
 8001062:	2001      	movs	r0, #1
 8001064:	e7e9      	b.n	800103a <xQueueGenericReset+0x4e>

08001066 <xQueueGenericCreate>:
    {
 8001066:	b570      	push	{r4, r5, r6, lr}
 8001068:	460d      	mov	r5, r1
        if( ( uxQueueLength > ( UBaseType_t ) 0 ) &&
 800106a:	4606      	mov	r6, r0
 800106c:	b910      	cbnz	r0, 8001074 <xQueueGenericCreate+0xe>
        Queue_t * pxNewQueue = NULL;
 800106e:	2400      	movs	r4, #0
    }
 8001070:	4620      	mov	r0, r4
 8001072:	bd70      	pop	{r4, r5, r6, pc}
            ( ( SIZE_MAX / uxQueueLength ) >= uxItemSize ) &&
 8001074:	fba1 2300 	umull	r2, r3, r1, r0
 8001078:	2b00      	cmp	r3, #0
 800107a:	d1f8      	bne.n	800106e <xQueueGenericCreate+0x8>
            ( ( SIZE_MAX - sizeof( Queue_t ) ) >= ( uxQueueLength * uxItemSize ) ) )
 800107c:	4348      	muls	r0, r1
            ( ( SIZE_MAX / uxQueueLength ) >= uxItemSize ) &&
 800107e:	f110 0f49 	cmn.w	r0, #73	; 0x49
 8001082:	d8f4      	bhi.n	800106e <xQueueGenericCreate+0x8>
            pxNewQueue = ( Queue_t * ) pvPortMalloc( sizeof( Queue_t ) + xQueueSizeInBytes ); /*lint !e9087 !e9079 see comment above. */
 8001084:	3048      	adds	r0, #72	; 0x48
 8001086:	f7ff f947 	bl	8000318 <pvPortMalloc>
            if( pxNewQueue != NULL )
 800108a:	4604      	mov	r4, r0
 800108c:	2800      	cmp	r0, #0
 800108e:	d0ee      	beq.n	800106e <xQueueGenericCreate+0x8>
    if( uxItemSize == ( UBaseType_t ) 0 )
 8001090:	b14d      	cbz	r5, 80010a6 <xQueueGenericCreate+0x40>
                pucQueueStorage += sizeof( Queue_t ); /*lint !e9016 Pointer arithmetic allowed on char types, especially when it assists conveying intent. */
 8001092:	f100 0348 	add.w	r3, r0, #72	; 0x48
    ( void ) xQueueGenericReset( pxNewQueue, pdTRUE );
 8001096:	2101      	movs	r1, #1
 8001098:	4620      	mov	r0, r4
    pxNewQueue->uxItemSize = uxItemSize;
 800109a:	e9c4 650f 	strd	r6, r5, [r4, #60]	; 0x3c
 800109e:	6023      	str	r3, [r4, #0]
    ( void ) xQueueGenericReset( pxNewQueue, pdTRUE );
 80010a0:	f7ff ffa4 	bl	8000fec <xQueueGenericReset>
        return pxNewQueue;
 80010a4:	e7e4      	b.n	8001070 <xQueueGenericCreate+0xa>
        pxNewQueue->pcHead = ( int8_t * ) pxNewQueue;
 80010a6:	4603      	mov	r3, r0
 80010a8:	e7f5      	b.n	8001096 <xQueueGenericCreate+0x30>

080010aa <xQueueGenericSend>:
{
 80010aa:	b5f0      	push	{r4, r5, r6, r7, lr}
 80010ac:	4604      	mov	r4, r0
 80010ae:	b085      	sub	sp, #20
 80010b0:	461d      	mov	r5, r3
 80010b2:	9201      	str	r2, [sp, #4]
 80010b4:	460e      	mov	r6, r1
        taskENTER_CRITICAL();
 80010b6:	f7ff fa05 	bl	80004c4 <vPortEnterCritical>
            if( ( pxQueue->uxMessagesWaiting < pxQueue->uxLength ) || ( xCopyPosition == queueOVERWRITE ) )
 80010ba:	6ba2      	ldr	r2, [r4, #56]	; 0x38
 80010bc:	6be3      	ldr	r3, [r4, #60]	; 0x3c
 80010be:	429a      	cmp	r2, r3
 80010c0:	d21a      	bcs.n	80010f8 <xQueueGenericSend+0x4e>
                    xYieldRequired = prvCopyDataToQueue( pxQueue, pvItemToQueue, xCopyPosition );
 80010c2:	462a      	mov	r2, r5
 80010c4:	4631      	mov	r1, r6
 80010c6:	4620      	mov	r0, r4
 80010c8:	f7ff ff25 	bl	8000f16 <prvCopyDataToQueue>
                    if( listLIST_IS_EMPTY( &( pxQueue->xTasksWaitingToReceive ) ) == pdFALSE )
 80010cc:	6a63      	ldr	r3, [r4, #36]	; 0x24
 80010ce:	b11b      	cbz	r3, 80010d8 <xQueueGenericSend+0x2e>
                        if( xTaskRemoveFromEventList( &( pxQueue->xTasksWaitingToReceive ) ) != pdFALSE )
 80010d0:	f104 0024 	add.w	r0, r4, #36	; 0x24
 80010d4:	f7ff fda6 	bl	8000c24 <xTaskRemoveFromEventList>
                    else if( xYieldRequired != pdFALSE )
 80010d8:	b148      	cbz	r0, 80010ee <xQueueGenericSend+0x44>
                        queueYIELD_IF_USING_PREEMPTION();
 80010da:	f04f 23e0 	mov.w	r3, #3758153728	; 0xe000e000
 80010de:	f04f 5280 	mov.w	r2, #268435456	; 0x10000000
 80010e2:	f8c3 2d04 	str.w	r2, [r3, #3332]	; 0xd04
 80010e6:	f3bf 8f4f 	dsb	sy
 80010ea:	f3bf 8f6f 	isb	sy
                taskEXIT_CRITICAL();
 80010ee:	f7ff f9f9 	bl	80004e4 <vPortExitCritical>
                return pdPASS;
 80010f2:	2001      	movs	r0, #1
}
 80010f4:	b005      	add	sp, #20
 80010f6:	bdf0      	pop	{r4, r5, r6, r7, pc}
            if( ( pxQueue->uxMessagesWaiting < pxQueue->uxLength ) || ( xCopyPosition == queueOVERWRITE ) )
 80010f8:	2d02      	cmp	r5, #2
 80010fa:	d0e2      	beq.n	80010c2 <xQueueGenericSend+0x18>
    BaseType_t xEntryTimeSet = pdFALSE, xYieldRequired;
 80010fc:	2300      	movs	r3, #0
        prvLockQueue( pxQueue );
 80010fe:	461f      	mov	r7, r3
 8001100:	e037      	b.n	8001172 <xQueueGenericSend+0xc8>
                else if( xEntryTimeSet == pdFALSE )
 8001102:	b913      	cbnz	r3, 800110a <xQueueGenericSend+0x60>
                    vTaskInternalSetTimeOutState( &xTimeOut );
 8001104:	a802      	add	r0, sp, #8
 8001106:	f7ff fde9 	bl	8000cdc <vTaskInternalSetTimeOutState>
        taskEXIT_CRITICAL();
 800110a:	f7ff f9eb 	bl	80004e4 <vPortExitCritical>
        vTaskSuspendAll();
 800110e:	f7ff fbd3 	bl	80008b8 <vTaskSuspendAll>
        prvLockQueue( pxQueue );
 8001112:	f7ff f9d7 	bl	80004c4 <vPortEnterCritical>
 8001116:	f894 3044 	ldrb.w	r3, [r4, #68]	; 0x44
 800111a:	2bff      	cmp	r3, #255	; 0xff
 800111c:	bf08      	it	eq
 800111e:	f884 7044 	strbeq.w	r7, [r4, #68]	; 0x44
 8001122:	f894 3045 	ldrb.w	r3, [r4, #69]	; 0x45
 8001126:	2bff      	cmp	r3, #255	; 0xff
 8001128:	bf08      	it	eq
 800112a:	f884 7045 	strbeq.w	r7, [r4, #69]	; 0x45
 800112e:	f7ff f9d9 	bl	80004e4 <vPortExitCritical>
        if( xTaskCheckForTimeOut( &xTimeOut, &xTicksToWait ) == pdFALSE )
 8001132:	a901      	add	r1, sp, #4
 8001134:	a802      	add	r0, sp, #8
 8001136:	f7ff fddd 	bl	8000cf4 <xTaskCheckForTimeOut>
 800113a:	2800      	cmp	r0, #0
 800113c:	d139      	bne.n	80011b2 <xQueueGenericSend+0x108>

static BaseType_t prvIsQueueFull( const Queue_t * pxQueue )
{
    BaseType_t xReturn;

    taskENTER_CRITICAL();
 800113e:	f7ff f9c1 	bl	80004c4 <vPortEnterCritical>
    {
        if( pxQueue->uxMessagesWaiting == pxQueue->uxLength )
 8001142:	6ba2      	ldr	r2, [r4, #56]	; 0x38
 8001144:	6be3      	ldr	r3, [r4, #60]	; 0x3c
 8001146:	429a      	cmp	r2, r3
 8001148:	d11a      	bne.n	8001180 <xQueueGenericSend+0xd6>
        else
        {
            xReturn = pdFALSE;
        }
    }
    taskEXIT_CRITICAL();
 800114a:	f7ff f9cb 	bl	80004e4 <vPortExitCritical>
                vTaskPlaceOnEventList( &( pxQueue->xTasksWaitingToSend ), xTicksToWait );
 800114e:	9901      	ldr	r1, [sp, #4]
 8001150:	f104 0010 	add.w	r0, r4, #16
 8001154:	f7ff fd56 	bl	8000c04 <vTaskPlaceOnEventList>
                prvUnlockQueue( pxQueue );
 8001158:	4620      	mov	r0, r4
 800115a:	f7ff ff0f 	bl	8000f7c <prvUnlockQueue>
                if( xTaskResumeAll() == pdFALSE )
 800115e:	f7ff fc63 	bl	8000a28 <xTaskResumeAll>
 8001162:	b1d8      	cbz	r0, 800119c <xQueueGenericSend+0xf2>
        taskENTER_CRITICAL();
 8001164:	f7ff f9ae 	bl	80004c4 <vPortEnterCritical>
            if( ( pxQueue->uxMessagesWaiting < pxQueue->uxLength ) || ( xCopyPosition == queueOVERWRITE ) )
 8001168:	6ba3      	ldr	r3, [r4, #56]	; 0x38
 800116a:	6be2      	ldr	r2, [r4, #60]	; 0x3c
 800116c:	429a      	cmp	r2, r3
 800116e:	d8a8      	bhi.n	80010c2 <xQueueGenericSend+0x18>
{
 8001170:	2301      	movs	r3, #1
                if( xTicksToWait == ( TickType_t ) 0 )
 8001172:	9a01      	ldr	r2, [sp, #4]
 8001174:	2a00      	cmp	r2, #0
 8001176:	d1c4      	bne.n	8001102 <xQueueGenericSend+0x58>
                    taskEXIT_CRITICAL();
 8001178:	f7ff f9b4 	bl	80004e4 <vPortExitCritical>
                    return errQUEUE_FULL;
 800117c:	2000      	movs	r0, #0
 800117e:	e7b9      	b.n	80010f4 <xQueueGenericSend+0x4a>
    taskEXIT_CRITICAL();
 8001180:	f7ff f9b0 	bl	80004e4 <vPortExitCritical>
                prvUnlockQueue( pxQueue );
 8001184:	4620      	mov	r0, r4
 8001186:	f7ff fef9 	bl	8000f7c <prvUnlockQueue>
                ( void ) xTaskResumeAll();
 800118a:	f7ff fc4d 	bl	8000a28 <xTaskResumeAll>
        taskENTER_CRITICAL();
 800118e:	f7ff f999 	bl	80004c4 <vPortEnterCritical>
            if( ( pxQueue->uxMessagesWaiting < pxQueue->uxLength ) || ( xCopyPosition == queueOVERWRITE ) )
 8001192:	6ba2      	ldr	r2, [r4, #56]	; 0x38
 8001194:	6be3      	ldr	r3, [r4, #60]	; 0x3c
 8001196:	429a      	cmp	r2, r3
 8001198:	d2ea      	bcs.n	8001170 <xQueueGenericSend+0xc6>
 800119a:	e792      	b.n	80010c2 <xQueueGenericSend+0x18>
                    portYIELD_WITHIN_API();
 800119c:	f04f 23e0 	mov.w	r3, #3758153728	; 0xe000e000
 80011a0:	f04f 5280 	mov.w	r2, #268435456	; 0x10000000
 80011a4:	f8c3 2d04 	str.w	r2, [r3, #3332]	; 0xd04
 80011a8:	f3bf 8f4f 	dsb	sy
 80011ac:	f3bf 8f6f 	isb	sy
 80011b0:	e7ed      	b.n	800118e <xQueueGenericSend+0xe4>
            prvUnlockQueue( pxQueue );
 80011b2:	4620      	mov	r0, r4
 80011b4:	f7ff fee2 	bl	8000f7c <prvUnlockQueue>
            ( void ) xTaskResumeAll();
 80011b8:	f7ff fc36 	bl	8000a28 <xTaskResumeAll>
            return errQUEUE_FULL;
 80011bc:	e7de      	b.n	800117c <xQueueGenericSend+0xd2>

080011be <xQueueCreateMutex>:
    {
 80011be:	4602      	mov	r2, r0
 80011c0:	b510      	push	{r4, lr}
        xNewQueue = xQueueGenericCreate( uxMutexLength, uxMutexSize, ucQueueType );
 80011c2:	2100      	movs	r1, #0
 80011c4:	2001      	movs	r0, #1
 80011c6:	f7ff ff4e 	bl	8001066 <xQueueGenericCreate>
        if( pxNewQueue != NULL )
 80011ca:	4604      	mov	r4, r0
 80011cc:	b138      	cbz	r0, 80011de <xQueueCreateMutex+0x20>
            pxNewQueue->u.xSemaphore.xMutexHolder = NULL;
 80011ce:	2300      	movs	r3, #0
            ( void ) xQueueGenericSend( pxNewQueue, NULL, ( TickType_t ) 0U, queueSEND_TO_BACK );
 80011d0:	461a      	mov	r2, r3
 80011d2:	4619      	mov	r1, r3
            pxNewQueue->u.xSemaphore.xMutexHolder = NULL;
 80011d4:	6083      	str	r3, [r0, #8]
            pxNewQueue->uxQueueType = queueQUEUE_IS_MUTEX;
 80011d6:	6003      	str	r3, [r0, #0]
            pxNewQueue->u.xSemaphore.uxRecursiveCallCount = 0;
 80011d8:	60c3      	str	r3, [r0, #12]
            ( void ) xQueueGenericSend( pxNewQueue, NULL, ( TickType_t ) 0U, queueSEND_TO_BACK );
 80011da:	f7ff ff66 	bl	80010aa <xQueueGenericSend>
    }
 80011de:	4620      	mov	r0, r4
 80011e0:	bd10      	pop	{r4, pc}

080011e2 <xQueueSemaphoreTake>:
{
 80011e2:	b5f0      	push	{r4, r5, r6, r7, lr}
        BaseType_t xInheritanceOccurred = pdFALSE;
 80011e4:	2500      	movs	r5, #0
{
 80011e6:	4604      	mov	r4, r0
    BaseType_t xEntryTimeSet = pdFALSE;
 80011e8:	462f      	mov	r7, r5
        prvLockQueue( pxQueue );
 80011ea:	462e      	mov	r6, r5
{
 80011ec:	b085      	sub	sp, #20
 80011ee:	9101      	str	r1, [sp, #4]
        taskENTER_CRITICAL();
 80011f0:	f7ff f968 	bl	80004c4 <vPortEnterCritical>
            const UBaseType_t uxSemaphoreCount = pxQueue->uxMessagesWaiting;
 80011f4:	6ba3      	ldr	r3, [r4, #56]	; 0x38
            if( uxSemaphoreCount > ( UBaseType_t ) 0 )
 80011f6:	b1e3      	cbz	r3, 8001232 <xQueueSemaphoreTake+0x50>
                pxQueue->uxMessagesWaiting = uxSemaphoreCount - ( UBaseType_t ) 1;
 80011f8:	3b01      	subs	r3, #1
 80011fa:	63a3      	str	r3, [r4, #56]	; 0x38
                    if( pxQueue->uxQueueType == queueQUEUE_IS_MUTEX )
 80011fc:	6823      	ldr	r3, [r4, #0]
 80011fe:	b913      	cbnz	r3, 8001206 <xQueueSemaphoreTake+0x24>
                        pxQueue->u.xSemaphore.xMutexHolder = pvTaskIncrementMutexHeldCount();
 8001200:	f7ff fe72 	bl	8000ee8 <pvTaskIncrementMutexHeldCount>
 8001204:	60a0      	str	r0, [r4, #8]
                if( listLIST_IS_EMPTY( &( pxQueue->xTasksWaitingToSend ) ) == pdFALSE )
 8001206:	6923      	ldr	r3, [r4, #16]
 8001208:	b173      	cbz	r3, 8001228 <xQueueSemaphoreTake+0x46>
                    if( xTaskRemoveFromEventList( &( pxQueue->xTasksWaitingToSend ) ) != pdFALSE )
 800120a:	f104 0010 	add.w	r0, r4, #16
 800120e:	f7ff fd09 	bl	8000c24 <xTaskRemoveFromEventList>
 8001212:	b148      	cbz	r0, 8001228 <xQueueSemaphoreTake+0x46>
                        queueYIELD_IF_USING_PREEMPTION();
 8001214:	f04f 23e0 	mov.w	r3, #3758153728	; 0xe000e000
 8001218:	f04f 5280 	mov.w	r2, #268435456	; 0x10000000
 800121c:	f8c3 2d04 	str.w	r2, [r3, #3332]	; 0xd04
 8001220:	f3bf 8f4f 	dsb	sy
 8001224:	f3bf 8f6f 	isb	sy
                taskEXIT_CRITICAL();
 8001228:	f7ff f95c 	bl	80004e4 <vPortExitCritical>
                return pdPASS;
 800122c:	2001      	movs	r0, #1
}
 800122e:	b005      	add	sp, #20
 8001230:	bdf0      	pop	{r4, r5, r6, r7, pc}
                if( xTicksToWait == ( TickType_t ) 0 )
 8001232:	9b01      	ldr	r3, [sp, #4]
 8001234:	b91b      	cbnz	r3, 800123e <xQueueSemaphoreTake+0x5c>
                        taskEXIT_CRITICAL();
 8001236:	f7ff f955 	bl	80004e4 <vPortExitCritical>
                    return errQUEUE_EMPTY;
 800123a:	2000      	movs	r0, #0
 800123c:	e7f7      	b.n	800122e <xQueueSemaphoreTake+0x4c>
                else if( xEntryTimeSet == pdFALSE )
 800123e:	b917      	cbnz	r7, 8001246 <xQueueSemaphoreTake+0x64>
                    vTaskInternalSetTimeOutState( &xTimeOut );
 8001240:	a802      	add	r0, sp, #8
 8001242:	f7ff fd4b 	bl	8000cdc <vTaskInternalSetTimeOutState>
        taskEXIT_CRITICAL();
 8001246:	f7ff f94d 	bl	80004e4 <vPortExitCritical>
        vTaskSuspendAll();
 800124a:	f7ff fb35 	bl	80008b8 <vTaskSuspendAll>
        prvLockQueue( pxQueue );
 800124e:	f7ff f939 	bl	80004c4 <vPortEnterCritical>
 8001252:	f894 3044 	ldrb.w	r3, [r4, #68]	; 0x44
 8001256:	2bff      	cmp	r3, #255	; 0xff
 8001258:	bf08      	it	eq
 800125a:	f884 6044 	strbeq.w	r6, [r4, #68]	; 0x44
 800125e:	f894 3045 	ldrb.w	r3, [r4, #69]	; 0x45
 8001262:	2bff      	cmp	r3, #255	; 0xff
 8001264:	bf08      	it	eq
 8001266:	f884 6045 	strbeq.w	r6, [r4, #69]	; 0x45
 800126a:	f7ff f93b 	bl	80004e4 <vPortExitCritical>
        if( xTaskCheckForTimeOut( &xTimeOut, &xTicksToWait ) == pdFALSE )
 800126e:	a901      	add	r1, sp, #4
 8001270:	a802      	add	r0, sp, #8
 8001272:	f7ff fd3f 	bl	8000cf4 <xTaskCheckForTimeOut>
 8001276:	bb50      	cbnz	r0, 80012ce <xQueueSemaphoreTake+0xec>
            if( prvIsQueueEmpty( pxQueue ) != pdFALSE )
 8001278:	4620      	mov	r0, r4
 800127a:	f7ff fe41 	bl	8000f00 <prvIsQueueEmpty>
 800127e:	b300      	cbz	r0, 80012c2 <xQueueSemaphoreTake+0xe0>
                    if( pxQueue->uxQueueType == queueQUEUE_IS_MUTEX )
 8001280:	6823      	ldr	r3, [r4, #0]
 8001282:	b93b      	cbnz	r3, 8001294 <xQueueSemaphoreTake+0xb2>
                        taskENTER_CRITICAL();
 8001284:	f7ff f91e 	bl	80004c4 <vPortEnterCritical>
                            xInheritanceOccurred = xTaskPriorityInherit( pxQueue->u.xSemaphore.xMutexHolder );
 8001288:	68a0      	ldr	r0, [r4, #8]
 800128a:	f7ff fd61 	bl	8000d50 <xTaskPriorityInherit>
 800128e:	4605      	mov	r5, r0
                        taskEXIT_CRITICAL();
 8001290:	f7ff f928 	bl	80004e4 <vPortExitCritical>
                vTaskPlaceOnEventList( &( pxQueue->xTasksWaitingToReceive ), xTicksToWait );
 8001294:	9901      	ldr	r1, [sp, #4]
 8001296:	f104 0024 	add.w	r0, r4, #36	; 0x24
 800129a:	f7ff fcb3 	bl	8000c04 <vTaskPlaceOnEventList>
                prvUnlockQueue( pxQueue );
 800129e:	4620      	mov	r0, r4
 80012a0:	f7ff fe6c 	bl	8000f7c <prvUnlockQueue>
                if( xTaskResumeAll() == pdFALSE )
 80012a4:	f7ff fbc0 	bl	8000a28 <xTaskResumeAll>
 80012a8:	b948      	cbnz	r0, 80012be <xQueueSemaphoreTake+0xdc>
                    portYIELD_WITHIN_API();
 80012aa:	f04f 23e0 	mov.w	r3, #3758153728	; 0xe000e000
 80012ae:	f04f 5280 	mov.w	r2, #268435456	; 0x10000000
 80012b2:	f8c3 2d04 	str.w	r2, [r3, #3332]	; 0xd04
 80012b6:	f3bf 8f4f 	dsb	sy
 80012ba:	f3bf 8f6f 	isb	sy
{
 80012be:	2701      	movs	r7, #1
 80012c0:	e796      	b.n	80011f0 <xQueueSemaphoreTake+0xe>
                prvUnlockQueue( pxQueue );
 80012c2:	4620      	mov	r0, r4
 80012c4:	f7ff fe5a 	bl	8000f7c <prvUnlockQueue>
                ( void ) xTaskResumeAll();
 80012c8:	f7ff fbae 	bl	8000a28 <xTaskResumeAll>
 80012cc:	e7f7      	b.n	80012be <xQueueSemaphoreTake+0xdc>
            prvUnlockQueue( pxQueue );
 80012ce:	4620      	mov	r0, r4
 80012d0:	f7ff fe54 	bl	8000f7c <prvUnlockQueue>
            ( void ) xTaskResumeAll();
 80012d4:	f7ff fba8 	bl	8000a28 <xTaskResumeAll>
            if( prvIsQueueEmpty( pxQueue ) != pdFALSE )
 80012d8:	4620      	mov	r0, r4
 80012da:	f7ff fe11 	bl	8000f00 <prvIsQueueEmpty>
 80012de:	2800      	cmp	r0, #0
 80012e0:	d0ed      	beq.n	80012be <xQueueSemaphoreTake+0xdc>
                    if( xInheritanceOccurred != pdFALSE )
 80012e2:	2d00      	cmp	r5, #0
 80012e4:	d0a9      	beq.n	800123a <xQueueSemaphoreTake+0x58>
                        taskENTER_CRITICAL();
 80012e6:	f7ff f8ed 	bl	80004c4 <vPortEnterCritical>
        if( listCURRENT_LIST_LENGTH( &( pxQueue->xTasksWaitingToReceive ) ) > 0U )
 80012ea:	6a61      	ldr	r1, [r4, #36]	; 0x24
 80012ec:	b119      	cbz	r1, 80012f6 <xQueueSemaphoreTake+0x114>
            uxHighestPriorityOfWaitingTasks = ( UBaseType_t ) configMAX_PRIORITIES - ( UBaseType_t ) listGET_ITEM_VALUE_OF_HEAD_ENTRY( &( pxQueue->xTasksWaitingToReceive ) );
 80012ee:	6b23      	ldr	r3, [r4, #48]	; 0x30
 80012f0:	6819      	ldr	r1, [r3, #0]
 80012f2:	f1c1 0105 	rsb	r1, r1, #5
                            vTaskPriorityDisinheritAfterTimeout( pxQueue->u.xSemaphore.xMutexHolder, uxHighestWaitingPriority );
 80012f6:	68a0      	ldr	r0, [r4, #8]
 80012f8:	f7ff fdb4 	bl	8000e64 <vTaskPriorityDisinheritAfterTimeout>
 80012fc:	e79b      	b.n	8001236 <xQueueSemaphoreTake+0x54>

080012fe <vListInitialise>:

    listSET_FIRST_LIST_ITEM_INTEGRITY_CHECK_VALUE( &( pxList->xListEnd ) );

    /* The list end value is the highest possible value in the list to
     * ensure it remains at the end of the list. */
    pxList->xListEnd.xItemValue = portMAX_DELAY;
 80012fe:	f04f 32ff 	mov.w	r2, #4294967295	; 0xffffffff
    pxList->pxIndex = ( ListItem_t * ) &( pxList->xListEnd ); /*lint !e826 !e740 !e9087 The mini list structure is used as the list end to save RAM.  This is checked and valid. */
 8001302:	f100 0308 	add.w	r3, r0, #8

    /* The list end next and previous pointers point to itself so we know
     * when the list is empty. */
    pxList->xListEnd.pxNext = ( ListItem_t * ) &( pxList->xListEnd );     /*lint !e826 !e740 !e9087 The mini list structure is used as the list end to save RAM.  This is checked and valid. */
 8001306:	e9c0 2302 	strd	r2, r3, [r0, #8]
    pxList->pxIndex = ( ListItem_t * ) &( pxList->xListEnd ); /*lint !e826 !e740 !e9087 The mini list structure is used as the list end to save RAM.  This is checked and valid. */
 800130a:	6043      	str	r3, [r0, #4]
    pxList->xListEnd.pxPrevious = ( ListItem_t * ) &( pxList->xListEnd ); /*lint !e826 !e740 !e9087 The mini list structure is used as the list end to save RAM.  This is checked and valid. */
 800130c:	6103      	str	r3, [r0, #16]
        pxList->xListEnd.pxContainer = NULL;
        listSET_SECOND_LIST_ITEM_INTEGRITY_CHECK_VALUE( &( pxList->xListEnd ) );
    }
    #endif

    pxList->uxNumberOfItems = ( UBaseType_t ) 0U;
 800130e:	2300      	movs	r3, #0
 8001310:	6003      	str	r3, [r0, #0]

    /* Write known values into the list if
     * configUSE_LIST_DATA_INTEGRITY_CHECK_BYTES is set to 1. */
    listSET_LIST_INTEGRITY_CHECK_1_VALUE( pxList );
    listSET_LIST_INTEGRITY_CHECK_2_VALUE( pxList );
}
 8001312:	4770      	bx	lr

08001314 <vListInitialiseItem>:
/*-----------------------------------------------------------*/

void vListInitialiseItem( ListItem_t * const pxItem )
{
    /* Make sure the list item is not recorded as being on a list. */
    pxItem->pxContainer = NULL;
 8001314:	2300      	movs	r3, #0
 8001316:	6103      	str	r3, [r0, #16]

    /* Write known values into the list item if
     * configUSE_LIST_DATA_INTEGRITY_CHECK_BYTES is set to 1. */
    listSET_FIRST_LIST_ITEM_INTEGRITY_CHECK_VALUE( pxItem );
    listSET_SECOND_LIST_ITEM_INTEGRITY_CHECK_VALUE( pxItem );
}
 8001318:	4770      	bx	lr

0800131a <vListInsert>:
}
/*-----------------------------------------------------------*/

void vListInsert( List_t * const pxList,
                  ListItem_t * const pxNewListItem )
{
 800131a:	b530      	push	{r4, r5, lr}
    ListItem_t * pxIterator;
    const TickType_t xValueOfInsertion = pxNewListItem->xItemValue;
 800131c:	680c      	ldr	r4, [r1, #0]
     * new list item should be placed after it.  This ensures that TCBs which are
     * stored in ready lists (all of which have the same xItemValue value) get a
     * share of the CPU.  However, if the xItemValue is the same as the back marker
     * the iteration loop below will not end.  Therefore the value is checked
     * first, and the algorithm slightly modified if necessary. */
    if( xValueOfInsertion == portMAX_DELAY )
 800131e:	1c63      	adds	r3, r4, #1
 8001320:	d10a      	bne.n	8001338 <vListInsert+0x1e>
    {
        pxIterator = pxList->xListEnd.pxPrevious;
 8001322:	6903      	ldr	r3, [r0, #16]
            /* There is nothing to do here, just iterating to the wanted
             * insertion position. */
        }
    }

    pxNewListItem->pxNext = pxIterator->pxNext;
 8001324:	685a      	ldr	r2, [r3, #4]
 8001326:	604a      	str	r2, [r1, #4]
    pxNewListItem->pxNext->pxPrevious = pxNewListItem;
 8001328:	6091      	str	r1, [r2, #8]
    pxNewListItem->pxPrevious = pxIterator;
 800132a:	608b      	str	r3, [r1, #8]
    pxIterator->pxNext = pxNewListItem;
 800132c:	6059      	str	r1, [r3, #4]

    /* Remember which list the item is in.  This allows fast removal of the
     * item later. */
    pxNewListItem->pxContainer = pxList;

    ( pxList->uxNumberOfItems )++;
 800132e:	6803      	ldr	r3, [r0, #0]
    pxNewListItem->pxContainer = pxList;
 8001330:	6108      	str	r0, [r1, #16]
    ( pxList->uxNumberOfItems )++;
 8001332:	3301      	adds	r3, #1
 8001334:	6003      	str	r3, [r0, #0]
}
 8001336:	bd30      	pop	{r4, r5, pc}
        for( pxIterator = ( ListItem_t * ) &( pxList->xListEnd ); pxIterator->pxNext->xItemValue <= xValueOfInsertion; pxIterator = pxIterator->pxNext ) /*lint !e826 !e740 !e9087 The mini list structure is used as the list end to save RAM.  This is checked and valid. *//*lint !e440 The iterator moves to a different value, not xValueOfInsertion. */
 8001338:	f100 0208 	add.w	r2, r0, #8
 800133c:	4613      	mov	r3, r2
 800133e:	6852      	ldr	r2, [r2, #4]
 8001340:	6815      	ldr	r5, [r2, #0]
 8001342:	42a5      	cmp	r5, r4
 8001344:	d9fa      	bls.n	800133c <vListInsert+0x22>
 8001346:	e7ed      	b.n	8001324 <vListInsert+0xa>

08001348 <uxListRemove>:

UBaseType_t uxListRemove( ListItem_t * const pxItemToRemove )
{
/* The list item knows which list it is in.  Obtain the list from the list
 * item. */
    List_t * const pxList = pxItemToRemove->pxContainer;
 8001348:	6903      	ldr	r3, [r0, #16]

    pxItemToRemove->pxNext->pxPrevious = pxItemToRemove->pxPrevious;
 800134a:	e9d0 1201 	ldrd	r1, r2, [r0, #4]
 800134e:	608a      	str	r2, [r1, #8]
    pxItemToRemove->pxPrevious->pxNext = pxItemToRemove->pxNext;
 8001350:	6051      	str	r1, [r2, #4]

    /* Only used during decision coverage testing. */
    mtCOVERAGE_TEST_DELAY();

    /* Make sure the index is left pointing to a valid item. */
    if( pxList->pxIndex == pxItemToRemove )
 8001352:	6859      	ldr	r1, [r3, #4]
 8001354:	4281      	cmp	r1, r0
    {
        pxList->pxIndex = pxItemToRemove->pxPrevious;
 8001356:	bf08      	it	eq
 8001358:	605a      	streq	r2, [r3, #4]
    else
    {
        mtCOVERAGE_TEST_MARKER();
    }

    pxItemToRemove->pxContainer = NULL;
 800135a:	2200      	movs	r2, #0
 800135c:	6102      	str	r2, [r0, #16]
    ( pxList->uxNumberOfItems )--;
 800135e:	681a      	ldr	r2, [r3, #0]
 8001360:	3a01      	subs	r2, #1
 8001362:	601a      	str	r2, [r3, #0]

    return pxList->uxNumberOfItems;
 8001364:	6818      	ldr	r0, [r3, #0]
}
 8001366:	4770      	bx	lr

08001368 <gpio_set_mode>:
	     If multiple pins are to be set, use bitwise OR '|' to separate
	     them.
*/

void gpio_set_mode(uint32_t gpioport, uint8_t mode, uint8_t cnf, uint16_t gpios)
{
 8001368:	e92d 41f0 	stmdb	sp!, {r4, r5, r6, r7, r8, lr}

		/* Use tmp32 to either modify crl or crh. */
		tmp32 = (i < 8) ? crl : crh;

		/* Modify bits are needed. */
		tmp32 &= ~(0xf << offset);	/* Clear the bits first. */
 800136c:	f04f 0c0f 	mov.w	ip, #15
	crh = GPIO_CRH(gpioport);
 8001370:	2500      	movs	r5, #0
	crl = GPIO_CRL(gpioport);
 8001372:	6807      	ldr	r7, [r0, #0]
	crh = GPIO_CRH(gpioport);
 8001374:	6846      	ldr	r6, [r0, #4]
		if (!((1 << i) & gpios)) {
 8001376:	fa43 f405 	asr.w	r4, r3, r5
 800137a:	07e4      	lsls	r4, r4, #31
 800137c:	d51c      	bpl.n	80013b8 <gpio_set_mode+0x50>
		offset = (i < 8) ? (i * 4) : ((i - 8) * 4);
 800137e:	2d07      	cmp	r5, #7
 8001380:	bf94      	ite	ls
 8001382:	46be      	movls	lr, r7
 8001384:	46b6      	movhi	lr, r6
 8001386:	b2ac      	uxth	r4, r5
 8001388:	ea4f 0484 	mov.w	r4, r4, lsl #2
 800138c:	bf8a      	itet	hi
 800138e:	3c20      	subhi	r4, #32
 8001390:	b2a4      	uxthls	r4, r4
		tmp32 = (i < 8) ? crl : crh;
 8001392:	b2a4      	uxthhi	r4, r4
		tmp32 &= ~(0xf << offset);	/* Clear the bits first. */
 8001394:	fa0c f804 	lsl.w	r8, ip, r4
 8001398:	ea2e 0808 	bic.w	r8, lr, r8
		tmp32 |= (mode << offset) | (cnf << (offset + 2));
 800139c:	f104 0e02 	add.w	lr, r4, #2
 80013a0:	fa02 fe0e 	lsl.w	lr, r2, lr
 80013a4:	fa01 f404 	lsl.w	r4, r1, r4
 80013a8:	ea4e 0404 	orr.w	r4, lr, r4
 80013ac:	ea44 0408 	orr.w	r4, r4, r8

		/* Write tmp32 into crl or crh, leave the other unchanged. */
		crl = (i < 8) ? tmp32 : crl;
		crh = (i >= 8) ? tmp32 : crh;
 80013b0:	2d08      	cmp	r5, #8
 80013b2:	bf2c      	ite	cs
 80013b4:	4626      	movcs	r6, r4
 80013b6:	4627      	movcc	r7, r4
	for (i = 0; i < 16; i++) {
 80013b8:	3501      	adds	r5, #1
 80013ba:	2d10      	cmp	r5, #16
 80013bc:	d1db      	bne.n	8001376 <gpio_set_mode+0xe>
	}

	GPIO_CRL(gpioport) = crl;
 80013be:	6007      	str	r7, [r0, #0]
	GPIO_CRH(gpioport) = crh;
 80013c0:	6046      	str	r6, [r0, #4]
}
 80013c2:	e8bd 81f0 	ldmia.w	sp!, {r4, r5, r6, r7, r8, pc}
	...

080013c8 <rcc_is_osc_ready>:
	return ((RCC_CIR & RCC_CIR_CSSF) != 0);
}

bool rcc_is_osc_ready(enum rcc_osc osc)
{
	switch (osc) {
 80013c8:	2806      	cmp	r0, #6
 80013ca:	d824      	bhi.n	8001416 <rcc_is_osc_ready+0x4e>
 80013cc:	e8df f000 	tbb	[pc, r0]
 80013d0:	130e0904 	.word	0x130e0904
 80013d4:	1d18      	.short	0x1d18
 80013d6:	20          	.byte	0x20
 80013d7:	00          	.byte	0x00
	case RCC_PLL:
		return RCC_CR & RCC_CR_PLLRDY;
 80013d8:	4b10      	ldr	r3, [pc, #64]	; (800141c <rcc_is_osc_ready+0x54>)
 80013da:	6818      	ldr	r0, [r3, #0]
 80013dc:	f3c0 6040 	ubfx	r0, r0, #25, #1
 80013e0:	4770      	bx	lr
	case RCC_PLL2:
		return RCC_CR & RCC_CR_PLL2RDY;
 80013e2:	4b0e      	ldr	r3, [pc, #56]	; (800141c <rcc_is_osc_ready+0x54>)
 80013e4:	6818      	ldr	r0, [r3, #0]
 80013e6:	f3c0 60c0 	ubfx	r0, r0, #27, #1
 80013ea:	4770      	bx	lr
	case RCC_PLL3:
		return RCC_CR & RCC_CR_PLL3RDY;
 80013ec:	4b0b      	ldr	r3, [pc, #44]	; (800141c <rcc_is_osc_ready+0x54>)
 80013ee:	6818      	ldr	r0, [r3, #0]
 80013f0:	f3c0 7040 	ubfx	r0, r0, #29, #1
 80013f4:	4770      	bx	lr
	case RCC_HSE:
		return RCC_CR & RCC_CR_HSERDY;
 80013f6:	4b09      	ldr	r3, [pc, #36]	; (800141c <rcc_is_osc_ready+0x54>)
 80013f8:	6818      	ldr	r0, [r3, #0]
 80013fa:	f3c0 4040 	ubfx	r0, r0, #17, #1
 80013fe:	4770      	bx	lr
	case RCC_HSI:
		return RCC_CR & RCC_CR_HSIRDY;
 8001400:	4b06      	ldr	r3, [pc, #24]	; (800141c <rcc_is_osc_ready+0x54>)
 8001402:	6818      	ldr	r0, [r3, #0]
	case RCC_LSE:
		return RCC_BDCR & RCC_BDCR_LSERDY;
 8001404:	f3c0 0040 	ubfx	r0, r0, #1, #1
 8001408:	4770      	bx	lr
 800140a:	4b04      	ldr	r3, [pc, #16]	; (800141c <rcc_is_osc_ready+0x54>)
 800140c:	6a18      	ldr	r0, [r3, #32]
 800140e:	e7f9      	b.n	8001404 <rcc_is_osc_ready+0x3c>
	case RCC_LSI:
		return RCC_CSR & RCC_CSR_LSIRDY;
 8001410:	4b02      	ldr	r3, [pc, #8]	; (800141c <rcc_is_osc_ready+0x54>)
 8001412:	6a58      	ldr	r0, [r3, #36]	; 0x24
 8001414:	e7f6      	b.n	8001404 <rcc_is_osc_ready+0x3c>
	switch (osc) {
 8001416:	2000      	movs	r0, #0
	}
	return false;
}
 8001418:	4770      	bx	lr
 800141a:	bf00      	nop
 800141c:	40021000 	.word	0x40021000

08001420 <rcc_wait_for_osc_ready>:

void rcc_wait_for_osc_ready(enum rcc_osc osc)
{
 8001420:	4602      	mov	r2, r0
 8001422:	b508      	push	{r3, lr}
	while (!rcc_is_osc_ready(osc));
 8001424:	4610      	mov	r0, r2
 8001426:	f7ff ffcf 	bl	80013c8 <rcc_is_osc_ready>
 800142a:	2800      	cmp	r0, #0
 800142c:	d0fa      	beq.n	8001424 <rcc_wait_for_osc_ready+0x4>
}
 800142e:	bd08      	pop	{r3, pc}

08001430 <rcc_osc_on>:
@param[in] osc Oscillator ID
*/

void rcc_osc_on(enum rcc_osc osc)
{
	switch (osc) {
 8001430:	2806      	cmp	r0, #6
 8001432:	d82a      	bhi.n	800148a <rcc_osc_on+0x5a>
 8001434:	e8df f000 	tbb	[pc, r0]
 8001438:	140f0a04 	.word	0x140f0a04
 800143c:	1e19      	.short	0x1e19
 800143e:	24          	.byte	0x24
 800143f:	00          	.byte	0x00
	case RCC_PLL:
		RCC_CR |= RCC_CR_PLLON;
 8001440:	4a12      	ldr	r2, [pc, #72]	; (800148c <rcc_osc_on+0x5c>)
 8001442:	6813      	ldr	r3, [r2, #0]
 8001444:	f043 7380 	orr.w	r3, r3, #16777216	; 0x1000000
		break;
	case RCC_PLL2:
		RCC_CR |= RCC_CR_PLL2ON;
 8001448:	6013      	str	r3, [r2, #0]
		break;
 800144a:	4770      	bx	lr
		RCC_CR |= RCC_CR_PLL2ON;
 800144c:	4a0f      	ldr	r2, [pc, #60]	; (800148c <rcc_osc_on+0x5c>)
 800144e:	6813      	ldr	r3, [r2, #0]
 8001450:	f043 6380 	orr.w	r3, r3, #67108864	; 0x4000000
 8001454:	e7f8      	b.n	8001448 <rcc_osc_on+0x18>
	case RCC_PLL3:
		RCC_CR |= RCC_CR_PLL3ON;
 8001456:	4a0d      	ldr	r2, [pc, #52]	; (800148c <rcc_osc_on+0x5c>)
 8001458:	6813      	ldr	r3, [r2, #0]
 800145a:	f043 5380 	orr.w	r3, r3, #268435456	; 0x10000000
 800145e:	e7f3      	b.n	8001448 <rcc_osc_on+0x18>
		break;
	case RCC_HSE:
		RCC_CR |= RCC_CR_HSEON;
 8001460:	4a0a      	ldr	r2, [pc, #40]	; (800148c <rcc_osc_on+0x5c>)
 8001462:	6813      	ldr	r3, [r2, #0]
 8001464:	f443 3380 	orr.w	r3, r3, #65536	; 0x10000
 8001468:	e7ee      	b.n	8001448 <rcc_osc_on+0x18>
		break;
	case RCC_HSI:
		RCC_CR |= RCC_CR_HSION;
 800146a:	4a08      	ldr	r2, [pc, #32]	; (800148c <rcc_osc_on+0x5c>)
 800146c:	6813      	ldr	r3, [r2, #0]
 800146e:	f043 0301 	orr.w	r3, r3, #1
 8001472:	e7e9      	b.n	8001448 <rcc_osc_on+0x18>
		break;
	case RCC_LSE:
		RCC_BDCR |= RCC_BDCR_LSEON;
 8001474:	4a05      	ldr	r2, [pc, #20]	; (800148c <rcc_osc_on+0x5c>)
 8001476:	6a13      	ldr	r3, [r2, #32]
 8001478:	f043 0301 	orr.w	r3, r3, #1
 800147c:	6213      	str	r3, [r2, #32]
		break;
 800147e:	4770      	bx	lr
	case RCC_LSI:
		RCC_CSR |= RCC_CSR_LSION;
 8001480:	4a02      	ldr	r2, [pc, #8]	; (800148c <rcc_osc_on+0x5c>)
 8001482:	6a53      	ldr	r3, [r2, #36]	; 0x24
 8001484:	f043 0301 	orr.w	r3, r3, #1
 8001488:	6253      	str	r3, [r2, #36]	; 0x24
		break;
	}
}
 800148a:	4770      	bx	lr
 800148c:	40021000 	.word	0x40021000

08001490 <rcc_set_sysclk_source>:
@param[in] clk Unsigned int32. System Clock Selection @ref rcc_cfgr_scs
*/

void rcc_set_sysclk_source(uint32_t clk)
{
	RCC_CFGR = (RCC_CFGR & ~RCC_CFGR_SW) |
 8001490:	4a03      	ldr	r2, [pc, #12]	; (80014a0 <rcc_set_sysclk_source+0x10>)
 8001492:	6853      	ldr	r3, [r2, #4]
 8001494:	f023 0303 	bic.w	r3, r3, #3
 8001498:	4303      	orrs	r3, r0
 800149a:	6053      	str	r3, [r2, #4]
			(clk << RCC_CFGR_SW_SHIFT);
}
 800149c:	4770      	bx	lr
 800149e:	bf00      	nop
 80014a0:	40021000 	.word	0x40021000

080014a4 <rcc_set_pll_multiplication_factor>:
@param[in] mul Unsigned int32. PLL multiplication factor @ref rcc_cfgr_pmf
*/

void rcc_set_pll_multiplication_factor(uint32_t mul)
{
	RCC_CFGR = (RCC_CFGR & ~RCC_CFGR_PLLMUL) |
 80014a4:	4a03      	ldr	r2, [pc, #12]	; (80014b4 <rcc_set_pll_multiplication_factor+0x10>)
 80014a6:	6853      	ldr	r3, [r2, #4]
 80014a8:	f423 1370 	bic.w	r3, r3, #3932160	; 0x3c0000
 80014ac:	ea43 4380 	orr.w	r3, r3, r0, lsl #18
 80014b0:	6053      	str	r3, [r2, #4]
			(mul << RCC_CFGR_PLLMUL_SHIFT);
}
 80014b2:	4770      	bx	lr
 80014b4:	40021000 	.word	0x40021000

080014b8 <rcc_set_pll_source>:
@param[in] pllsrc Unsigned int32. PLL clock source @ref rcc_cfgr_pcs
*/

void rcc_set_pll_source(uint32_t pllsrc)
{
	RCC_CFGR = (RCC_CFGR & ~RCC_CFGR_PLLSRC) |
 80014b8:	4a03      	ldr	r2, [pc, #12]	; (80014c8 <rcc_set_pll_source+0x10>)
 80014ba:	6853      	ldr	r3, [r2, #4]
 80014bc:	f423 3380 	bic.w	r3, r3, #65536	; 0x10000
 80014c0:	ea43 4300 	orr.w	r3, r3, r0, lsl #16
 80014c4:	6053      	str	r3, [r2, #4]
			(pllsrc << 16);
}
 80014c6:	4770      	bx	lr
 80014c8:	40021000 	.word	0x40021000

080014cc <rcc_set_pllxtpre>:
@param[in] pllxtpre Unsigned int32. HSE division factor @ref rcc_cfgr_hsepre
*/

void rcc_set_pllxtpre(uint32_t pllxtpre)
{
	RCC_CFGR = (RCC_CFGR & ~RCC_CFGR_PLLXTPRE) |
 80014cc:	4a03      	ldr	r2, [pc, #12]	; (80014dc <rcc_set_pllxtpre+0x10>)
 80014ce:	6853      	ldr	r3, [r2, #4]
 80014d0:	f423 3300 	bic.w	r3, r3, #131072	; 0x20000
 80014d4:	ea43 4340 	orr.w	r3, r3, r0, lsl #17
 80014d8:	6053      	str	r3, [r2, #4]
			(pllxtpre << 17);
}
 80014da:	4770      	bx	lr
 80014dc:	40021000 	.word	0x40021000

080014e0 <rcc_set_adcpre>:
@param[in] adcpre uint32_t. Prescale divider taken from @ref rcc_cfgr_adcpre
*/

void rcc_set_adcpre(uint32_t adcpre)
{
	RCC_CFGR = (RCC_CFGR & ~RCC_CFGR_ADCPRE) |
 80014e0:	4a03      	ldr	r2, [pc, #12]	; (80014f0 <rcc_set_adcpre+0x10>)
 80014e2:	6853      	ldr	r3, [r2, #4]
 80014e4:	f423 4340 	bic.w	r3, r3, #49152	; 0xc000
 80014e8:	ea43 3380 	orr.w	r3, r3, r0, lsl #14
 80014ec:	6053      	str	r3, [r2, #4]
			(adcpre << RCC_CFGR_ADCPRE_SHIFT);
}
 80014ee:	4770      	bx	lr
 80014f0:	40021000 	.word	0x40021000

080014f4 <rcc_set_ppre2>:
@param[in] ppre2 Unsigned int32. APB2 prescale factor @ref rcc_cfgr_apb2pre
*/

void rcc_set_ppre2(uint32_t ppre2)
{
	RCC_CFGR = (RCC_CFGR & ~RCC_CFGR_PPRE2) |
 80014f4:	4a03      	ldr	r2, [pc, #12]	; (8001504 <rcc_set_ppre2+0x10>)
 80014f6:	6853      	ldr	r3, [r2, #4]
 80014f8:	f423 5360 	bic.w	r3, r3, #14336	; 0x3800
 80014fc:	ea43 23c0 	orr.w	r3, r3, r0, lsl #11
 8001500:	6053      	str	r3, [r2, #4]
			(ppre2 << RCC_CFGR_PPRE2_SHIFT);
}
 8001502:	4770      	bx	lr
 8001504:	40021000 	.word	0x40021000

08001508 <rcc_set_ppre1>:
@param[in] ppre1 Unsigned int32. APB1 prescale factor @ref rcc_cfgr_apb1pre
*/

void rcc_set_ppre1(uint32_t ppre1)
{
	RCC_CFGR = (RCC_CFGR & ~RCC_CFGR_PPRE1) |
 8001508:	4a03      	ldr	r2, [pc, #12]	; (8001518 <rcc_set_ppre1+0x10>)
 800150a:	6853      	ldr	r3, [r2, #4]
 800150c:	f423 63e0 	bic.w	r3, r3, #1792	; 0x700
 8001510:	ea43 2300 	orr.w	r3, r3, r0, lsl #8
 8001514:	6053      	str	r3, [r2, #4]
			(ppre1 << RCC_CFGR_PPRE1_SHIFT);

}
 8001516:	4770      	bx	lr
 8001518:	40021000 	.word	0x40021000

0800151c <rcc_set_hpre>:
@param[in] hpre Unsigned int32. AHB prescale factor @ref rcc_cfgr_ahbpre
*/

void rcc_set_hpre(uint32_t hpre)
{
	RCC_CFGR = (RCC_CFGR & ~RCC_CFGR_HPRE) |
 800151c:	4a03      	ldr	r2, [pc, #12]	; (800152c <rcc_set_hpre+0x10>)
 800151e:	6853      	ldr	r3, [r2, #4]
 8001520:	f023 03f0 	bic.w	r3, r3, #240	; 0xf0
 8001524:	ea43 1300 	orr.w	r3, r3, r0, lsl #4
 8001528:	6053      	str	r3, [r2, #4]
			(hpre << RCC_CFGR_HPRE_SHIFT);

}
 800152a:	4770      	bx	lr
 800152c:	40021000 	.word	0x40021000

08001530 <rcc_clock_setup_in_hse_8mhz_out_24mhz>:
/** @brief RCC Set System Clock PLL at 24MHz from HSE at 8MHz

*/

void rcc_clock_setup_in_hse_8mhz_out_24mhz(void)
{
 8001530:	b508      	push	{r3, lr}
	/* Enable internal high-speed oscillator. */
	rcc_osc_on(RCC_HSI);
 8001532:	2004      	movs	r0, #4
 8001534:	f7ff ff7c 	bl	8001430 <rcc_osc_on>
	rcc_wait_for_osc_ready(RCC_HSI);
 8001538:	f7ff ff72 	bl	8001420 <rcc_wait_for_osc_ready>

	/* Select HSI as SYSCLK source. */
	rcc_set_sysclk_source(RCC_CFGR_SW_SYSCLKSEL_HSICLK);
 800153c:	2000      	movs	r0, #0
 800153e:	f7ff ffa7 	bl	8001490 <rcc_set_sysclk_source>

	/* Enable external high-speed oscillator 8MHz. */
	rcc_osc_on(RCC_HSE);
 8001542:	2003      	movs	r0, #3
 8001544:	f7ff ff74 	bl	8001430 <rcc_osc_on>
	rcc_wait_for_osc_ready(RCC_HSE);
 8001548:	f7ff ff6a 	bl	8001420 <rcc_wait_for_osc_ready>
	rcc_set_sysclk_source(RCC_CFGR_SW_SYSCLKSEL_HSECLK);
 800154c:	2001      	movs	r0, #1
 800154e:	f7ff ff9f 	bl	8001490 <rcc_set_sysclk_source>

	/*
	 * Set prescalers for AHB, ADC, APB1, APB2.
	 * Do this before touching the PLL (TODO: why?).
	 */
	rcc_set_hpre(RCC_CFGR_HPRE_NODIV);    /* Set. 24MHz Max. 72MHz */
 8001552:	2000      	movs	r0, #0
 8001554:	f7ff ffe2 	bl	800151c <rcc_set_hpre>
	rcc_set_adcpre(RCC_CFGR_ADCPRE_DIV2);  /* Set. 12MHz Max. 14MHz */
 8001558:	f7ff ffc2 	bl	80014e0 <rcc_set_adcpre>
	rcc_set_ppre1(RCC_CFGR_PPRE_NODIV);    /* Set. 24MHz Max. 36MHz */
 800155c:	f7ff ffd4 	bl	8001508 <rcc_set_ppre1>
	rcc_set_ppre2(RCC_CFGR_PPRE_NODIV);    /* Set. 24MHz Max. 72MHz */
 8001560:	f7ff ffc8 	bl	80014f4 <rcc_set_ppre2>
	 * Sysclk runs with 24MHz -> 0 waitstates.
	 * 0WS from 0-24MHz
	 * 1WS from 24-48MHz
	 * 2WS from 48-72MHz
	 */
	flash_set_ws(FLASH_ACR_LATENCY_0WS);
 8001564:	f000 f8c8 	bl	80016f8 <flash_set_ws>

	/*
	 * Set the PLL multiplication factor to 3.
	 * 8MHz (external) * 3 (multiplier) = 24MHz
	 */
	rcc_set_pll_multiplication_factor(RCC_CFGR_PLLMUL_PLL_CLK_MUL3);
 8001568:	2001      	movs	r0, #1
 800156a:	f7ff ff9b 	bl	80014a4 <rcc_set_pll_multiplication_factor>

	/* Select HSE as PLL source. */
	rcc_set_pll_source(RCC_CFGR_PLLSRC_HSE_CLK);
 800156e:	f7ff ffa3 	bl	80014b8 <rcc_set_pll_source>

	/*
	 * External frequency undivided before entering PLL
	 * (only valid/needed for HSE).
	 */
	rcc_set_pllxtpre(RCC_CFGR_PLLXTPRE_HSE_CLK);
 8001572:	2000      	movs	r0, #0
 8001574:	f7ff ffaa 	bl	80014cc <rcc_set_pllxtpre>

	/* Enable PLL oscillator and wait for it to stabilize. */
	rcc_osc_on(RCC_PLL);
 8001578:	f7ff ff5a 	bl	8001430 <rcc_osc_on>
	rcc_wait_for_osc_ready(RCC_PLL);
 800157c:	f7ff ff50 	bl	8001420 <rcc_wait_for_osc_ready>

	/* Select PLL as SYSCLK source. */
	rcc_set_sysclk_source(RCC_CFGR_SW_SYSCLKSEL_PLLCLK);
 8001580:	2002      	movs	r0, #2
 8001582:	f7ff ff85 	bl	8001490 <rcc_set_sysclk_source>

	/* Set the peripheral clock frequencies used */
	rcc_ahb_frequency = 24000000;
 8001586:	4b04      	ldr	r3, [pc, #16]	; (8001598 <rcc_clock_setup_in_hse_8mhz_out_24mhz+0x68>)
 8001588:	4a04      	ldr	r2, [pc, #16]	; (800159c <rcc_clock_setup_in_hse_8mhz_out_24mhz+0x6c>)
 800158a:	6013      	str	r3, [r2, #0]
	rcc_apb1_frequency = 24000000;
 800158c:	4a04      	ldr	r2, [pc, #16]	; (80015a0 <rcc_clock_setup_in_hse_8mhz_out_24mhz+0x70>)
 800158e:	6013      	str	r3, [r2, #0]
	rcc_apb2_frequency = 24000000;
 8001590:	4a04      	ldr	r2, [pc, #16]	; (80015a4 <rcc_clock_setup_in_hse_8mhz_out_24mhz+0x74>)
 8001592:	6013      	str	r3, [r2, #0]
}
 8001594:	bd08      	pop	{r3, pc}
 8001596:	bf00      	nop
 8001598:	016e3600 	.word	0x016e3600
 800159c:	2000000c 	.word	0x2000000c
 80015a0:	20000010 	.word	0x20000010
 80015a4:	20000014 	.word	0x20000014

080015a8 <rcc_periph_clock_enable>:
 * For available constants, see #rcc_periph_clken (RCC_UART1 for example)
 */

void rcc_periph_clock_enable(enum rcc_periph_clken clken)
{
	_RCC_REG(clken) |= _RCC_BIT(clken);
 80015a8:	2201      	movs	r2, #1
 80015aa:	0943      	lsrs	r3, r0, #5
 80015ac:	f103 4380 	add.w	r3, r3, #1073741824	; 0x40000000
 80015b0:	f503 3304 	add.w	r3, r3, #135168	; 0x21000
 80015b4:	6819      	ldr	r1, [r3, #0]
 80015b6:	f000 001f 	and.w	r0, r0, #31
 80015ba:	4082      	lsls	r2, r0
 80015bc:	430a      	orrs	r2, r1
 80015be:	601a      	str	r2, [r3, #0]
}
 80015c0:	4770      	bx	lr
	...

080015c4 <usart_set_baudrate>:
void usart_set_baudrate(uint32_t usart, uint32_t baud)
{
	uint32_t clock = rcc_apb1_frequency;

#if defined USART1
	if ((usart == USART1)
 80015c4:	4a06      	ldr	r2, [pc, #24]	; (80015e0 <usart_set_baudrate+0x1c>)
	uint32_t clock = rcc_apb1_frequency;
 80015c6:	4b07      	ldr	r3, [pc, #28]	; (80015e4 <usart_set_baudrate+0x20>)
	if ((usart == USART1)
 80015c8:	4290      	cmp	r0, r2
	uint32_t clock = rcc_apb1_frequency;
 80015ca:	681b      	ldr	r3, [r3, #0]
#if defined USART6
		|| (usart == USART6)
#endif
		) {
		clock = rcc_apb2_frequency;
 80015cc:	bf04      	itt	eq
 80015ce:	4b06      	ldreq	r3, [pc, #24]	; (80015e8 <usart_set_baudrate+0x24>)
 80015d0:	681b      	ldreq	r3, [r3, #0]
			+ ((clock % baud) * 256 + baud / 2) / baud;
		return;
	}
#endif

	USART_BRR(usart) = (clock + baud / 2) / baud;
 80015d2:	eb03 0351 	add.w	r3, r3, r1, lsr #1
 80015d6:	fbb3 f1f1 	udiv	r1, r3, r1
 80015da:	6081      	str	r1, [r0, #8]
}
 80015dc:	4770      	bx	lr
 80015de:	bf00      	nop
 80015e0:	40013800 	.word	0x40013800
 80015e4:	20000010 	.word	0x20000010
 80015e8:	20000014 	.word	0x20000014

080015ec <usart_set_databits>:
*/

void usart_set_databits(uint32_t usart, uint32_t bits)
{
	if (bits == 8) {
		USART_CR1(usart) &= ~USART_CR1_M; /* 8 data bits */
 80015ec:	68c3      	ldr	r3, [r0, #12]
	if (bits == 8) {
 80015ee:	2908      	cmp	r1, #8
		USART_CR1(usart) &= ~USART_CR1_M; /* 8 data bits */
 80015f0:	bf0c      	ite	eq
 80015f2:	f423 5380 	biceq.w	r3, r3, #4096	; 0x1000
	} else {
		USART_CR1(usart) |= USART_CR1_M;  /* 9 data bits */
 80015f6:	f443 5380 	orrne.w	r3, r3, #4096	; 0x1000
 80015fa:	60c3      	str	r3, [r0, #12]
	}
}
 80015fc:	4770      	bx	lr

080015fe <usart_set_stopbits>:

void usart_set_stopbits(uint32_t usart, uint32_t stopbits)
{
	uint32_t reg32;

	reg32 = USART_CR2(usart);
 80015fe:	6903      	ldr	r3, [r0, #16]
	reg32 = (reg32 & ~USART_CR2_STOPBITS_MASK) | stopbits;
 8001600:	f423 5340 	bic.w	r3, r3, #12288	; 0x3000
 8001604:	430b      	orrs	r3, r1
	USART_CR2(usart) = reg32;
 8001606:	6103      	str	r3, [r0, #16]
}
 8001608:	4770      	bx	lr

0800160a <usart_set_parity>:

void usart_set_parity(uint32_t usart, uint32_t parity)
{
	uint32_t reg32;

	reg32 = USART_CR1(usart);
 800160a:	68c3      	ldr	r3, [r0, #12]
	reg32 = (reg32 & ~USART_PARITY_MASK) | parity;
 800160c:	f423 63c0 	bic.w	r3, r3, #1536	; 0x600
 8001610:	430b      	orrs	r3, r1
	USART_CR1(usart) = reg32;
 8001612:	60c3      	str	r3, [r0, #12]
}
 8001614:	4770      	bx	lr

08001616 <usart_set_mode>:

void usart_set_mode(uint32_t usart, uint32_t mode)
{
	uint32_t reg32;

	reg32 = USART_CR1(usart);
 8001616:	68c3      	ldr	r3, [r0, #12]
	reg32 = (reg32 & ~USART_MODE_MASK) | mode;
 8001618:	f023 030c 	bic.w	r3, r3, #12
 800161c:	430b      	orrs	r3, r1
	USART_CR1(usart) = reg32;
 800161e:	60c3      	str	r3, [r0, #12]
}
 8001620:	4770      	bx	lr

08001622 <usart_set_flow_control>:

void usart_set_flow_control(uint32_t usart, uint32_t flowcontrol)
{
	uint32_t reg32;

	reg32 = USART_CR3(usart);
 8001622:	6943      	ldr	r3, [r0, #20]
	reg32 = (reg32 & ~USART_FLOWCONTROL_MASK) | flowcontrol;
 8001624:	f423 7340 	bic.w	r3, r3, #768	; 0x300
 8001628:	430b      	orrs	r3, r1
	USART_CR3(usart) = reg32;
 800162a:	6143      	str	r3, [r0, #20]
}
 800162c:	4770      	bx	lr

0800162e <usart_enable>:
usart_reg_base
*/

void usart_enable(uint32_t usart)
{
	USART_CR1(usart) |= USART_CR1_UE;
 800162e:	68c3      	ldr	r3, [r0, #12]
 8001630:	f443 5300 	orr.w	r3, r3, #8192	; 0x2000
 8001634:	60c3      	str	r3, [r0, #12]
}
 8001636:	4770      	bx	lr

08001638 <usart_send_blocking>:
usart_reg_base
@param[in] data unsigned 16 bit.
*/

void usart_send_blocking(uint32_t usart, uint16_t data)
{
 8001638:	b538      	push	{r3, r4, r5, lr}
 800163a:	4604      	mov	r4, r0
 800163c:	460d      	mov	r5, r1
	usart_wait_send_ready(usart);
 800163e:	f000 f80a 	bl	8001656 <usart_wait_send_ready>
	usart_send(usart, data);
 8001642:	4629      	mov	r1, r5
 8001644:	4620      	mov	r0, r4
}
 8001646:	e8bd 4038 	ldmia.w	sp!, {r3, r4, r5, lr}
	usart_send(usart, data);
 800164a:	f000 b800 	b.w	800164e <usart_send>

0800164e <usart_send>:
*/

void usart_send(uint32_t usart, uint16_t data)
{
	/* Send data. */
	USART_DR(usart) = (data & USART_DR_MASK);
 800164e:	f3c1 0108 	ubfx	r1, r1, #0, #9
 8001652:	6041      	str	r1, [r0, #4]
}
 8001654:	4770      	bx	lr

08001656 <usart_wait_send_ready>:
*/

void usart_wait_send_ready(uint32_t usart)
{
	/* Wait until the data has been transferred into the shift register. */
	while ((USART_SR(usart) & USART_SR_TXE) == 0);
 8001656:	6803      	ldr	r3, [r0, #0]
 8001658:	061b      	lsls	r3, r3, #24
 800165a:	d5fc      	bpl.n	8001656 <usart_wait_send_ready>
}
 800165c:	4770      	bx	lr

0800165e <blocking_handler>:

}

void blocking_handler(void)
{
	while (1);
 800165e:	e7fe      	b.n	800165e <blocking_handler>

08001660 <null_handler>:
}

void null_handler(void)
{
	/* Do nothing. */
}
 8001660:	4770      	bx	lr
	...

08001664 <reset_handler>:
{
 8001664:	b538      	push	{r3, r4, r5, lr}
	for (src = &_data_loadaddr, dest = &_data;
 8001666:	4a1a      	ldr	r2, [pc, #104]	; (80016d0 <reset_handler+0x6c>)
 8001668:	4b1a      	ldr	r3, [pc, #104]	; (80016d4 <reset_handler+0x70>)
		dest < &_edata;
 800166a:	491b      	ldr	r1, [pc, #108]	; (80016d8 <reset_handler+0x74>)
 800166c:	428b      	cmp	r3, r1
 800166e:	d31a      	bcc.n	80016a6 <reset_handler+0x42>
		*dest++ = 0;
 8001670:	2100      	movs	r1, #0
	while (dest < &_ebss) {
 8001672:	4a1a      	ldr	r2, [pc, #104]	; (80016dc <reset_handler+0x78>)
 8001674:	4293      	cmp	r3, r2
 8001676:	d31b      	bcc.n	80016b0 <reset_handler+0x4c>
	SCB_CCR |= SCB_CCR_STKALIGN;
 8001678:	f04f 22e0 	mov.w	r2, #3758153728	; 0xe000e000
 800167c:	f8d2 3d14 	ldr.w	r3, [r2, #3348]	; 0xd14
	for (fp = &__preinit_array_start; fp < &__preinit_array_end; fp++) {
 8001680:	4c17      	ldr	r4, [pc, #92]	; (80016e0 <reset_handler+0x7c>)
	SCB_CCR |= SCB_CCR_STKALIGN;
 8001682:	f443 7300 	orr.w	r3, r3, #512	; 0x200
	for (fp = &__preinit_array_start; fp < &__preinit_array_end; fp++) {
 8001686:	4d17      	ldr	r5, [pc, #92]	; (80016e4 <reset_handler+0x80>)
	SCB_CCR |= SCB_CCR_STKALIGN;
 8001688:	f8c2 3d14 	str.w	r3, [r2, #3348]	; 0xd14
	for (fp = &__preinit_array_start; fp < &__preinit_array_end; fp++) {
 800168c:	42ac      	cmp	r4, r5
 800168e:	d312      	bcc.n	80016b6 <reset_handler+0x52>
	for (fp = &__init_array_start; fp < &__init_array_end; fp++) {
 8001690:	4c15      	ldr	r4, [pc, #84]	; (80016e8 <reset_handler+0x84>)
 8001692:	4d16      	ldr	r5, [pc, #88]	; (80016ec <reset_handler+0x88>)
 8001694:	42ac      	cmp	r4, r5
 8001696:	d312      	bcc.n	80016be <reset_handler+0x5a>
	(void)main();
 8001698:	f7fe fdac 	bl	80001f4 <main>
	for (fp = &__fini_array_start; fp < &__fini_array_end; fp++) {
 800169c:	4c14      	ldr	r4, [pc, #80]	; (80016f0 <reset_handler+0x8c>)
 800169e:	4d15      	ldr	r5, [pc, #84]	; (80016f4 <reset_handler+0x90>)
 80016a0:	42ac      	cmp	r4, r5
 80016a2:	d310      	bcc.n	80016c6 <reset_handler+0x62>
}
 80016a4:	bd38      	pop	{r3, r4, r5, pc}
		*dest = *src;
 80016a6:	f852 0b04 	ldr.w	r0, [r2], #4
 80016aa:	f843 0b04 	str.w	r0, [r3], #4
		src++, dest++) {
 80016ae:	e7dd      	b.n	800166c <reset_handler+0x8>
		*dest++ = 0;
 80016b0:	f843 1b04 	str.w	r1, [r3], #4
 80016b4:	e7de      	b.n	8001674 <reset_handler+0x10>
		(*fp)();
 80016b6:	f854 3b04 	ldr.w	r3, [r4], #4
 80016ba:	4798      	blx	r3
	for (fp = &__preinit_array_start; fp < &__preinit_array_end; fp++) {
 80016bc:	e7e6      	b.n	800168c <reset_handler+0x28>
		(*fp)();
 80016be:	f854 3b04 	ldr.w	r3, [r4], #4
 80016c2:	4798      	blx	r3
	for (fp = &__init_array_start; fp < &__init_array_end; fp++) {
 80016c4:	e7e6      	b.n	8001694 <reset_handler+0x30>
		(*fp)();
 80016c6:	f854 3b04 	ldr.w	r3, [r4], #4
 80016ca:	4798      	blx	r3
	for (fp = &__fini_array_start; fp < &__fini_array_end; fp++) {
 80016cc:	e7e8      	b.n	80016a0 <reset_handler+0x3c>
 80016ce:	bf00      	nop
 80016d0:	080018c0 	.word	0x080018c0
 80016d4:	20000000 	.word	0x20000000
 80016d8:	20000018 	.word	0x20000018
 80016dc:	20001520 	.word	0x20001520
 80016e0:	080018c0 	.word	0x080018c0
 80016e4:	080018c0 	.word	0x080018c0
 80016e8:	080018c0 	.word	0x080018c0
 80016ec:	080018c0 	.word	0x080018c0
 80016f0:	080018c0 	.word	0x080018c0
 80016f4:	080018c0 	.word	0x080018c0

080016f8 <flash_set_ws>:

void flash_set_ws(uint32_t ws)
{
	uint32_t reg32;

	reg32 = FLASH_ACR;
 80016f8:	4a03      	ldr	r2, [pc, #12]	; (8001708 <flash_set_ws+0x10>)
 80016fa:	6813      	ldr	r3, [r2, #0]
	reg32 &= ~(FLASH_ACR_LATENCY_MASK << FLASH_ACR_LATENCY_SHIFT);
 80016fc:	f023 0307 	bic.w	r3, r3, #7
	reg32 |= (ws << FLASH_ACR_LATENCY_SHIFT);
 8001700:	4303      	orrs	r3, r0
	FLASH_ACR = reg32;
 8001702:	6013      	str	r3, [r2, #0]
}
 8001704:	4770      	bx	lr
 8001706:	bf00      	nop
 8001708:	40022000 	.word	0x40022000

0800170c <memcpy>:
 800170c:	4684      	mov	ip, r0
 800170e:	ea41 0300 	orr.w	r3, r1, r0
 8001712:	f013 0303 	ands.w	r3, r3, #3
 8001716:	d149      	bne.n	80017ac <memcpy+0xa0>
 8001718:	3a40      	subs	r2, #64	; 0x40
 800171a:	d323      	bcc.n	8001764 <memcpy+0x58>
 800171c:	680b      	ldr	r3, [r1, #0]
 800171e:	6003      	str	r3, [r0, #0]
 8001720:	684b      	ldr	r3, [r1, #4]
 8001722:	6043      	str	r3, [r0, #4]
 8001724:	688b      	ldr	r3, [r1, #8]
 8001726:	6083      	str	r3, [r0, #8]
 8001728:	68cb      	ldr	r3, [r1, #12]
 800172a:	60c3      	str	r3, [r0, #12]
 800172c:	690b      	ldr	r3, [r1, #16]
 800172e:	6103      	str	r3, [r0, #16]
 8001730:	694b      	ldr	r3, [r1, #20]
 8001732:	6143      	str	r3, [r0, #20]
 8001734:	698b      	ldr	r3, [r1, #24]
 8001736:	6183      	str	r3, [r0, #24]
 8001738:	69cb      	ldr	r3, [r1, #28]
 800173a:	61c3      	str	r3, [r0, #28]
 800173c:	6a0b      	ldr	r3, [r1, #32]
 800173e:	6203      	str	r3, [r0, #32]
 8001740:	6a4b      	ldr	r3, [r1, #36]	; 0x24
 8001742:	6243      	str	r3, [r0, #36]	; 0x24
 8001744:	6a8b      	ldr	r3, [r1, #40]	; 0x28
 8001746:	6283      	str	r3, [r0, #40]	; 0x28
 8001748:	6acb      	ldr	r3, [r1, #44]	; 0x2c
 800174a:	62c3      	str	r3, [r0, #44]	; 0x2c
 800174c:	6b0b      	ldr	r3, [r1, #48]	; 0x30
 800174e:	6303      	str	r3, [r0, #48]	; 0x30
 8001750:	6b4b      	ldr	r3, [r1, #52]	; 0x34
 8001752:	6343      	str	r3, [r0, #52]	; 0x34
 8001754:	6b8b      	ldr	r3, [r1, #56]	; 0x38
 8001756:	6383      	str	r3, [r0, #56]	; 0x38
 8001758:	6bcb      	ldr	r3, [r1, #60]	; 0x3c
 800175a:	63c3      	str	r3, [r0, #60]	; 0x3c
 800175c:	3040      	adds	r0, #64	; 0x40
 800175e:	3140      	adds	r1, #64	; 0x40
 8001760:	3a40      	subs	r2, #64	; 0x40
 8001762:	d2db      	bcs.n	800171c <memcpy+0x10>
 8001764:	3230      	adds	r2, #48	; 0x30
 8001766:	d30b      	bcc.n	8001780 <memcpy+0x74>
 8001768:	680b      	ldr	r3, [r1, #0]
 800176a:	6003      	str	r3, [r0, #0]
 800176c:	684b      	ldr	r3, [r1, #4]
 800176e:	6043      	str	r3, [r0, #4]
 8001770:	688b      	ldr	r3, [r1, #8]
 8001772:	6083      	str	r3, [r0, #8]
 8001774:	68cb      	ldr	r3, [r1, #12]
 8001776:	60c3      	str	r3, [r0, #12]
 8001778:	3010      	adds	r0, #16
 800177a:	3110      	adds	r1, #16
 800177c:	3a10      	subs	r2, #16
 800177e:	d2f3      	bcs.n	8001768 <memcpy+0x5c>
 8001780:	320c      	adds	r2, #12
 8001782:	d305      	bcc.n	8001790 <memcpy+0x84>
 8001784:	f851 3b04 	ldr.w	r3, [r1], #4
 8001788:	f840 3b04 	str.w	r3, [r0], #4
 800178c:	3a04      	subs	r2, #4
 800178e:	d2f9      	bcs.n	8001784 <memcpy+0x78>
 8001790:	3204      	adds	r2, #4
 8001792:	d008      	beq.n	80017a6 <memcpy+0x9a>
 8001794:	07d2      	lsls	r2, r2, #31
 8001796:	bf1c      	itt	ne
 8001798:	f811 3b01 	ldrbne.w	r3, [r1], #1
 800179c:	f800 3b01 	strbne.w	r3, [r0], #1
 80017a0:	d301      	bcc.n	80017a6 <memcpy+0x9a>
 80017a2:	880b      	ldrh	r3, [r1, #0]
 80017a4:	8003      	strh	r3, [r0, #0]
 80017a6:	4660      	mov	r0, ip
 80017a8:	4770      	bx	lr
 80017aa:	bf00      	nop
 80017ac:	2a08      	cmp	r2, #8
 80017ae:	d313      	bcc.n	80017d8 <memcpy+0xcc>
 80017b0:	078b      	lsls	r3, r1, #30
 80017b2:	d0b1      	beq.n	8001718 <memcpy+0xc>
 80017b4:	f010 0303 	ands.w	r3, r0, #3
 80017b8:	d0ae      	beq.n	8001718 <memcpy+0xc>
 80017ba:	f1c3 0304 	rsb	r3, r3, #4
 80017be:	1ad2      	subs	r2, r2, r3
 80017c0:	07db      	lsls	r3, r3, #31
 80017c2:	bf1c      	itt	ne
 80017c4:	f811 3b01 	ldrbne.w	r3, [r1], #1
 80017c8:	f800 3b01 	strbne.w	r3, [r0], #1
 80017cc:	d3a4      	bcc.n	8001718 <memcpy+0xc>
 80017ce:	f831 3b02 	ldrh.w	r3, [r1], #2
 80017d2:	f820 3b02 	strh.w	r3, [r0], #2
 80017d6:	e79f      	b.n	8001718 <memcpy+0xc>
 80017d8:	3a04      	subs	r2, #4
 80017da:	d3d9      	bcc.n	8001790 <memcpy+0x84>
 80017dc:	3a01      	subs	r2, #1
 80017de:	f811 3b01 	ldrb.w	r3, [r1], #1
 80017e2:	f800 3b01 	strb.w	r3, [r0], #1
 80017e6:	d2f9      	bcs.n	80017dc <memcpy+0xd0>
 80017e8:	780b      	ldrb	r3, [r1, #0]
 80017ea:	7003      	strb	r3, [r0, #0]
 80017ec:	784b      	ldrb	r3, [r1, #1]
 80017ee:	7043      	strb	r3, [r0, #1]
 80017f0:	788b      	ldrb	r3, [r1, #2]
 80017f2:	7083      	strb	r3, [r0, #2]
 80017f4:	4660      	mov	r0, ip
 80017f6:	4770      	bx	lr

080017f8 <memset>:
 80017f8:	0783      	lsls	r3, r0, #30
 80017fa:	b530      	push	{r4, r5, lr}
 80017fc:	d048      	beq.n	8001890 <memset+0x98>
 80017fe:	1e54      	subs	r4, r2, #1
 8001800:	2a00      	cmp	r2, #0
 8001802:	d03f      	beq.n	8001884 <memset+0x8c>
 8001804:	4603      	mov	r3, r0
 8001806:	b2ca      	uxtb	r2, r1
 8001808:	e001      	b.n	800180e <memset+0x16>
 800180a:	3c01      	subs	r4, #1
 800180c:	d33a      	bcc.n	8001884 <memset+0x8c>
 800180e:	f803 2b01 	strb.w	r2, [r3], #1
 8001812:	079d      	lsls	r5, r3, #30
 8001814:	d1f9      	bne.n	800180a <memset+0x12>
 8001816:	2c03      	cmp	r4, #3
 8001818:	d92d      	bls.n	8001876 <memset+0x7e>
 800181a:	b2cd      	uxtb	r5, r1
 800181c:	ea45 2505 	orr.w	r5, r5, r5, lsl #8
 8001820:	2c0f      	cmp	r4, #15
 8001822:	ea45 4505 	orr.w	r5, r5, r5, lsl #16
 8001826:	d936      	bls.n	8001896 <memset+0x9e>
 8001828:	f1a4 0210 	sub.w	r2, r4, #16
 800182c:	f022 0c0f 	bic.w	ip, r2, #15
 8001830:	f103 0e20 	add.w	lr, r3, #32
 8001834:	44e6      	add	lr, ip
 8001836:	ea4f 1c12 	mov.w	ip, r2, lsr #4
 800183a:	f103 0210 	add.w	r2, r3, #16
 800183e:	e942 5504 	strd	r5, r5, [r2, #-16]
 8001842:	e942 5502 	strd	r5, r5, [r2, #-8]
 8001846:	3210      	adds	r2, #16
 8001848:	4572      	cmp	r2, lr
 800184a:	d1f8      	bne.n	800183e <memset+0x46>
 800184c:	f10c 0201 	add.w	r2, ip, #1
 8001850:	f014 0f0c 	tst.w	r4, #12
 8001854:	eb03 1202 	add.w	r2, r3, r2, lsl #4
 8001858:	f004 0c0f 	and.w	ip, r4, #15
 800185c:	d013      	beq.n	8001886 <memset+0x8e>
 800185e:	f1ac 0304 	sub.w	r3, ip, #4
 8001862:	f023 0303 	bic.w	r3, r3, #3
 8001866:	3304      	adds	r3, #4
 8001868:	4413      	add	r3, r2
 800186a:	f842 5b04 	str.w	r5, [r2], #4
 800186e:	4293      	cmp	r3, r2
 8001870:	d1fb      	bne.n	800186a <memset+0x72>
 8001872:	f00c 0403 	and.w	r4, ip, #3
 8001876:	b12c      	cbz	r4, 8001884 <memset+0x8c>
 8001878:	b2ca      	uxtb	r2, r1
 800187a:	441c      	add	r4, r3
 800187c:	f803 2b01 	strb.w	r2, [r3], #1
 8001880:	429c      	cmp	r4, r3
 8001882:	d1fb      	bne.n	800187c <memset+0x84>
 8001884:	bd30      	pop	{r4, r5, pc}
 8001886:	4664      	mov	r4, ip
 8001888:	4613      	mov	r3, r2
 800188a:	2c00      	cmp	r4, #0
 800188c:	d1f4      	bne.n	8001878 <memset+0x80>
 800188e:	e7f9      	b.n	8001884 <memset+0x8c>
 8001890:	4603      	mov	r3, r0
 8001892:	4614      	mov	r4, r2
 8001894:	e7bf      	b.n	8001816 <memset+0x1e>
 8001896:	461a      	mov	r2, r3
 8001898:	46a4      	mov	ip, r4
 800189a:	e7e0      	b.n	800185e <memset+0x66>
 800189c:	54746547 	.word	0x54746547
 80018a0:	0d706d65 	.word	0x0d706d65
 80018a4:	000a      	.short	0x000a
 80018a6:	4155      	.short	0x4155
 80018a8:	0a0d5452 	.word	0x0a0d5452
 80018ac:	00          	.byte	0x00
 80018ad:	4c          	.byte	0x4c
 80018ae:	6465      	.short	0x6465
 80018b0:	616f6c46 	.word	0x616f6c46
 80018b4:	61550074 	.word	0x61550074
 80018b8:	7472      	.short	0x7472
 80018ba:	00          	.byte	0x00
 80018bb:	49          	.byte	0x49
 80018bc:	00454c44 	.word	0x00454c44
